:0400000500009AD984
:020000040000FA
:1000000048430020A964000001CA011001CA011080
:1000100001CA011001CA011001CA011001CA011070
:1000200001CA011001CA011001CA011001CA011060
:1000300001CA011001CA01103FCA01102149086814
:10004000C2430A600A680242FAD170471E490A6830
:10005000002AFCD1CA610860C8690028FCD00020D1
:10006000C86148687047194801686FF00202114082
:1000700041F40071016003211548816041F23001B3
:1000800041610121C160502141610121C1604FF4F2
:10009000CA6141610121C160016070470D48026879
:1000A0000A6082684A60C2688A60406B20F07840CB
:1000B00040F08050C86070477047014610220648E3
:1000C00001F000BD10100440001004400000046066
:1000D000004104404C1300501800002170470120DB
:0C00E00070470000200000000A00000033
:100100003C0000000000000000000000340100007E
:1001100000000000000000000100000000000000DE
:1001200000000000000000000000000001000000CE
:100130000000000008000000000000003400000083
:100140000000000000000000680100000000000046
:10015000000000000100000000000000010000009D
:100160000000000000000000080000000000000087
:1001700030000000000000000000000098010000B6
:10018000040000000000000001000000FFFFFFFF6E
:10019000FF00000001000000080000000000000057
:1001A0002C0000000000000000000000C40100005E
:1001B000040000000000000001000000FFFFFFFF3E
:1001C000FFFFFFFF080000000000000034050000F2
:1001D000E401000099A1011095A70110A5C201102A
:1001E00009B2011045B80110000000000000000035
:1001F0002F000000280000000000000000000000A8
:10020000140200000000000000000000FFFFFFFFDC
:1002100000000000080000000000000030050000A1
:100220003002000069C201106DC101101FC201102F
:1002300095BA011000000000000000002D00000031
:10024000300500005402000075C20110A9B601106B
:100250009DBF011049B60110000000000000000021
:100260002E0000002400000000000000000000003C
:1002700080020000000000000000000000000000FC
:100280000800000000000000240000000000000042
:1002900000000000A40200000000000000000000B8
:1002A0000000000008000000000000002400000022
:1002B0000000000000000000C80200000000000074
:1002C0000100000000000000080000000000000025
:1002D00000000000200300200400000000000000D7
:1002E000000000002000000070010000300000004D
:1002F0001C02000040030020040000000000000079
:10030000000000000C000000300400001800000095
:10031000400200004803002004000000000000002C
:100320000000000024000000480400001800000045
:10033000000000008803002004000000000000000E
:100340000000000010000000A00100002C000000D0
:10035000CC01000090030020040000000000000019
:1003600000000000200000006402000024000000E3
:10037000FFFFFFFFB00300200400000000000000AA
:100380000000000028000000880200002400000097
:10039000FFFFFFFFD8030020040000000000000062
:1003A00000000000580000003C0100003400000084
:1003B000FFFFFFFFE003002004000000000000003A
:1003C00000000000100000006004000018000000A1
:1003D000FFFFFFFFE8030020040000000000000012
:1003E000000000001C000000AC020000240000001F
:1003F000FFFFFFFFF00300200400000000000000EA
:100400000000000038000000F40100002800000097
:10041000FFFFFFFF58040020040000000000000060
:100420000000000054000000000100003C0000003B
:100430001800000000000000000000004004000060
:10044000080000000000000018000000000000008C
:100450000000000058040000080000000000000038
:100460001800000000000000000000007004000000
:10047000080000000000000001000000E864000027
:01048000007B
:100484000100000000000E0000000F003200000018
:10049400010000002803002000020000000000000A
:1004A40001CA011000000000000000000800000064
:1004B40000002300500300200100000098030020E6
:1004C4000800000000000000000000000000000020
:1004D400000000000000000001000000F8030020FC
:1004E400060000000100000060040020000000007D
:0C04F400000000000002000000000000FA
:0F0502002900010025002D002E002F000100010F
:1005140004000000D464000000000000000000009B
:10052400000001000000030087C40110380500002A
:10053400380500000000000090000000900000005A
:100544000000000098030020F95D00002000000076
:10055400C0640000E86200000DC30110911A00009D
:10056400931A000099C801109BC8011000000000F4
:100574008004000028620000406200001062000055
:090584000800090001000000015B
:10059000000000000000000000000000000000005B
:1005A000DD190000FD19000001190000271A0000E4
:1005B000491900001F1900007B190000531A0000A0
:1005C000715D0000BD5E0000C15E0000080000001B
:1005D0002400000018000000280000002000000097
:1005E0003C0000000C00000034000000DFF800F0C8
:1005F00049C10110DFF800F019C20110DFF800F066
:1006000041AC0110DFF800F0CDA00110DFF800F0E0
:1006100085C10110DFF800F0C1C20110DFF800F061
:10062000E3BF0110DFF800F0CDC10110DFF800F0EA
:100630003DC10110DFF800F0DDB20110DFF800F07D
:1006400085B00110DFF800F029AF0110DFF800F0ED
:1006500079B50110DFF800F0C1C10110DFF800F03A
:1006600009B70110DFF800F0D5C00110DFF800F085
:10067000E1B5011020B1082328220021FFF7D2BFE5
:10068000704720B1082330220021FFF7CFBF704709
:1006900038B500F091FF25680DB129682160FFF79A
:1006A000A9FF284632BD70B504460D4626680020D5
:1006B00028601EB9FFF79AFF25600DE0FFF796FF4F
:1006C00000E0366831680029FBD1AE4203D1FFF764
:1006D00091FF002070BD3560FFF78CFF012070BDD9
:1006E0000022DFF8541C01EB4211CB7F1B0605D51D
:1006F000B1F91C30834201D108467047521C082AC8
:10070000EFDB0020704770B50646FFF76FFFDFF89C
:10071000545C0446A87E01001AD0401EA876C0B2E0
:10072000B0B9082100F026FC96B1A86B703001F03A
:100730007CF800F010FE301AB0FBF1F1022938BF4E
:100740000121EC352846FFF765FF2846FFF766FFD5
:10075000204600F065BE10B50446207B00F00F0077
:1007600002280FD100F012FDA168081ADFF8F41B6F
:10077000896BC968800801F57A71814238BFB0F190
:10078000405F00D3002010BD38B5DFF84C0ADFF819
:100790004C2A0168DFF87C4C02EA0105E94301605C
:1007A000A90608D54068800605D54FF4005104F12C
:1007B0004C0001F062F815F4602F08D0206905F4B0
:1007C000602108432061002104F19C00D0E131BD8B
:1007D00070B5FFF70BFFDFF83C4C0646206910F4BC
:1007E000602F27D02069C5012D0EE80748BF0025DE
:1007F00006D4A80748BF012502D4680748BF0225D0
:10080000681D40B200F040FF2069012105F111028E
:100810009140884320613046FFF7ECFE04EB8500F1
:100820004668300009D0206800224FF00063691D3F
:10083000B04702E03046FFF7DDFE206930B104F139
:100840009C00BDE87040002101F017B870BD70B584
:10085000FFF7F4FBDFF80C5BDFF8BC4BAB6A02463A
:1008600090071DD4D3E90401104007D0EB629969C9
:10087000084398614FF4804100F07CFBA86A00288F
:1008800047D16E6A002E44D0F068A96B884224D00C
:1008900005F14C00BDE870404FF4805100F0EDBF11
:1008A0000BB9A86AEAE70020A862D3E904019E69AF
:1008B000024042F0020232439A61626982436261FD
:1008C000E26822EA0100E060194605F13000FFF716
:1008D000EAFE022100F04EFBE3E7B068FFF73BFFC2
:1008E000A86408B1A86CD8E0D6E9040162690243A3
:1008F0006261E26841EA0200E0600020E061B06805
:100900002060E0690028FCD005F12400FFF7C0FE5C
:10091000AE6270BD0020F6E6F8B506461446376EA6
:100920001D4607B1B847A00708D4D6E916012040F4
:1009300029400022914208BF904207D0C6E91A45DB
:1009400006F13800BDE8F240FFF758BEF1BDFEE702
:1009500080B500F082FFDFF8BC2A0146906BD26BB5
:10096000BDE80840104710B5DFF8A84A0FF2311172
:10097000E06B884202D101F099F8206404F14C0048
:10098000BDE81040042100F078BF80B5FFF756FBAA
:10099000DFF8881A084207D0BDE804404FF0005144
:1009A000DFF8100C00F069BF01BD70B5040073D012
:1009B000A168202001E04968401E79B1C2B26AB145
:1009C0000A8840F603039A421CBF40F604039A4289
:1009D000F1D1E0681822203001F084F8A0690021EC
:1009E000A1616168D9B140F00202E07F002300F00C
:1009F0000700012807D0022809D0042804BF0022DC
:100A00004FF0805306E000224FF0005302E0002236
:100A10004FF08043B4F91C10E0686568A847FFF701
:100A2000E5FDDFF840590646E88E401CC0F30B0098
:100A3000E8860020296BC87705F13000FFF728FE13
:100A40003046FFF7D7FDB5F93610E06800F1B8027F
:100A5000B2F90030994204BF297E00291CD1917857
:100A600009B9016811B90020907016E0AA6B1268EC
:100A700012F1010F10D0DFF8F42B1268B1FBF2F184
:100A8000022938BF01217030FFF7C4FDE068BDE8DE
:100A900070407030FFF7C2BD70BDBDE8704032E6F7
:100AA00038B50D46A807DFF8BC4816D5206BFFF710
:100AB0007CFF206B25F0020510B145F0020109E032
:100AC000680702D4606A002851D004F1EC0000F0FD
:100AD000ACFE042104F14C004AE0680747D5606A87
:100AE00008B1C068A063A06BDFF8E42A41680B7806
:100AF0001360126809788A421CBF8569002D05D0F1
:100B000000224FF000736FF0FF01A847022001F0B0
:100B10004DF9112001F05FF901206077A06BE17EB3
:100B2000007C084204BF0E2001F055F9A06BDFF8ED
:100B3000E81840688268002A04BFC068002804D012
:100B40000020C861DFF8D80A086040F2FF70DFF8C3
:100B5000D42A106000208861DFF8C00848610FF2D5
:100B60001900E0631920BDE83240FFF763BD31BDD5
:100B7000BDE8344000F081BE2DE9FF478046880083
:100B800040F1B580DFF8DC57A86B40684068010091
:100B900018BF8047A86BDFF88098406881680029FB
:100BA00004BFC168002914D0D9F81C100029FBD05B
:100BB0000021C9F81C108068010018BF8047A86B8D
:100BC0004068C068010018BF8047DFF8B40AFFF72B
:100BD0003DFA0020C9F81C0040F60A0ADFF8A40A12
:100BE000DFF8E07AC9F8000008F108040120FFF7F7
:100BF00075FA0FF25110E863A7F800A00020788082
:100C0000002100F0B0F900F0A7F9206806467180D5
:100C1000E97E09B1617A99B1018840F602029142F8
:100C200005D1318A4FF60F421140318204E0318BF9
:100C30004FF60F421140318300216172FFF73CFAF9
:100C400020686946FFF72AFA6846FFF736FA00E09F
:100C50000646706800281CBF01885145F8D17760AE
:100C600040F60301707B00F0F0007073686A8068E2
:100C7000008888421CBF40F60401884202D100204F
:100C8000286417E0208BA8B100206083E06108F1A0
:100C90002C00017801F0F0010170417801F0F001C1
:100CA00041F00101417008F120007860787B00F08C
:100CB000F0007873D9F81C000028FBD00020C9F898
:100CC0001C00012001F046FB012808D0707B00F0D9
:100CD000F00040F0010070730FF21900E8634FF666
:100CE000FF322068018A11400182C9F80000BDE886
:100CF000FF870000DFF8D009014200D170470120D2
:100D000010B501F027FB0128DFF8584608D10FF293
:100D10003500DFF80417E063DFF8A809086010BDAC
:100D2000DFF8481909683220B0FBF1F1022938BF19
:100D30000121EC342046FFF76DFC2046BDE8104051
:100D4000FFF76CBC2DE9FE4306460C466004DFF855
:100D5000145619D5FFF74AFCEE6AB769B9070ED4E5
:100D60006EB10021B161FFF745FC706848B1B6F97A
:100D70001C10F06876683A460023B04701E0FFF7A0
:100D800039FC24F48044E1E0A0070AD5286BFFF782
:100D90000CFE286B002824F0020401D044F0020469
:100DA000D4E0A00005F1800840F60909DFF81479C5
:100DB00071D5B068018840F60202914205D1028ADD
:100DC0002D2161F30912028204E0028B2D2161F3CF
:100DD00009120283286CB8B1042001F0BBFA98B163
:100DE00000F064FE296C814228BF401E401A718ABF
:100DF00011EB1030F06040F2D761A0F2EE20884293
:100E000024BF40F6C410F060D6F818C0BCF1000F43
:100E10001CBFDFF8BC188C450DD0787B0F21084231
:100E200004BF708C484506D100224FF000736FF468
:100E300080713046E0470022DFF89818404600F005
:100E40002FFD287F50B10220ADF800006846FFF763
:100E5000FDF8BDF80800A8820020287701206876F8
:100E6000A87E401CA87600206877686A18B119200F
:100E700000F019FD01E044F00204D6F81480B8F146
:100E8000000F05D000224FF0806300213046C0479C
:100E900024F000545AE095F8200024F0080628B108
:100EA000200703D5002085F820003CE020073CD532
:100EB000002068760120A8770020FFF70FF90FF2D5
:100EC000BD00DFF81418DFF86047E86300224046F1
:100ED00000F0E6FC297FE87E81F00101084202D1A2
:100EE0000120E8760FE0A86CB8B100F0DFFD296CB6
:100EF0006A6C401A02EB10306864A96CB0EBC11F39
:100F00000BD300206864A7F8009000F025F80020BB
:100F1000788000F028F8276003E04FF0005100F0DF
:100F200029F800202864344610E0A0040ED5AE6AEB
:100F3000002E1CBF7068002806D0B6F91C10F0689F
:100F4000766800222023B04724F4005414B12146CF
:100F500000F010F8BDE8F783787B00F0F00040F077
:100F6000010078737047387B00F0F0003873002080
:100F70007860704705F14C0000F07FBC70B5054605
:100F80000E46B007DFF8DC430BD5206BFFF70DFDF5
:100F9000206B08B1022129E0B0002DD54FF000519F
:100FA00024E0B00028D5FFF75EF8DFF83007DFF85F
:100FB0003067E063307818B905F13800FFF71EFBA1
:100FC000DFF8601600200860022000F085FE112086
:100FD00000F096FE287C10B90E2000F091FE002053
:100FE000E083B07840B10020B070042104F14C00DF
:100FF000BDE8704000F041BC70BD30B58DB000F070
:10100000ECFDDFF8E006DFF8E0460168DFF8545356
:1010100041F00201016001A8FFF72CFBA078DFF886
:10102000CC160790002301AA05F14C00FFF706FB40
:1010300001A8FFF726FB0020ADF81C0001AB2078CB
:10104000DFF89426099019210020009005F1800016
:10105000FFF7F8FA01A8FFF70DFBE078DFF890162C
:101060000790002301AA05F19C00FFF7E7FA01A809
:10107000FFF707FB0120ADF81C0001AB6078DFF83B
:10108000742609901A210020009005F1D000FFF786
:10109000D9FA00230022DFF8601605F1EC00FFF713
:1010A000D5FADFF83806E8630DB04FF6FF70A88276
:1010B000012028770020E875E8766877E88385F8CE
:1010C0002000286430BD2DE9F041DFF814660446A5
:1010D00030788EB00F4690461D4618B9FFF78DFF49
:1010E00001203070002F1CBF6760B8F1000F4BD09B
:1010F000C4F80880FFF77AFA7178002942D10121FB
:101100007170FFF777FA35B909A80FF2246114223C
:1011100000F0E8FC09AD286820606868E060287C81
:101120002074A868606101206074688A6082E86841
:10113000010018BFA061A02104F1200001F0C0F956
:101140000823242200216846FFF784FA01208DF845
:1011500018006A46002104F13800FFF77FFA0823DF
:10116000242200216846FFF751FA06946B460022BC
:10117000DFF8881504F17000FFF768FA20460EB01A
:10118000BDE8F081FFF736FA0020F8E738B5FFF741
:101190002DFA7449497E31B1DFF868150C68FFF704
:1011A00029FA204632BDFFF725FA00F07FFC10F542
:1011B0000030DFF8542541F10001A2FB0045DFF8C3
:1011C0000C0502FB015501690020221845EB0103C3
:1011D000184632BD000000000810044020000E0038
:1011E0002DE9F84F04460E4692469B46FFF7FEF95E
:1011F0005C4D8046B5F93400B5F93610401AC0F39D
:101200000B0008286FF0010944DAA88E401CC0F3D7
:101210000B00A886B5F93400ADF80000002046495F
:1012200001EB4017F97F090604D5401CC0B208281D
:10123000F5DB002704F1700000F0F7FABE6087F8D4
:101240001EA0C7F804B02021BDF80000B883FC60E0
:10125000DDE90A23DFF8B40410401940C7E90401AE
:10126000B8340020F87740F6FF76686A00283946DF
:1012700005F1240006D0FFF716FA30B100F05EF851
:1012800040464BE0FFF70FFA40B9A88E3018C0F384
:101290000B00A88600F070F948464AE000F04EF8CE
:1012A000E87F697E084208D0012085F820000020F0
:1012B000E8772877A87E401CA87600F05DF9A86A38
:1012C000002834D1687E18B1192000F0ECFA2EE025
:1012D000687F60BBFFF78AF90446A87F20B1DFF87A
:1012E00000140120887018E0B868FFF734FAA86489
:1012F000B8B100F030F8AA6C121AB2FBF1F2022A6F
:1013000023BFAA6C101AB0FBF1F10121EC3528467D
:10131000FFF780F92846FFF781F92046FFF76AF9C1
:1013200005E02046FFF766F90421FFF723FEBDF92B
:101330000000BDE8F28F0000F8050020BDF80000B5
:101340002080F87F40F08000F877A07810B100206E
:10135000A07028777047A86BDFF81013C068096881
:1013600070470000101A00202DE9F04106460F4694
:1013700014461D46FFF776F980463846FFF7B0F968
:10138000070003D14046FFF771F90AE0F87F072113
:10139000084209D04046FFF769F90721F87F084263
:1013A000FCD10220002116E07968DFF86403814255
:1013B00002D0796831667860C6E916454046FFF785
:1013C00055F94FF0FF3106F13800FFF71BF9002007
:1013D0003066D6E91A01BDE8F081DCB5DDE90667C3
:1013E0000446CDE90067180008BFDFF82433204623
:1013F000FFF7F6FE002803D500204FF00041DCBDCA
:101400000146204602B0BDE8D04002224FF0E04342
:10141000AAE70000101A002000100440020000405B
:10142000BDE87040FFF7E6B801E042F002022DE9A6
:10143000F843DFF8CC42606A0090894603271546DE
:10144000FFF7D4F819F1010F05F0010680460AD123
:10145000A06A002819BFA06AB0F91C90E08E00F1C4
:1014600001090020E0750FFA89F0FFF739F9010052
:1014700070D0A06A814205F0020525D1280003D072
:10148000606A0090002060620122C87FB240104371
:10149000C877FFF7E7F80746002E14BFDFF874029D
:1014A000DFF87402FEF7D2FD00F066F825B906E019
:1014B00000F055F800F05BF800980028F8D13846A5
:1014C000FFF7D4F8832747E0009A8A4204F1EC0042
:1014D00016D100F0AAF9280012BF0020606A006847
:1014E000606200F049F8009800F039F800F03FF829
:1014F000009818B32800F6D120E0009A12680092F4
:10150000009AEAB112688A42F7D100F08EF9009889
:1015100000681DB1009A0021116004E00168009A82
:10152000116000210160009003E000F018F800F065
:101530001EF800980028F8D100F01EF8832701E07B
:1015400000F01AF8607F38B9022104F14C0000F075
:1015500094F901E000F010F83846BDE8F283C07F4E
:10156000009940F00400C8776846FFF791B801463B
:1015700004F13000FFF797B84046FFF73BB838B5A5
:1015800000F01AF805465E48407E68B12046FEF736
:101590005DFD044600F04AF804F0FF00012801D187
:1015A000812032BD022032BD00F040F8012032BD62
:1015B000000000005C1A00200446FFF717B80A4636
:1015C0004F49896B884201D00320704709E0000031
:1015D000D02108400A464A49896B884201D003203D
:1015E000704700211046CAE770B545498A6B9042A2
:1015F0006FF07F0411D1487E78B1FEF7F7FF054602
:101600004648FEF723FD064600F010F806F0FF00FE
:10161000012802D13002001670BD204670BD0000C6
:101620005100070600000460001004402846FEF741
:10163000E1BF70B50E461546FEF7D8FF832430494A
:101640001EB1022E0DD005D30EE08A6A3AB1896A26
:10165000898B02E00A7F12B9898A298005E08024FB
:1016600003E0497E297000E003245BE0E80000000D
:1016700080B50846FFF734F800B1806802BD00006D
:101680000100070601010E0438B5FFF795FF1C495C
:10169000CA7D520702D58B7D9C420FD001228B8AD6
:1016A00002FA04F52B438B820C341D4B1D68A240BB
:1016B00025EA02021A601A6802B90A76BDE83240C9
:1016C000FEF798BF201B002004000020201B0020F4
:1016D0004F0900004F0800008B090000A10A00001C
:1016E000371D0020002009407061000051090000F2
:1016F000D1070000890700006709000015090000F4
:10170000101A00200430044000093D00F1EFFF9F53
:101710001909000001000204010001040100030492
:101720000C100440FEF766FF204670BD000000006C
:10173000FFFFFFFFC4090000000000004F09000088
:1017400001001A01DFF800F021B30110DFF800F00A
:1017500095C00110DFF800F00DA80110DFF800F0CF
:10176000BDBE0110FEE7DFF8FC00007D70476BE0B6
:1017700038B5FFF7FCFFDFF8F4500446A8680021F5
:10178000FFF7E4FF6969081AA969814238BF0020A0
:1017900084F3118832BD2DE9F041FFF7E8FFDFF84F
:1017A000CC500446A8680121FFF7D0FF0121A9838E
:1017B0000021E9836E6929682A68871B801A711ADB
:1017C000884204D20020A88384F311882BE084F39C
:1017D0001188002406E0A61931460120FFF7BAFF60
:1017E0003F1B0446A742F6D2FFF7C1FF8046E88BB5
:1017F000012804D131460020FFF7ACFF0446A96957
:1018000014F1010F08BF084603D0E01B814238BF26
:1018100008468119FFF7A2FF012028840020A88331
:101820002E6088F31188BDE8F08100218182DFF805
:101830003810C0684969884204D1DFF85800006850
:10184000FEF7ECBE70477047DFF84C100968EFF305
:10185000118081F311887047F6E7DFF84000806857
:1018600070470000A40100207801002078010020CA
:10187000616280F311882046704738B504460D46F2
:10188000FFF7EAFF616A2943FFF7F2FFBDE8324044
:10189000FFF758BFE4640000E4000000C801002026
:1018A000816042607047102804D3DFF80C101038B4
:1018B000C1F8000F7047000000E000E000F004BE37
:1018C000FFF7C2BFDFF89811C20744BF01220A60C8
:1018D000820744BF4FF480720A60400744BF4FF450
:1018E000803008607047DFF87C21C30748BF116073
:1018F000830748BF5160400748BF916070470000B0
:1019000010B504460020D4E90A2347F6906100F0A0
:1019100087FE0123994228BF4FF0FF3010BD10B55C
:101920000C4600F0B9F8011D201AB0F1004F05D89F
:10193000081BB0F1004F38BF8C4200D20C46214644
:10194000BDE810400120CEE72DE9F04180460A466F
:10195000D8E90A01D8E90C45A0FB026701FB027730
:10196000A6196F41340C002244EA07414046FFF7B4
:10197000D6FFC8E90E67BDE8F081F8B50646FFF767
:101980009FFF0446DFF8E050DFF8E0700120E861D7
:10199000FFF798FFF96A096A142088473069B0F5A3
:1019A000802F34BF0421010C0120FFF79CFF3A680F
:1019B0001268232100209047DFF8B410012008604E
:1019C000DFF8B400016821F4E02141F480310160C6
:1019D0000120286084F31188F1BD000000F066B892
:1019E00010B5DFF89000446800F006F86069A1695E
:1019F000BDE8104008470000012063E7F8B5044641
:101A00000D4600F053F8D4E90A6732463B4600F031
:101A100007FE3DB1A6FB002306FB013307FB0033A5
:101A2000C4E90C23F2BD10B5DFF83C00DFF84C40F0
:101A3000002101600121C16121602068FFF7DCFF06
:101A4000DFF848100968096A14208847206810BD2B
:101A5000000080B500F02AF8000C40EA014002BD09
:101A6000042009401820094000002443840100108C
:101A700080022443E4010020002009402C2009407A
:101A8000DFF81000C088704700000000B0010010AF
:101A9000FEE77047F00100200948016842680368CA
:101AA0009942FAD1100C40EA0140704710B5044A3F
:101AB000136850681468A3421946F9D110BD00009C
:101AC0000820094062B38B0708D0521E11F8013B71
:101AD00000F8013B00F024808B07F6D1830740F02B
:101AE000208000BF103A07D330B4B1E83810103A64
:101AF000A0E83810F9D230BC530724BFB1E8081071
:101B0000A0E8081044BF51F8043B40F8043BD2075A
:101B100024BF31F8022B20F8022B44BF0B7803704E
:101B20007047083A07D3B1E80810083A40F8043B78
:101B300040F804CBF7D25307E4E70000DFF800F0E9
:101B4000F5C00110DFF800F049BA011020B10823F8
:101B500024220021FEF75ABD704780B50120009075
:101B600009234FF400720021DFF8080700F015FE8A
:101B700001BD80B5002301223421DFF8F80600F012
:101B80001FFE00B10120C0B202BDDFF8EC06806884
:101B90007047DFF8E416401890F8ED007047002217
:101BA000022904D1012806D140F2EE2203E00128E7
:101BB00008BF4FF47A7210467047DFF8BC06D0F8C1
:101BC000DC007047DFF8B00690F8E61021B1D0F8DD
:101BD0000C01010018BF004770472DE9F041DFF804
:101BE000988608F1E1058AB0A879002861D1012022
:101BF000A871DFF88866DFF88876307B68717068D6
:101C0000C8F80C0101A8FFF7A1FF00200690ADF86D
:101C10001400079001AB00220FF2F54108F10C000F
:101C2000FEF714FD01AB00220FF2A15108F13000C4
:101C3000FEF70CFD01AB00220FF2D94108F1540070
:101C4000FEF704FDB16801208847DFF83806007808
:101C50007868C0F38154707B20B1032C02D101203D
:101C6000287003E0032C18BF022C16D1022000F0CC
:101C70009DF8032CDFF810160CBF4FF47A7042F277
:101C800010700968B0FBF1F108F15400FEF7C2FCD6
:101C900008F15400FEF7C2FC05E0012C03D100F06E
:101CA00063FAFFF75AFF386840075CBF002000F076
:101CB0007DF80AB0BDE8F08110B508B1140001D17B
:101CC000022010BD8160C26003610146DFF8A805F3
:101CD00000F090FD002010BD10B50446FEF786FC14
:101CE000DFF89415621892F8E8305B1E82F8E8304D
:101CF000DBB223B98A680123A3409A438A6066E075
:101D00002DE9F0410546FEF771FC8046DFF86815C5
:101D1000681890F8ED20521E80F8ED20D2B2002A0B
:101D20003FD10FF2A050DFF8644500EB85052E7817
:101D30006F88300615D52168096A384688472168BA
:101D4000896A384688472168096B38468847DFF832
:101D5000401501200860DFF83C0500688007FAD5CF
:101D600012E0700606D501EB87010020D1F80011C2
:101D7000884709E021688969384688472168496BA6
:101D8000384688470228F9D106F03F003F2818BF9F
:101D9000FFF7B6FF687800F03F003F2818BFFFF755
:101DA000AFFF4046BDE8F041FEF724BC10B5044645
:101DB000FEF71CFCDFF8C0148A680123A3401A4315
:101DC0008A60611891F8E820521C81F8E820BDE88B
:101DD0001040FEF70FBCF8B50646FEF707FC0446B8
:101DE000DFF89454701990F8ED104A1C002980F81F
:101DF000ED2039D10FF2CC4000EB8607387800F0A7
:101E00003F003F2818BFFFF7E6FF787800F03F005B
:101E10003F2818BFFFF7DFFF7E883878DFF86C7443
:101E200001060ED53968C969304688473968496A5C
:101E3000304688473968C96A3046884700F019F843
:101E400012E0400606D505EB86010120D1F800110D
:101E5000884709E039684969304688473968496BDD
:101E6000304688470128F9D12046BDE8F240FEF708
:101E7000C1BBDFF81C1401200860DFF818040068FB
:101E80008007FAD570472DE9F04F002483B04FF05A
:101E9000000A0128D04618BF012664D1DFF8D89384
:101EA000D9F8DC0001285DD10220C9F8DC00FFF779
:101EB00045FE0090012000F062F9060054D1FEF7C3
:101EC000D1FBDFF8D81301900C60012000F042FA3A
:101ED000012804D1002000F0A7F94FF0010ADFF833
:101EE000C013DFF8B4030C6000681120FFF751FE47
:101EF00008B14FF001081020FFF74BFE08B148F081
:101F000002080F20FFF745FE08B148F004080B2037
:101F1000FFF73FFEDFF8746320B13168096B4FF4BF
:101F2000806088470A20FFF734FE20B13168096BD2
:101F30004FF481608847DFF85813DFF86873DFF8E3
:101F400068B30120086048F020003168896988473B
:101F5000DFF858130120086099F80800C00707D57A
:101F6000012416E0042673E00120C9F8DC006CE0CF
:101F7000584600F061FC0546042DF9D0012D04D12E
:101F8000326A5268032158469047386880088000BA
:101F90003860002000F05CFCBF4800683068806B4F
:101FA000804754B9012D04D1326A52680121584644
:101FB0009047386840F0030038600120B849086055
:101FC00040463168496988470B20FFF7E2FD20B1A0
:101FD0003168C96A4FF4806088470A20FFF7D9FD4D
:101FE00020B13168C96A4FF481608847A84901204F
:101FF00008600020AD4908600320C9F8DC003168A2
:10200000496B404688470128F9D1042000F0B7F811
:10201000A24901200860A0480068A5480068800621
:10202000FBD5BAF1000F1CBF012000F0FDF800F055
:102030005BFD082000F0A3F806460120C9F8DC008B
:102040000198FEF713FB00F0D3FC0098FFF77AFD30
:102050003046BDE8FE8F38B50446FEF7C7FA0546A0
:102060002146854800F0DAFB28464BE030B50024D5
:1020700001288BB004D021D303281DD018D31DE034
:1020800001A8FFF763FD7C4D8A490694ADF8144022
:10209000079401AB012205F17800FEF7D7FA00940E
:1020A0000023854A2C2105F19C00FEF7CBFA05E0C0
:1020B00000F036FD044601E000F0D8FD20460BB0EC
:1020C00030BD00F054B938B5FEF790FA05466A48BD
:1020D00090F8E000012410B1FFF74BFD04462846BC
:1020E000FEF788FA204632BD38B5FEF77FFA624D1A
:1020F000044695F8E00020B100F080F9002085F852
:10210000E0002046BDE83240FEF774BA000000004F
:102110007047000010B582B0042000F01BF90228BF
:1021200018BF032807D100F01FF8FFF716FDBDE820
:1021300016400220D0E56148534900684E4CC0F378
:10214000815003280CBF4FF47A7041F2883009683F
:10215000B0FBF1F104F15400FEF75CFA04F1540015
:10216000BDE81640FEF75ABA032000901C234FF03A
:10217000405200213F4800F010BB0020704770B56E
:1021800004463D4E304600F02BFB002598B9304602
:1021900000F02CFB0646B068204207D03269F36895
:1021A0000021204698470546012D05D0304600F015
:1021B0001FFB0600EFD1284670BD414901280CBF26
:1021C00040F2FF70002008600020704770B5FEF7F5
:1021D0000DFA294E294D044696F8E00028B100F08A
:1021E0000DF968B1002086F8E0000220AD68A8472C
:1021F00006461020FFF7C3FF8EB10320A8470EE06C
:10220000214909683220B0FBF1F101B9012106F141
:102210003000FEF7FFF906F13000FEF7FFF9204627
:10222000BDE87040FEF7E6B938B501281ED100F0D0
:1022300091F801281CD000F0D7F80F4C124901206A
:1022400084F8E00032200968B0FBF1F505B90125FA
:1022500004F13000FFF7E9FA294604F13000FEF7F7
:10226000D9F904F13000FEF7D9F901E000F0E8F8FF
:10227000002032BD00A00C40E004002028610000D6
:10228000B03F00503D1D0020E8000000B8010010E4
:1022900028200860282008402C2009400C400940D4
:1022A00000022243242208400040034080010443EE
:1022B00014100940A92D0000792B0000B43F0050F4
:1022C000000004608F3F00008F3F01008F3F02003D
:1022D0008F3F0300903F00018F3F0101903F0002BC
:1022E000903F00038F3F01048F3F00058F120804C9
:1022F0008F3F00048F3F0006513F00007F3F0100E9
:102300003F3F04003F3F02003F3F01007F3F02008C
:1023100070B50446E00782B00D46624E05D5A8B2FE
:1023200000900023012200F011F8A00705D5A8B203
:1023300000900123022200F009F8600705D5ADB234
:10234000009502230C2200F001F873BD00213046F5
:1023500000F023BA0146042907BF1D234FF0C042F5
:102360001C234FF080524F48342100F029BA38B571
:102370000546FFF791FB4C4CA168401A4FF47A7167
:10238000484305EB104500F0E5FD2169401A48BFC0
:10239000404240F6B9318D4207D2062805DAA068DE
:1023A000E168814201D322685AB940494A68D2079C
:1023B0004FF4FA6017D4086800F0FF007D2148430D
:1023C00008E0081A3A494843000C00EB900090429C
:1023D00038BF1046C82801D2C82032BDB0F57A6F88
:1023E00088BF4FF47A6032BD80B501210320FFF72A
:1023F0008FFFFFF751FB2C49886001BD80B501209C
:10240000FFF7A8FF012819D0002301223421254815
:1024100000F0D6F998B100F026F8FFF73DFB22490D
:102420008B680A68C860A2EB9202C01A204B58431E
:10243000000C0860904238BF10460860012002BDC1
:1024400010B500210320FFF763FF0120FFF782FF93
:1024500008B100F008F8144CFFF71EFB606000F0B4
:1024600079FD206110BD1348006800F087BD10B5EC
:1024700011490A6811490968140424161B38444399
:10248000E41004EB2244120600FB00F312160906C6
:102490005A435843091604EBA222484302EBA040DA
:1024A00010BD000000A00C40141D0020AC3F0050E7
:1024B00040420F008000001090130050A410005004
:1024C000002200F077BD000010B54048046814F108
:1024D000010F08BF002400F0EFFD3D490020086017
:1024E00001203C4908603C49086000F0B5FF3B48CA
:1024F000006820B13A480068204600F01CF83949CD
:10250000394A00200860394801686FF31B411143C4
:10251000016037480168C1F30131012906D1016822
:10252000344A114041F400320260016032480068D0
:102530000028FBD110BD70B505463048012101606F
:102540002F4909680029FBD02E4C2F4AC021216059
:1025500053682E499B075DBF13681B0C43F0F003C3
:1025600072230B70002101639668304600F0AEFDC7
:102570003146284600F0DDFD2548816D89B240F2E4
:102580000F22914213D201680068C1F30361C0F3C6
:10259000034001B1491E072805D006280EBF0720B9
:1025A000801C00F00F0041EA00101A490870304604
:1025B00000F02EFE18490968C968022088474020AB
:1025C000206001201549086070BD00001C130050F8
:1025D000840460425C600C4008220443800128436C
:1025E000000120438C2108400000390148200340AD
:1025F00004000940FFFFFCFC0C0068421010094079
:102600009402224300600C40AC3F005056620840E8
:10261000BC12005002600840A00100109404604207
:102620001B4213D1094236D12AB18446B0FBF2F0E5
:1026300002FB10C2704700F07FBFFCD300220023D2
:1026400070470B000200002100207047904271EBA0
:10265000030CF6D370B5B1FA81F4B3FA83F52C1BF1
:10266000A340C4F1200532FA05F63343A2405FF0DF
:102670000046E64002E05B085FEA3202841A71EB32
:10268000030524BF204629467641F4D302000B00FF
:102690003000002170BD012ACFD970B5140C20D0B4
:1026A000B1FA81F4B2FA82F5C4F120046419B4F1EC
:1026B0002006D6D3B2405FF00044F440002502E08B
:1026C00052085FEA3303C61A71EB020E24BF30468C
:1026D000714664416D41F3D302000B0020002900D4
:1026E00070BD0C46B1FBF2F102FB11452D0445EA29
:1026F0001045B5FBF2F402FB145580B240EA0545E3
:10270000B5FBF2F002FB105240EA044070BD00003D
:1027100070B504460D46164600F0E2F9401E8041B1
:10272000C00F1A490A68002AFCD0012E02D0022EDE
:1027300002D003E0257002E0258000E02560012240
:102740000A6000281CBFBDE8704000F0CDB970BD24
:1027500038B504460D4600F0C3F9401E8041C00F55
:102760000A490A68002AFCD0012D02D0022D02D0AD
:1027700003E0247802E0248800E0246801220A6053
:1027800008B100F0B1F9204632BD000000800C40D5
:102790000B46114604221818BAE710B500EB4100A9
:1027A000102B144600F5007002D3103B001D240CC2
:1027B0000299994041EA0441BDE810400422A7E78C
:1027C00038B51D460818102D144602D3103D801C44
:1027D000240C0221FFF7BCFF204080B2E84032BD4C
:1027E000006800280CBF0120002070470068704777
:1027F0000068704738B504460D4600F09EFE002183
:102800002960616869606168002914BF0D602560F6
:102810006560FFE7BDE8324000F091BE0B684A6892
:10282000002B0CBF42605A604A680968002A0CBF3E
:102830000160116070470000006801074CBF042070
:1028400000F00300704700001628A8BF203870472A
:102850002DE9F84F06469348934C0068934D800746
:1028600004D50820A87192482060BFE000F072FBF8
:1028700080469048006800900027001700F1010989
:102880000098800208D4C8F13E00C0100928A8BFF3
:1028900008208145B8BF814687480068C0F30460BE
:1028A000FFF7D2FF824685480068C0F30440FFF777
:1028B000CBFF09EB0A011629A8BF152104DA6FF036
:1028C00009029142B8BF114601F01F027C4B42F44D
:1028D000F8521A807B4A126812F0030F18BF0127C2
:1028E000520748BF47F002070EB147F0040795F9B9
:1028F0000720A8EB0202052A02DAAA7997425DD0E6
:10290000A8F10F0C0026BCF1000FB64607F001023B
:1029100007F00403DFF8B09123D40CEB0C1C4FEA52
:102920002C2EBEF1080F28BF4FF0070E7646072E5B
:1029300028BF062609EB860A59F82660DAF804A0B3
:10294000AAEB060A0AF0FF0613B1CAF3072B5E448E
:102950005FEA877B44BFCAF3074B5E440AB106EBCC
:102960001A6659F82E9009F0FF0A13B1C9F307232C
:102970009A44BB0744BFC9F307439A440AB10AEB20
:10298000196A401AACEB0E220099AF717243803283
:102990000128B8BF0120342301F0FF0158430AEB9E
:1029A00012224843B0FBF2F0B0F5803F28BF4FF64B
:1029B000FF7008F30708A88085F80780434800687F
:1029C000A988286000201F2904D21F21A98004E0C3
:1029D0004908401CB1F5007FFAD20F39090940EAD5
:1029E000C1003B490843206000206060BDE8F18FD2
:1029F00010B53848006884B21CB300F0ABFA2B491C
:102A000091F90720904205DA6FF07F029042B8BF3B
:102A10001046C8718888844201D28C8010BD2B4A30
:102A200012680B68D21A921C202A28BF1F22231A70
:102A30005208D3401818B0F5803F28BF4FF6FF70FA
:102A4000888010BD2448026802B9704710B5234B36
:102A5000996801F04060B0F1406F21D011480468DE
:102A6000A4071DD45C68A4071AD404681B68C3F3C8
:102A700003531C331B0114F0050F06D09A420FD2EA
:102A80006FF005012140016010BD934208D20A0198
:102A900058BF44F00104490158BF44F004040460E5
:102AA00010BD00000000094030100940281D002022
:102AB000FDFDA400B43F0050B81200503C1100507E
:102AC0006E620840242208409C13005008200940F0
:102AD00000E7A4803410094028500940AC3F005062
:102AE000EFF3108072B67047EFF3108062B6704754
:102AF000DFF800F099C8011010B50C18FFF7F0FFCF
:102B0000401E8041C00FDFF8F0130A68002AFCD095
:102B1000246801220A6008B1FFF7E6FF204610BDD5
:102B200038B5DFF8D843DFF8D8132078897B002543
:102B300008430AD0FDF75AFDA178002906BF0121FC
:102B4000A1700125FDF756FD0DB1002032BD022018
:102B5000FFF72CF90E20FFF73EF9DFF8A803016814
:102B600009B1012032BDDFF8A0234021116001210D
:102B7000C1610020607032BD70B5DFF88C0382B097
:102B8000002101604821C160DFF8800300F1D80412
:102B9000A17A002968D00129DFF8742329D11068AF
:102BA0004BF2F5214843050ADFF868030068C0F3DB
:102BB0008140012806D100F0CDF9FFF758FC6843A9
:102BC00005EB9055607B10B10020607305E0D248A2
:102BD0000068000215EB10204508D0480560290C5C
:102BE000416001218160C648807B00283AD00520E1
:102BF00039E0022909D11568284600F0FDF8A5F250
:102C0000FF5003282ED308202DE003292CD1116872
:102C100000F1B805A1F5C0612868E961002848BF46
:102C20004042002948BF49428842A8BF002018DA24
:102C30006868BB4E80B2009008234FF47F42302179
:102C40003046FFF7AAFDA86800F072F9042130466B
:102C5000FFF7A3FDA86900F071F93046FFF79DFD6D
:102C6000012020700B202073BDE873402DE9F04156
:102C7000A64CDFF8AC82AB4FAB4EA34804F1E105A4
:102C800082B0E9784A1E0B2A00F28080DFE802F069
:102C9000062233465B33465B3346636EA3490968BD
:102CA0000968202088470F20F860072341F61D504F
:102CB00038614FF4C0720220009000F070F80723D2
:102CC0004FF4C07200214046FFF77AFD01203060CA
:102CD000022044E00120F861287800281DBF002070
:102CE000306103200620E870032038600020706007
:102CF0007068800734D4E878032804D1022000F0FB
:102D00004BF8042007E0002000F046F8E878062899
:102D10000CBF07200A20E87001201AE0042903D123
:102D20002021B961012105E00122BA610A290CBF05
:102D3000032102216970002139600821C16001600E
:102D40000120386026E005290CBF06200920E87024
:102D50000020706004E00020306070600C20E8709B
:102D600004F17800BDE8F641FDF758BC0021016090
:102D70000120644908600E20FEF7C2FF0220FEF722
:102D8000ABFF0120E8700020A87003E0BDE8F3412C
:102D9000FFF7AEBEBDE8F38100900523602200215D
:102DA0004046FFF7FABC000080B558495E4891F8EC
:102DB000E410891E0A291AD8DFE801F0060A0E1964
:102DC0000A0E190A0E19120001688907FCD510E0D5
:102DD00041688907FCD40CE041688907FCD508E00C
:102DE00001688907FCD441688907FCD401E0FFF73A
:102DF0007FFEBDE8014039E7F8B50746484C302171
:102E00002046FFF779FE414E06F1B805C0F30720D2
:102E1000686004212046FFF76FFEC0F38440A8607D
:102E200020212046FFF768FEC0F38120A861B7F596
:102E3000C060286002D186F8D800F1BD296996F8F3
:102E4000D8202AB96A68A968EA60E861AA696A6153
:102E5000E86900284CBF6FF00102022200EB40003D
:102E60001018421000EB927001EBA0006968E96055
:102E7000012810DA6A69032A04D1153001281DDA05
:102E800001201BE00B300128B8BF0120491E48BFBC
:102E90000021E96007E01F2812DB6A692AB91538AA
:102EA0001F28A8BF1E20032109E00B381F28A8BF38
:102EB0001E20491C4029A8BF3F21E960002169610B
:102EC00028610823E86880B200904FF47F423021E7
:102ED00000F03CF80120009011234FF4003200F084
:102EE00034F8286900F024F800F02FF8686900F041
:102EF00025F800F02BF8F1BD00800C40C105002042
:102F00002861000004800C402C500C40E00400209C
:102F100008400C40B43F0050102009403C600C4079
:102F200000A00C4000400C4034600C40A001001098
:102F300080B2009012234FF4F802704780B20090E4
:102F40000A234FF440622021704704212046FFF7F6
:102F500024BC00000748084A81681278006852B211
:102F6000A0F54070C9035043C913A1EB2010803075
:102F700000127047285009400C13005070B50446E9
:102F8000FFF7AEFD451EAD41ED0F074E306800283E
:102F9000FCD0A04701203060002D1CBFBDE8704070
:102FA000FFF7A2BD70BD000000800C4062F30F224D
:102FB00062F31F4200B500BF1300964694461039D5
:102FC00028BFA0E80C50FAD85FEA417C28BF0CC0AB
:102FD00048BF40F8042BC90728BF20F8022B48BF80
:102FE00000F8012B00BD000030480068000C00F024
:102FF0000700052828BF4FF0FF3070472C490A68AA
:10300000C2F30F324BF69A139A424FF0FF3006D1BB
:103010000868000F0B280CBF0420002070474BF6F7
:10302000BE118A4201D1012070474BF641318A42DC
:1030300001D1032070474BF620318A4208BF02209D
:10304000704700001A48F8B50068050F1948006875
:1030500000F0FF06802E28BF0026FFF7CFFF0428D0
:103060004FF0FF3406F10A071DD8DFE800F0031225
:103070001A1A1B00012D12D0032D06D0072D06D0E1
:10308000082D08BF06F116040DE014240BE01524EA
:1030900009E025B1022D08BF06F1140403E00A245B
:1030A00001E005B93C4660B2F2BD00009412005048
:1030B00018130050A010005080B5FFF79FFF20B9F3
:1030C000FFF7C0FF162800DB01BDFEE7DFF8E813BD
:1030D0000968C1F304611629A8BF203901EB2071EA
:1030E000491C1629A8BF152104DA6FF00902914284
:1030F000B8BF114601F01F01DFF8C02341F4F851B9
:103100001180DFF8BC13096889074FBF40F04060A9
:103110000021DFF8B0231160DFF8AC13C0F3C06208
:1031200082F00102C0F380600A6080F001008860D4
:10313000704770B5054682B0084600F0EEF80246CA
:10314000DFF88843182100F060F800F012F980B22F
:103150000090002340F2FF322C212046FFF71DFB98
:10316000DFF86C63F068C0F30D021C2100F04DF82D
:10317000706800F0FC32142100F047F83068DFF886
:103180005413DFF8546301EA0002102100F03DF807
:10319000284600F0F8F802460C2100F036F82846E0
:1031A00000F01CF9400040F020003072284600F08A
:1031B0001EF940F010003072284600F021F9024656
:1031C000282100F022F8284600F0FFF8400040F0E7
:1031D0006000F072284600F02DF9C00040F0800039
:1031E0003070284600F02FF98000BC4940F47C4044
:1031F0000880284600F011F90246082100F005F881
:10320000B7494FF48000086073BD2046FFF7C0BA8D
:10321000F8B5810C01F003010129B24CB04D02D088
:1032200002292AD026E0216A8A0323D44FF480425F
:103230002A606FF08F06AC4AD2F8023033404E0A53
:1032400006F080063343C1F303363343C2F802303D
:10325000C1F30326D2F801301B0946EA0313C2F872
:1032600001306FF0E7061368334001F0E7011943BE
:10327000116002E04FF0004129609C4E9C4AB16809
:1032800009075CBF4021A9624FF400712964800DD9
:10329000216AC90C01F0030141F0300110F0030074
:1032A000117003D0022826D008D326E00121042083
:1032B000FFF72EF88F4800F0F0F822E00120FFF72A
:1032C00049F8074639460420FFF722F80420FFF7A3
:1032D00041F8B842FAD1366826F07F4000F0DDF8B8
:1032E000854B1B681B684FF060220721300E984702
:1032F0004FF480602860032100E002210420FFF7E2
:1033000007F820687D4900F03F00087047F6180074
:103310007B4908807B480068F1BD7B490968C1F39F
:1033200083628303C1F38F2120D4000400164FF67B
:10333000FF7307E0490804D11946520804BF01226F
:103340000121401C0028F5D401280FDB490041F081
:103350000101B1F5803F21BF0121520042F001027D
:10336000102A24BF0F221946401EEDE741EA024011
:1033700070476548016800680002C1F3870100F4E6
:1033800040700843704730B5604C61490A68656811
:10339000ED07C2F30351C2F303430AD424682505A1
:1033A00001EB2571240481F3040103EB247383F3FF
:1033B00004031B0443EA015193B21943222824BF9A
:1033C00002F080400143084630BD0021202803D38D
:1033D00050480068C0F30151084670470121222877
:1033E00003D34D480068C0F30071084670470121BF
:1033F000222803D348480068C0F34071084670474C
:103400000021202807D343480068C10C01F4407113
:10341000C0F3845001430846704720283F4907D332
:103420003C483F4A0068810A02EA003040EA815184
:10343000084670470021222803D337480068C0F3AC
:10344000C061084670470021222803D33248006833
:10345000C0F3455108467047324800680028FBD148
:103460003148324A416812688908890041F00051A8
:1034700041F00401520748BF41F001010BD402683A
:1034800012F0030F07D041F003024260026802F01D
:103490000302032AFAD141607047254982B20A60CB
:1034A000C0F3074048600120886022480068002877
:1034B000FBD0002088607047B81200506E62084050
:1034C0000000094094042A430000204300A00C405F
:1034D00070130050FFFFFC0041A10C40DCA10C4028
:1034E00040A00C406C1300500A600840A83F0050F8
:1034F00008A10C40BD378600B40100100BB00C4091
:1035000070B00C402C20094050130050AC3F0050CC
:1035100078130050981300508C13005000803F40E7
:1035200000F03F000C00684200400340B03F0050F4
:103530003C600C4084088C437047FDF757B8FDF79A
:1035400059B80000DFF800F0D9C10110DFF800F031
:10355000ADB50110DFF800F019AE0110DFF800F092
:10356000E5C10110DFF800F085C20110DFF800F0BE
:1035700081C20110DFF800F055C10110DFF800F042
:1035800043C20110DFF800F079AB0110DFF800F062
:10359000D9B60110DFF800F0EDB3011020B1082317
:1035A0002C22002100F012BD704720B108233C22DC
:1035B0000021FFF7C7BF704780B5FEF7BFFAADF82F
:1035C0000000FDF713F8ADF80200009802BD01B548
:1035D000BDF80200FDF70EF8BDF80000BDE802409E
:1035E000FEF7B0BA38B5DFF8A008DFF8A018DFF8AA
:1035F000A04880088000091A2161E060034602E0CB
:10360000002523F8025B0D18AB42F9D38B0800EBC1
:103610008303002223F8042CE82202804FF6FC7278
:103620001140EC39A0F8E810E8306060002000F0AC
:1036300004F8A060E068606031BDF8B500240025A2
:10364000061D16F003001CBF311D0E1AFFF7B4FF54
:10365000DFF83C28B6B21060112EB4BF57689768E7
:103660003A88130403D582F4004200251AE02B00A7
:1036700014D0238839880B4423809BB2B34211D3E2
:1036800027461A46B7B1921B92B2042AA7BFBA5373
:1036900046F40041398841F4004109E0B242F1DAD0
:1036A00001253C4617443A88002ADAD1002701E078
:1036B00027F8041BFFF78BFF3846F2BD10B5044610
:1036C000FFF77AFFDFF8C817086034F8042CC2F35C
:1036D0000E0224F8042C221F4B689A4238BF4A601D
:1036E000BDE8104073E738B50446FFF765FF0021D9
:1036F0000C23DFF8A0274B43D518AA6C4AB194429B
:1037000004D1FFF764FF05F1480032BD491C0329CD
:10371000EED3FFF75CFF002032BD70B50546FFF722
:103720004BFF044600200C22DFF8681742438E1836
:10373000B16C49B900203065B5640022FFF706FF7F
:10374000F06418B900F04CFC8D4205D12046FFF71B
:103750003EFF06F1480070BD401C0328E3D320461D
:10376000FFF735FF002070BD38B50446FFF724FF92
:103770000025DFF820170C226A438A5A130008D06C
:10378000944203D1FFF723FFE8B232BD6D1C062D32
:10379000F1D3FFF71CFFFF2032BD10B5044620888F
:1037A000FFF7E2FFFF2800D16BE10C22DFF8E416FF
:1037B000504308448168080002D16FF0010010BD39
:1037C0002046BDE81040084702460FF23870104707
:1037D00010B500200C21DFF8BC26002401FB00F30B
:1037E0001344401C03289C641C65F7D3002000236D
:1037F00001FB00F4401C13530628F9D30820108065
:103800000FF2E9609060BDE81040EBE670B590B053
:10381000FEF794F904466846FFF7C7FE05200690B8
:10382000002240F2B6300890694649F6D92004904B
:10383000DFF864060590DFF86406FFF78BFE0500ED
:1038400006D0FFF7B9FE06462846FFF766FF08B91F
:1038500000F0C6FB3046FFF7BAFE2046FEF772F9CD
:1038600010B070BDF8B500F0E6F8FFF756FF0500A0
:103870006FF0020616D0FFF79FFEA28800210C27EA
:10388000DFF810364F433B441F883FB91A805D6014
:10389000A2689A60217369682161C4E2BA4203D1C7
:1038A000FFF795FE3046F2BD491C0629E7D300F02C
:1038B00097FB00BF38B500F0BEF8FFF72EFF0500FC
:1038C00016D0FFF779FE00210C23DFF8C8254B4303
:1038D0001A4413884BB94FF6F873138055600023D0
:1038E000936021716968A16013E7491C0629EBD335
:1038F00000F076FB00BF10B5044660680C3080B263
:10390000FFF79BFE00B91AE06168018100210160A8
:10391000FF2181720C30A060002010BD80B540688E
:103920000C3811E080B288E610B50446606880B2B9
:10393000FFF783FEA06000B901E0002010BD6FF02A
:10394000030010BD80B54068FFF7B8FE002002BD3F
:1039500038B504460D46FFF72FFE002145F80C1C34
:10396000216811B9256006E0114651F80C2C002A97
:10397000FAD141F80C5CBDE8324028E62DE9F0416F
:1039800004466FF00206E068A0F10C05A079062855
:10399000BCBF207906280BDAFFF70EFEA179DFF80D
:1039A000F4840C2779434144496819B9FFF70FFEA5
:1039B000304617E0FFF70BFE20792871A079687177
:1039C000207AA871A079E1687843404440680830C3
:1039D000FFF7BEFFA0797843404440684068FCF799
:1039E0000DFE0020BDE8F08170B500F024F8FFF76F
:1039F0007AFE060002D16FF0040070BDFFF7DCFD17
:103A0000B168002541B10D46A5F10C010A68B2600C
:103A100000220A60FF228A72FFF7D9FD2800A56004
:103A200001D1022070BDA5F10C000179217140790E
:103A3000A071002070BD0446FFF790BD06280ADA89
:103A40000C23DFF850245843105A02001CBF4FF6D5
:103A5000F872904202D14FF0FF307047088000208A
:103A60007047811D0079E9E710B50446E088FFF74B
:103A70007BFEFF2800D104E0A0712046BDE8104085
:103A80007CE74FF0FF3010BD3EB50446FFF7ACFFBA
:103A9000050017D120796946FFF7D0FF78B10820DB
:103AA000ADF804000320ADF80600DFF8F413A068B9
:103AB0008968029001A888476FF005003EBDBDF8F7
:103AC0000000A08028463EBD10B5DFF8D82312685C
:103AD0000C464FF47A71A1FB00010023FEF7A0FD14
:103AE000002399424FF0004201D8904202D36FF078
:103AF000020010BD2060002010BD38B5FFF79BFF0D
:103B0000FFF7F1FD0546FDF72EFE002818BF01283E
:103B100000D015B96FF0040032BD606840B9009064
:103B200000996868FCF76EFD401E8041C00F32BDF1
:103B300010F1010F08BF4FF0FF30F0D06946FFF7DA
:103B4000C3FF0028ECD032BD80B54068FCF756FDBD
:103B5000002002BD00F044FA00BF80B54068FFF7C6
:103B600001FD002002BD80B54068FFF7FFFC00208A
:103B700002BD80B5FFF7FEFCFFF700FD002002BD8F
:103B800080B5FDF7DBFFFCF731FD002002BD10B56D
:103B90008CB004466846FFF701FDE02000F013F802
:103BA00008B900F01DFA0BE010B58CB00446684669
:103BB000FFF7F4FCE06800F006F808B900F010FA2E
:103BC00000200CB010BD08900023A16860686A4610
:103BD000FFF7D8BC10B50446FFF7D8FC60600020A2
:103BE00010BD0146886849680847F0B507468BB0A4
:103BF000BC68AB4D6CBB0C20FFF71FFD04006FF0E1
:103C000003061ED008232422002101A8FCF7FEFC95
:103C10000020ADF814000690079400237968A248AC
:103C200001AAFFF7B7FC206068B90820ADF80000D2
:103C30000C20ADF802006846A96888472046FFF7C7
:103C40003DFD304618E0F86860603869A060BC60EF
:103C50000AE02868804706462068FDF7E6FD3869D7
:103C6000A06030466968884779682068FCF7D2FC14
:103C70002068FCF7D3FC00200BB0F0BD10B5044663
:103C800082B060686946FFF71FFF20B90098606046
:103C90002046FFF7AAFF16BD80B5406810B96FF047
:103CA000020002BD0068FDF7C0FD002002BD7D4995
:103CB000096841600020704750B5044679480268A1
:103CC0006FF00046A6FB020100234FF47A72FEF764
:103CD000A7FC002399424FF0004201D8904200D344
:103CE00030466060002050BD2DE9F04186B00646A8
:103CF000FFF734FCFFF7F7FC044600200290002594
:103D0000FDF731FD002818BF012800D014B96FF06D
:103D1000040063E0706820B110F1010F03D14FF08F
:103D2000FF30009004E06946FFF7CEFE070054D153
:103D3000FFF72CFC0099012701EB000800E0009040
:103D400000996068FCF75EFC78B303A8FFF74CFEAF
:103D500007001AD19DF8100001A9FFF76FFE80B986
:103D6000059A9DF81210BDF80400B368984740B159
:103D7000BDF80400B0819DF81200B0730598306161
:103D800013E0059902A8FFF7E3FD009801276D1CD9
:103D900010F1010F18BF0028D2D0FFF7F7FBB8EBE6
:103DA000000002D000998142C9D2029EFFF704FCB4
:103DB00056B1314600E0114651F80C2C002AFAD1D8
:103DC000A26841F80C2CA660FFF701FC002D03E06F
:103DD0006068FCF713FC6D1EFAD1384606B0BDE8EA
:103DE000F081F8B5FFF727FE0546FDF7BCFC00287B
:103DF00018BF01286FF0040613D0FFF7DDFB002188
:103E0000244A0C234B43D75A4FB113445B681B68B9
:103E1000AB4201D1217106E0491C0629F1D3FFF71D
:103E2000D6FB3046F2BDFFF7D2FB0020F2BDF8B55D
:103E30000446FDF798FC002818BF012802D16FF056
:103E40000400F2BDFFF78AFB0546FFF7B5FB002132
:103E5000104A0C234B43D65A37000ED0A788BE42D7
:103E600008D1D11849680968A9420CBF0121002175
:103E7000A160D8E7491C0629EBD3FFF7A8FB4FF058
:103E8000FF30F2BD00000000441D0020483F00202C
:103E9000E413002078130020F0020020C93700004E
:103EA000DC020020E8000000E33B000070B504469F
:103EB0003C20FFF7C2FB05006FF0030611D0FFF7AF
:103EC00074FB207AA8610022608928622946E06894
:103ED00028616068FFF73EFB04462846FFF7EEFBCB
:103EE0000CB9304670BD002070BD000041882D29FE
:103EF00002D36FF0010070470FF2140252F8211044
:103F0000084700009B370000B9350000CF3500009E
:103F100065380000B5380000F73800001D39000092
:103F200029390000453900007D390000E9390000D9
:103F3000693A0000893A0000FB3A0000493B000062
:103F4000553B00005B3B0000673B0000733B0000FB
:103F5000813B00008F3B0000D53B00007D3C000012
:103F6000AF3C0000B93C0000633A0000DB5B00009E
:103F7000AF5C0000E93C0000E33D0000EB3B0000CB
:103F8000993C0000495C0000815C0000955C0000E9
:103F90002F3E0000E15C0000F95C0000AD3E000037
:103FA0000000000000000000EF5C0000075D000062
:103FB000A93B00000000000000000000000000001D
:103FC00000000000DFF800F0F1C5011001B901495F
:103FD000FFF7F8BFA0010000DFF800F0ED8C011042
:103FE0000120FFF7F9BF0000DFF800F061C2011007
:103FF000DFF800F0E9C20110DFF800F0E1C20110C3
:10400000DFF800F0B9C20110DFF800F0F9BF0110CD
:1040100050F8382F11430160704750F8382F22EACA
:10402000010101607047817DFF291DBFC07DFF2810
:1040300001200020704738B50446FCF7D7FA054642
:10404000207820B90220FDF7B1FE012020700BE09E
:1040500038B50446FCF7CAFA0546207820B102209C
:10406000FDF73AFE002020702846BDE83240FCF7FC
:10407000C1BA4068D030FCF7C1BA4068EC30FCF7F8
:10408000BDBA70B5446885680E4606E0206A401CDB
:104090002062761E606A401C60624EB1206ADFF8C2
:1040A0008828126801782868926990470028EDD125
:1040B000304670BD70B5456886680C4608E0296BCF
:1040C0000870641E286B401C2863686B401C686382
:1040D0002CB100F01AF8884710F1010FEFD12046FB
:1040E00070BD70B5456886680C4605E0C1B205F143
:1040F000400000F088FC641E2CB100F006F88847F0
:1041000010F1010FF2D1204670BDDFF81C180968CC
:1041100030680969704770B5446804F584750E46C7
:104120002846FDF782FB217F627FDFF800080068E8
:104130005118C91D7143DFF8F8275143A269B1FB3B
:10414000F2F141186331B1FBF0F0411C2846FCF755
:1041500061FA2846BDE87040FCF760BAF8B504463D
:104160006568A76805F584763046FDF75EFB38681C
:104170008069000711D5DFF8B41709684FF4FA70A9
:10418000B0FBF1F1022938BF01213046FCF742FAB9
:104190003046BDE8F240FCF741BADFF89807FFF778
:1041A00057FF38682021FFF738FF00F080FA00F051
:1041B00077FA01B0BDE8F040184738B504460D461F
:1041C00020212868FFF729FF297D606E01221BF05E
:1041D000F5F8297D606E01221BF00AF9297D606ED9
:1041E00000221BF02CF9A97D606E00221BF027F93C
:1041F000A078012804D1286880690007FBD405E075
:104200004FF0FF3104F1D000FCF7FCF900F0A6FB01
:104210002846FFF708FF30B1A97D606EBDE8384041
:1042200011221BF00CB931BD2DE9F0478046002664
:10423000D8F808502A68D8F80490146C546409F12E
:1042400028073869FB69D7F820C014F4F06F0146DD
:10425000A3EB0C0A34D0600518D5101D026802F0DB
:104260000F06002202602129ACBF20250D462946F9
:1042700000F05DF8C5F120015145C8BF51464046E8
:10428000FFF72FFF16E03869401E3861386988B1A2
:10429000012100F04CF8286850F8041F01F00F06C7
:1042A0000021002E0160EED0B868401EB860F868AA
:1042B000401EF86089F81F60404600F07BFA25E058
:1042C000620609F19C050AD5E1B100F030F83861C9
:1042D000787908B13E6111E0386900280DE0E20606
:1042E00014D579B1397D4E1E864228BF0646314627
:1042F00000F01DF83869801B386107D12846FDF7AA
:1043000021FA03E051464046FFF7EBFEA0060CD52C
:104310003D6855B129464046FFF7B3FE386020B9E5
:10432000291D4046BDE8F047F5E6BDE8F087404668
:10433000C0E638B50446DFF800066568FFF788FE7A
:1043400056E2406800210170DFF8EC050170417011
:104350007047F0B504468DB06568A6680F46FCF757
:1043600045F92978002944D101212970FCF742F947
:104370003878687000217878A87078686860B868C4
:10438000A860F868E86038692861387D2875787D0C
:104390006875B87DA875B869A861387F2877787F77
:1043A0006877B87FA8770020286205F12C0041606B
:1043B00069628160A962C16001704170102101745D
:1043C000002141747068FDF706FD204600F01AFADE
:1043D000204600F069FA80B9DFF84C1509683068AA
:1043E000C96888477068FDF78BFCFCF7FFF800216F
:1043F0002970FCF7FFF8002064E008233022002138
:1044000001A8FCF713F9069401AB307BDFF82C25EB
:1044100009900020009005F18000B168FCF712F9C6
:1044200008232822002101A8FCF7FCF805940023AA
:104430003069DFF80C15079001AA05F19C00FCF724
:10444000FDF808232422002101A8FCF703F901202C
:104450008DF81C00A87840B901AA002105F1D00010
:10446000FCF7FCF8DFF8DC042861687840B901AAA1
:10447000002105F1EC00FCF7F1F8DFF8CC04E8606E
:1044800008232422002101A8FCF7C0F80020069090
:10449000ADF81400079401AB0A22DFF8B01405F55B
:1044A0008470FCF7D3F8F269B16905F1400000F0BF
:1044B00083FA23460FF2B142042105F16C00FDF7A7
:1044C000FBFB20460DB0F0BD38B544688568606ED2
:1044D0001AF065FF286840F2F271FFF79EFDDFF8E1
:1044E000481409682868C96888476868FDF708FCA7
:1044F00004F18000FFF778FD04F19C00FFF778FDE0
:10450000A07818B904F1D000FFF776FD607818B9EB
:1045100004F1EC00FFF770FD04F58470FFF770FD07
:10452000FCF764F800212170FCF764F804F16C00DA
:10453000BDE83240FDF78FBD70B5024620295468B2
:104540006FF0010004D023D3222909D004D370BD19
:10455000012084F82D001AE0002084F82D0070BDA1
:104560009668FCF743F80546FFF7CFFD884710F142
:10457000010FF9D104F1380000210161C168491E21
:1045800041610021816101602846FCF733F8002079
:1045900070BD2DE9F84304466668A76889469046D1
:1045A000FCF724F80546B06A18B12846FCF722F853
:1045B00043E006F58470FDF738F90020F07770626B
:1045C000C6F820902846FCF715F8DB4D681CFFF76D
:1045D00032FDDFF87C03016841F480710160204600
:1045E0004146FFF74EFDB06206F1D00958B9414689
:1045F0002046FFF790FDB07820BBB1684846FCF735
:1046000001F8E8B90FE038682021FFF701FDB07824
:10461000C0B9B1684846FBF7F5FF88B94146204666
:10462000FFF779FD0020B06239461020F077304660
:10463000FFF7C3FD681CFFF70BFD4FF0FF3002E0F2
:10464000706A00E00020BDE8F283B0E070B5044677
:104650006568A668FBF7CAFFA96A39B93168896934
:1046600009075CBFBDE87040FBF7C4BF0021A96229
:10467000FBF7C0FF3046FFF7D6FC18B1314628469D
:10468000FFF79BFD30682021FFF7C7FC00F00FF813
:10469000A848FFF7DDFC00F003F8BDE870401847BC
:1046A0006A6A286A2B69811A296220467047A848DD
:1046B000016821F48071016070472DE9F84381465B
:1046C0008846D9F80850D9F80440286817464FF4AE
:1046D000FA61FFF7A2FC04F13006B06820B100F0E7
:1046E00061F84FF0FF305BE0B760271DF876C6F841
:1046F000008070600CE031689DF800000870306840
:10470000401C30607068401C7060B068401EB06033
:10471000B068002837D0694604F1400000F056F92F
:104720000028E8D5DFF810924846FFF784FC884857
:10473000016841F4007101604FF4FA612868FFF7E5
:1047400067FC607880B9396804F1EC00FBF75AFF28
:1047500028BBB0604846FFF77BFC30687168401AA0
:1047600030601020F8761AE094F82D0000281CBF65
:104770007068002805D00020B06004F19C00FCF7B0
:10478000E1FF00200CE000F00DF872683068811A3B
:1047900031606078012802D1BB684846984770684C
:1047A000BDE8F28328684FF4FA6131E400BF4FF0AE
:1047B000FF30704738B504464FF4FA61A068656869
:1047C0000068FFF72AFC6248016821F4007101606B
:1047D0005948FFF73DFCFBF709FFA96B002904BF0F
:1047E000BDE83240FBF706BF0021A963FBF702FFDB
:1047F0006A6B286BEB68811A2963204601B0BDE81B
:1048000030401847F0B587B0044602A80FF268118F
:10481000454E1422FDF766F96568A4683168206882
:10482000C968884740F2F27720683946FFF7F5FB00
:10483000206805F13C01476402AB4A780978C90851
:1048400053F82110114341636846FFF7DDFB05F182
:1048500018000FF23811027951F822100FF23C12B1
:10486000437952F82320837935686D6811430FF23C
:10487000341252F8232042EA0103026801992068A9
:10488000A847344D286840F010002860686840F060
:10489000010068602046FFF7C6FB18B1686840F465
:1048A0004040686007B0F0BD2DE9F04186B08568F2
:1048B0004468687DDFF8A08040F0004000906E46BC
:1048C000287D48EA0000706008272846FFF7ABFB08
:1048D00040B1A87D40F00040B0601027E87D48EA74
:1048E00000000390FE20B851694604F158001AF008
:1048F000EEFC6066A0B1697D0F221AF0A0FD00F009
:104900002DF82846FFF78FFB48B1A97D606E112274
:104910001AF095FDE97D606E12221AF090FD0120DB
:1049200006B0BDE8F0810000D0010010E8000000F2
:1049300040420F003C1D00203B1D0020294200008A
:1049400033430000734000007B4000005D410000E5
:10495000301000402C1000400000C0A0297D606E87
:1049600010221AF06CBD000080B5042804BF104668
:10497000FFF748FF002002BD000000000800000013
:1049800010000000180000002000000000000000DF
:104990002000000040000000600000000000000057
:1049A00008000000000000000600000002000000F7
:1049B00086000000820000000160426000218160EA
:1049C000511EC160002101614161704738B500F09E
:1049D00016F8A16801B92FE021682269515C29709D
:1049E00021696268491CB1FBF2F302FB13112161DA
:1049F000A168491EA160FBF7FDFDA06832BD044619
:104A00000D46FBF7F3BD38B5FFF7F9FF6168A26803
:104A10008A4211D0E268521CB2FBF1F301FB132170
:104A200022688D54E160A1686269491CA1608A42D4
:104A300038BF0A466261DEE7FBF7DCFD4FF0FF306E
:104A400032BD0000DFF800F025B10110DFF800F002
:104A50002DBF0110DFF800F0A9C10110DFF800F050
:104A600013C10110DFF800F011BF0110DFF800F0F2
:104A700021B9011000B583B000F00DF8032114E056
:104A8000E0B500F008F8042100F012F808B10020A9
:104A90000EBD02980EBD0821ADF8001001907047C0
:104AA00000B583B0FFF7F7FF052100F001F807BD5F
:104AB000ADF802106846DFF8C413096808472DE90D
:104AC000F04784B0DFF8B483DFF8B453DFF8B463A1
:104AD000DFF8B4730EE0B869FBF790FDB8884107C2
:104AE00008D54FF6FB710840B88000F0D7F808B938
:104AF00000F0D7F8B8694FF0FF31FBF783FD30685D
:104B00008047FA883B89B9881A437B891A43114345
:104B1000B9800021F9803981798129688847B8886E
:104B2000010603D54FF67F710840B8800820ADF824
:104B300000000920ADF802006846D8F80010884748
:104B4000002801BF029C9DF806003978884231D1C7
:104B5000396A080007D0B878012802D002281BD093
:104B600001E02046884720461AF0BEFC040021D010
:104B70000C20FFF785FF5FEA000919D030688047F5
:104B80008246C9F80840207848B9F8684946FFF7D6
:104B90005DFF00F086F807E0204688470AE04846B7
:104BA000FFF77EFF00F01AF929685046884701E0B8
:104BB00000F014F93879C0062ED500F06FF8F8B976
:104BC0001AF0EEFDE0B930688047044600F066F860
:104BD00098B9F868FFF73EFF5FEA00090DD0D9F8F1
:104BE00008104868786149881AF014FED9F808005E
:104BF000FFF756FF4846FFF753FF296820468847CE
:104C000000F04CF828B1B8884FF6EF710840B88032
:104C100002E0B869FBF7F2FC387980070DD51AF08D
:104C200095FC00F068F928B9B8884FF6FD71084086
:104C3000B88002E0B869FBF7E1FC387900072CD5B1
:104C40003869FFF70BFFE8B93869FFF70BFF04007D
:104C500018D0F96938780A001CBF7A78002A0CD07D
:104C6000022A01D002D30BE0A06804E0A16800F0A2
:104C700098F8A068F969884702E0A16800F091F807
:104C800000F0ACF83869FFF7E9FE00283FF423AFE5
:104C9000B8884FF6F7710840B8801FE7F868FFF74B
:104CA000DDBEB88840F01000B880B869FBF7A6BC3C
:104CB00010B5754C0020A080606186B00021FFF720
:104CC000D5FEE06000210020FFF7D0FE2061082023
:104CD000ADF800000020ADF802003820ADF8040067
:104CE0000020664909680290684688479DF80C00D4
:104CF00020700498A0610FF209101AF0ECFB0FF27B
:104D000095120FF259110FF2D9001AF031FDFFF789
:104D1000D6FE06B010BDCBE730B55C4C20604FF43A
:104D200000758FB0DD22294604F15400FEF73EF9EC
:104D300008233C2200216846FEF704FC04F15400DD
:104D4000079008950220069000236A465049201DCE
:104D5000FFF778FE0FB030BD70B51AF0C5FB044602
:104D60000C20FFF78DFE0546464800688047002C62
:104D700018BF002D06460ED0AC60207858B9424CC2
:104D8000E0682946FFF762FEA08840F01000A0808E
:104D9000A069FBF733FC3046BDE87040384909682C
:104DA000084730B585B00C468DF804000821374817
:104DB0000068ADF80600ADF8001000208DF808007E
:104DC000ADF8021060682D4909680390684688476D
:104DD000054600F003F8284605B030BD20465FE6E2
:104DE00010B5294C606918B1FFF744FE00206061DE
:104DF0000420E080A069BDE81040FBF7FFBB000085
:104E0000F8B504460D4616460C20FFF739FE074656
:104E10000820FFF735FE002F18BF00281CD0456082
:104E20004480B8607EB90021174C01703946206972
:104E3000FFF70CFEA08840F00800A080A069BDE844
:104E4000F240FBF7DBBBFFF72BFE3846FFF728FEEF
:104E50002846BDE8F2400DE6F1BD000010B504465D
:104E600000F059F8844208DAA0B200F01DF80648B4
:104E700002214181BDE8104012E0FEE7E40200207B
:104E8000E0020020DC020020801700202C1500200A
:104E9000174D0000004801E08017002080210181AB
:104EA0008069FBF7ABBB0000F8B52C4C2C4F0646D5
:104EB000608800258119B1F5877F08DDC0F5877509
:104EC000A9B238181AF08FFC0020761B6080B1B2AE
:104ED000608838441AF087FC6088301880B24FF43C
:104EE000877190FBF1F14FF4877202FB1100608033
:104EF000A81980B2F2BD194841880088081A00F547
:104F000087704FF4877190FBF1F14FF4877202FBC9
:104F1000110080B2704780B5FFF7EDFFC0F58770D4
:104F200080B202BDF0B50D4B0D4D1C8800220EE085
:104F3000A4B24FF487772E5D00F8016B641CA4B215
:104F40004FF4877694FBF6F607FB1644521C96B294
:104F50008E42EDD31C800846F0BD0000301D0020BD
:104F60001C140020E0B50821ADF8001001900221CA
:104F700000F00FF808B100200EBD02980EBD00B57C
:104F800083B00821ADF800100190032100F001F872
:104F900007BDADF802106846DFF8901209680847AF
:104FA0001FB5ADF806108DF804000824DFF87C1258
:104FB0008DF808200393ADF80040ADF80240684634
:104FC0000968884704B010BD30B585B01446082282
:104FD0000291ADF800201922DFF850120968019003
:104FE000ADF802201D466846884714B1BDF80C1084
:104FF000218015B19DF80E102970089A049911604E
:1050000005B030BD00B583B00820ADF800001A200F
:1050100000F015F810B99DF804000EBDFF200EBD7C
:1050200000B583B0ADF800008DF80610002000F048
:1050300006F810B99DF807000EBDFF200EBDDFF881
:10504000EC110968ADF802006846084750B110F14C
:10505000040F01D10420704710F1030F01D1022089
:105060007047012070478123037042EAC111002379
:1050700041F47C41C370818070478223037081803A
:105080000023C370827170473EB504460820ADF816
:1050900000000D462020ADF802001020DFF88C1132
:1050A0000968ADF804006846884720B9029810B135
:1050B0006FF004003EBD00950023002221464FF012
:1050C000FF30FFF781FF3EBD10B582B01446CA78AD
:1050D000012A03D18A88DFF8A0311A8000F010F885
:1050E00058B9009069462046FFF7CEFF28B90098CE
:1050F0004478FFF744FF204616BDFFF7A7FF16BD13
:105100000B46022210214BE7F8B500F0BBF800F087
:10511000ACF807000DD032462946FFF7AEFF00F08D
:10512000A0F83872FFF76EFF3B4601B0BDE8F040D3
:1051300021E0F1BD10220121E6E71022FFE7002166
:10514000E2E7002204215CE00420BDE8F08110B514
:1051500000F0B0F804000AD0112200F00AF8FFF7BE
:1051600051FF2146BDE81040DFF81021ACE70420D4
:1051700010BD022181E70222102111E70022032144
:105180003FE000B583B00FF249030193062300937B
:10519000032300F04DF80EBD1078802802BF508820
:1051A00040F27F61884208D19088984202BF91798D
:1051B0000098814201D1012070470020704710B54E
:1051C00082B00624FFE70094FFF7E6FF16BD00005B
:1051D0000323F4E71078802802BF508840F27F61F3
:1051E00088420CD19088032818BF042807D19079F1
:1051F00001001CBF1028112801D101207047002098
:105200007047F8B500F04DF807000CD0324629463B
:10521000FFF733FFBC60FFF7F5FE3946BDE8F84005
:10522000DFF85C2050E70420F2BD0000E40200201B
:105230002DE9F04100F00EF807000AD0069A414629
:10524000FFF71BFF3C817D8100F041F8079A00F0D9
:1052500034B879E704460D46164698461020FFF705
:1052600081BE21465020FFF7DBBE0A20FFF77ABE41
:1052700004460C20FFF776BEF4050020995200008A
:10528000D551000004460D46164670470093012391
:10529000FFF782FF02BD000080B5112300930223B7
:1052A000F6E704460D4616460C20FFF75BBE0020CD
:1052B0008DF804000820FFF755BE3946BDE8F041DF
:1052C000FFF702BF0521FFF7CEBE3C81BD72FE6035
:1052D000FFF798BE1078802802BF508840F27F61A7
:1052E00088420DD190884FF6807101404FF6806260
:1052F000914204BF00F07F00984201D10120704725
:1053000000207047000038B5FFF7B2FF05000CD051
:105310000422FFF7D7FFAC60FFF774FE2946BDE813
:1053200038400FF20D02FFF7CFBE042032BD00005F
:105330000423CFE710B5514CE0628AB02163A2622A
:10534000684600F0B9F84FF4E13006906946002055
:105350008DF815008DF8160003208DF81C00002034
:105360008DF81D0001208DF800008DF8010000204F
:105370008DF817000FF2410003900FF22100049006
:10538000002000F084F8606218B10022202100F0B3
:105390007BF800F045F80AB010BD000010B53848A1
:1053A0000068804704463548826A110002D0418C6B
:1053B0000020904740E00000F8B500F05AF814468D
:1053C00080470546CCB1318C002089B2B1F5877F8A
:1053D00009DAF76A335C7B5400223254401C491CC2
:1053E000C0B2A042F1D38442318406D0B26A100028
:1053F00009D0718C4FF487709047B26A100002D0C8
:105400000021A0B29047002030842022706A3146EB
:1054100000F057F82846BDE8F4401A4909680847E3
:1054200010B51748006880470446144900200884D6
:105430002022486A00F045F8204612490968BDE874
:105440001040084770B5044600F013F88047054641
:10545000316B706A7484224600F036F8094910F105
:10546000010F04BF00207084096828468847708CAB
:1054700070BD0348014E006870470000DC19002031
:10548000DC020020E002002003685B681847084A3D
:105490001268904201D30020704709B90FF2300121
:1054A000044A0C2303FB00200268D2681047000066
:1054B000F0050020586100000FF214012422FCF7CF
:1054C00011BB03681B6918470368DB6918470000B4
:1054D00000000000FFFFFFFFFFFFFFFF00000000D4
:1054E000000000000101010100C2010003000000F2
:1054F00000000000E0B50821ADF800100190022185
:10550000ADF8021068468F490968884708B1002045
:105510000EBD02980EBD00B58FB008233C220021BD
:105520006846FEF70FF8884800F150010791002304
:105530004FF4217108916A46012106910FF2A501ED
:10554000FFF780FA0FB000BD10B584B00820ADF8A9
:10555000000001207B497D4C0968ADF802006846D7
:1055600088479DF80400207000212161FFF7E2FDCB
:10557000FFF7EDFD201DFFF7C6FE4FF0FF30FFF7F0
:10558000FDFD4FF0FF30FFF7DCFDE08900F00C017E
:105590000C2903D10A220FF2B8210DE0010703D52F
:1055A0000E220FF2B82107E0400747BF11220FF289
:1055B000BC210E220FF2C82104F11800FCF792FA68
:1055C00004F1180000F064F9C1B204F118020020DF
:1055D000FFF7D7FD04F1140202210120FFF7D1FDEE
:1055E0001FBD000070B586B0FFF7AEFF574C554D9C
:1055F0000820ADF800000A20ADF802004FF0FF309F
:1056000001906846296888470028F1D10820ADF844
:1056100008000920ADF80A0002A829688847BDF8EB
:105620000C109DF80E20049E0028E1D1102904BF23
:105630002078824205D13078912804BF304600F0AE
:105640000BF80820ADF800000320ADF80200019629
:10565000684629688847CBE77CB5411C3C4B0C78F1
:105660001D88021D0E2C4FF6FF7608D00F2C11D08E
:10567000102C55D03E2C39D0FF2C56D073BD11883C
:105680008D4255D0536830F8040CA0F10C02D2B210
:105690000E2053E01488A5424AD042F232008442E0
:1056A0004ED14D780F20FFF725FF002848D0042168
:1056B0000170FF2141700721418000F10801416024
:1056C0000421426811700F21426851700421426820
:1056D00091704168CD7001214268117141684C712F
:1056E000210A42689171FFF737FB73BD48780C2897
:1056F00026D18DF80000062089788DF801101188D8
:105700008DF802101188090A8DF8031091788DF830
:105710000410D1788DF80510694600F070F873BD5B
:105720000021082000F002F973BD1488A54201D1C0
:105730001E8073BD53684A782146FF2000F00AF8A6
:1057400073BD0000E4020020A4100020AC02002081
:10575000F40500202DE9F04281460C461546B9F1CA
:10576000FF0F05F10B0014BF0321022108181E468C
:10577000C0B2FFF7BFFE07003FD004203870FF2003
:10578000787007F1080078600420796808707868FC
:1057900080F80190200A7968B9F1FF0F10D0EA1C57
:1057A0008A7001217A68D1702A4679680C7179680B
:1057B000487131467868801DFCF784F9A81D15E012
:1057C000AA1C8A707A683178D1707A687178117100
:1057D0007A68B1785171EA1E79688C717968C871FC
:1057E000F11C78680830FCF76DF9681DC0B278804C
:1057F0003846BDE8F042FFF7AFBABDE8F08270B5B9
:10580000044604F10B000D46C0B2FFF773FE06001C
:105810001DD004203070FF207070E01C708006F1F5
:10582000080070600420716808703E20716848703C
:1058300070688470200005D0706822462946C01C1C
:10584000FCF740F93046BDE87040FFF785BA70BDFF
:10585000544920424C4520416C6C00005449204280
:105860004C452043656E7472616C000054492042BF
:105870004C45205065726970686572616C0000006B
:10588000544920424C4520556E6B6E6F776E000078
:1058900000F10103810704D010F8011B89B18107D1
:1058A000FAD10268B2F10131914311F0803F04BF97
:1058B00050F8042FF6E710F8011B11B110F8011B86
:1058C000FBE7C01A70470000DFF800F055C0011078
:1058D00038B50FF25900124C124D00F03FF8124843
:1058E00019F039FC23681B680122012128469847DA
:1058F000226852680121284690470220FCF756FA98
:105900000320FCF753FAFDF763FFFDF77FFFFFF776
:1059100002FE1020FFF700FAFFF7D6FF002032BD8D
:10592000D801001000400340F4600000022818BFB6
:10593000042881B010D0052807D101208DF800007F
:105940009DF800000028FBD106E001208DF8000042
:105950009DF800000028FBD101B0704701490860A4
:1059600070470000A802002081B001208DF80000DF
:105970009DF800000028FBD101B070477047016816
:105980000A680A4482604B681A44C26008310160A8
:1059900070478168C268914208D101680A680A4468
:1059A00082604B681A44C260083101608168491CFA
:1059B000816011F8010D704738B504460D46A068A6
:1059C000E168884212D120686168884208BFFEF70A
:1059D00007FB2068227C016802B14944A16042684B
:1059E0000A44E260083091422060ECD0A068401C7C
:1059F000A06000F8015D31BD2DE9F0418AB000F1F1
:105A0000080105910268520801EBC20106910021CC
:105A1000079108910168490800EBC1010831009124
:105A2000017901F001018DF81010406800994008DB
:105A300001EBC000019000200290039006E005A851
:105A4000FFF79DFF07980899884207D105980699A6
:105A50008842F4D101980AB0BDE8F08105A8FFF7AB
:105A600098FF044614F0030603D105A8FFF791FF41
:105A7000C61C25090F2D14D105A8FFF78AFF00F1D8
:105A80000F050EE007980899884204BF05A8FFF7A4
:105A900076FF0798401C079010F8011D6846FFF735
:105AA0008BFF761EEED1002DCCD005A8FFF771FF3D
:105AB0000646A00800F00300032804BF05A8FFF76E
:105AC00068FFDDF800800299039F06EB002008E0E4
:105AD000A8F10808A8F10801801A0A68496857184F
:105AE000394658F8082C8A1A8242F1D340420C18E1
:105AF000AE1CA7D0BC4206D158F8044B58F8040B92
:105B00002718BC42F8D00298039914F8015B884228
:105B100017D100980199884208BFFEF761FA0098F2
:105B200000689DF81010029009B148440290009955
:105B300002984968009A0144083288420391009211
:105B4000E7D00298401C0290761E00F8015D3FF4F9
:105B500079AFCFE780B501280CD002280CD00428FB
:105B600002D008280AD00BE00020114612689047A6
:105B7000002002BD0220F8E70420F6E70520F4E744
:105B8000FEF72EFA00BF10B5044601E0FCF70EF94F
:105B9000B4FA84F0202800D110BD00F016F8F5DB2F
:105BA000401FFCF718F9F3E710B5044601E0FCF7D5
:105BB00093F8B4FA84F0202800D110BD00F005F865
:105BC000F5DB401FFCF79CF8F3E7C0F11F00C0B203
:105BD000012181404C400528704738B50546012019
:105BE00068713D4C2879A8B1FDF7E6FC05462078A0
:105BF000FF2805D12846FDF7EAFC6FF0060032BD0C
:105C0000401C2070C0B2012804BF6068FFF7BBFFD2
:105C1000284615E0FDF7D0FC21780A0004D1FDF7F5
:105C2000D6FC6FF0070032BD491E2170C9B239B9E8
:105C3000FDF7CDFC6068FFF7B7FF0020687101E059
:105C4000FDF7C5FC002032BD70B50446606810F059
:105C50007F4F02D06FF0020070BDFDF7ADFC1E4E0D
:105C60000546307828B17068FFF79EFF6068FFF73F
:105C70008AFF606870602846FDF7A9FC002070BDAF
:105C800080B5406810F07F4F00D00DE0FFF77BFF3C
:105C9000002002BD80B5406810F07F4F00D003E0C7
:105CA000FFF782FF002002BD6FF0020002BD10B5B9
:105CB000044682B0A168606808601420FDF732FED7
:105CC000009010B96FF0030016BDA368034A0F21BE
:105CD000FBF7F2FF002016BDE8020020555B000034
:105CE00010B50446FCF7EFF92071002010BD80B517
:105CF000FCF7FAF9002002BD10B50446FBF75DFF82
:105D00006060002010BD10B504466068FCF7D9F94A
:105D1000A060002010BD0000DFF800F00DC30110EE
:105D2000DFF800F081C60110DFF800F095B7011030
:105D3000DFF800F08DC20110DFF800F03DC2011065
:105D4000DFF800F009C30110DFF800F045C00110D2
:105D5000DFF800F0D1C70110DFF800F067BE0110D6
:105D6000DFF800F011C80110DFF800F021C80110C1
:105D70000C381F283ED8DFE800F0103D3D3D3D3D8A
:105D80003D3D3D3D3D3D3D153D3D3D1A3D3D1F24C5
:105D90003D3D3D293D3D3D2E3338DFF8280100686B
:105DA00000687047DFF81C01006840687047DFF842
:105DB0001401006880687047DFF808010068C06857
:105DC0007047DFF80001006800697047DFF8F400F1
:105DD000006840697047DFF8EC0000688069704730
:105DE000DFF8E0000068C0697047DFF8D80000689D
:105DF000006A70470020704700B589B009216846E5
:105E0000FFF78AFF09B000BD00B581B0FBF756FD72
:105E1000DFF8B400DFF8B4100068884218BF00F063
:105E200039F8DFF8AC00B0F5B26F03D001B05DF81F
:105E300004EB30E001B000BD00B581B0FBF720FEFF
:105E4000012818BFFBF78EFC0FF21D00FFF768FF5B
:105E5000FFF76AFFFFF76CFFFFF76EFF01B05DF819
:105E600004EBFFF76DBF000000B581B0FAF7FAFB55
:105E7000FBF764FE01B05DF804EB0320FFF764BF9D
:105E800010B504460320FFF75FFF2046BDE8104031
:105E9000FFF75EBFFEE7FEE700B581B0FFF75CFFEE
:105EA000DFF83000C06801B05DF804EBFBF74ABCD6
:105EB000DFF82410DFF8240088617047FFF750BF37
:105EC000FFF752BFF001002098CA01107047282048
:105ED000900500007801002044010020000400002B
:105EE00080B5FAF783FB36490A7822B9354B1B682F
:105EF0001A7001220A7080B2BDE80240FAF77ABB3C
:105F000038B5FAF773FB04462E4D284600F064F8C6
:105F1000A0B2FAF76FFB284632BD70B50E461446A4
:105F2000FAF764FB85B227480168097809B900F0DF
:105F300053F826B94FF480710122084612E030462A
:105F400000F027F858B114B14FF0FF30207008204E
:105F5000FBF7D6FE2846FAF74DFB002070BDB2686D
:105F60007168306800F042F817490120086017484E
:105F70000068C007FBD502201549096849688847B1
:105F800006460CB1002020702846FAF733FB304655
:105F900070BD4FF0FF3180B102681AB1403AB2F5DE
:105FA0007F5F0AD2426822B1A2F58072094B9A4201
:105FB00003D28068102838BF0021084670470000CF
:105FC0003A1D002078610000A8025042088002407B
:105FD000CC01001000FFFF0001680A782AB90122F5
:105FE0000A7040680068FBF7F6BE704710B50A4BB0
:105FF0001C6824F480641C6009021202090CA4B21B
:1060000002F4706244EA014442EA0141C0F387109D
:106010001C600843586010BD1480024030BF7047B8
:1060200038B5FCF75DFDFCF70DFDFBF7AEFD044652
:1060300004F00C000C2849D0600721D4FBF798FB32
:10604000054601210120FBF7AAFD2349096801FB50
:1060500005F2904214D28220B0FBF1F01F4C291AB5
:1060600004F10C00FAF7D6FA04F10C00FAF7D6FAAC
:106070000120FBF708FF04F10C00FBF7D6FB27E03B
:10608000200723D41648FCF7D7FB0428FAD0E206F1
:10609000144900D418B9086840F0010002E008680B
:1060A000400840000860104C1048114D016841F054
:1060B00003010160202021688969884728682068D9
:1060C000806B804701202860286801E0FFF7A6FF69
:1060D000BDE83140FCF708BDE8000000E004002006
:1060E000004003408C210840B801001024220840E1
:1060F0002C20094006088080070880800D2007C0FA
:106100000E2007C01400C080024000800300C08041
:1061100009400080084000800A400080FE00000026
:10612000FF000000000000000000000021600000EF
:106130006D20000001010100001000400600000079
:1061400015000000FF000000000000000302FFFF38
:10615000000000000000000098620000780F00209E
:106160003861000000000000000000000000000096
:10617000FFFF050508000000361D002074610000C7
:106180000000000000000000EBC70CEEC90CF1CBD2
:106190000CF44B14F74E19FA521DFD5825006131CD
:1061A00001144202184E031C5A0424930530930034
:1061B000886100000D070000C71000006959000049
:1061C000E111000069590000DB13000029140000F0
:1061D0002B1400006959000069590000BF15000028
:1061E000D51500006959000069590000695900007F
:1061F000695900008D110000E915000033160000F8
:1062000071160000E15E0000015F00001B5F0000EE
:106210007B756E6B6E6F776E2D696E7374616E63D6
:10622000652D6E616D657D007B656D7074792D697E
:106230006E7374616E63652D6E616D657D00000027
:106240007B7374617469632D696E7374616E6365C9
:106250002D6E616D657D000019E050F8041BCB07C1
:1062600044BFA9F101035918121F0023042A41F861
:10627000043BF9D25FEA827C0B4604D54FF0000C58
:10628000A1F800C09B1CD10744BF0021197050F831
:10629000042B002AE1D17047C944000039450000B1
:1062A0004343000053430000BB460000AD470000DD
:1062B000B5470000934500004B4600004D460000E6
:1062C00010B5074979441831064C7C44163404E073
:1062D0000A68081D114488470146A142F8D110BD43
:1062E0002C0000006C0100007FC80110C9BC011027
:1062F00051B2011037C20110BDAD0110C1B1011082
:1063000071BA011069BB011021C001104DFFFFFFE0
:1063100048170000F805002000000000DDF6FFFF30
:1063200002000000020000009503000018000000B9
:10633000780100202C000000C1F6FFFF02000000E1
:1063400002000000C603000003000000EC01002072
:1063500004000000A5F6FFFF02000000020000009C
:10636000A403000003000000F0010020080000006A
:1063700089F6FFFF02000000020000005903000040
:106380001A000000A4010020240000006DF6FFFFA9
:106390000200000002000000570300000C00000093
:1063A000C80100201C00000051F6FFFF02000000A1
:1063B00002000000CB0200001B00000000010020D2
:1063C0004400000035F6FFFF02000000020000005C
:1063D0003D03000006000000000200200400000051
:1063E00019F6FFFF02000000020000001B0300007E
:1063F00003000000F801002008000000FDF5FFFF89
:1064000002000000020000009202000023000000D1
:106410004401002034000000E1F5FFFF020000000D
:1064200002000000D702000009000000E401002083
:1064300008000000C5F5FFFF020000000200000098
:10644000AC0000009301000008020020EE030000F1
:10645000DFF800F059C501100548012808BFFFF713
:10646000D3BC70470348012808BFFFF7F1BF70474E
:106470000100000001000000F9F731FE002803D000
:10648000FFF71EFFFFF7EEFF0020FFF721FAFFF7EF
:106490005FFC00B581B0FFF7DFFFAFF3008001B014
:1064A0005DF804EBFFF7E8BF44F24830C2F20000A9
:1064B000854646F29340C0F200008047FEE70000A8
:1064C00001000000000000000000000000000100CA
:1064D0000000000045B50110B15E000099A6011052
:1064E00019B80110B8030020C51B00001200018379
:1064F00001000143C5A70D63995E15B0070100288F
:10650000030020C5A7000161106108100F071000EB
:1065100000384035002D400140028460005D0810C5
:106520001700F80118A384070083057EA40306E082
:10653000EA2306010003040102351C102308047F2E
:10654000176304003888604500C3003801AC52600E
:1065500003A302AD0163026801438AFF00430228DE
:1065600004FF01F001047D590001F309110001103D
:1065700003B9350000CF04439B3725120607800C72
:1065800008051B0050020020B0610000B8613D10FA
:106590000304620000A818100703030000F81300AA
:1065A00020FC04162C111220F42104612A1002E1AF
:1065B00019000023300200FF00141312401C2104B4
:1065C000524804834002544550100101006418F2FF
:1065D00006641C128018210452880452900412CCC4
:1065E0002112082443F8067C4380061012B01C21B7
:1065F00004439C0104C70100B84347180D12D82476
:10660000210452E00452E80452F00452F804839743
:10661000173D12050BC32000014350041312280834
:10662000210452300452380452400452480452505B
:1066300004525804526004830000A86204641510D8
:1066400043780D1CD0030BC201100001D2011112BE
:10665000AC48210452B40452BC0452C40452CC04C9
:1066600052D4046178F1C7016520F3090101E640C5
:1066700008BB210000292200007B212432FF018376
:10668000010001A10CD003AC040020000152DC1475
:1066900020023401002004523C041200011008348E
:1066A0001D0020FC1B0020001C04110143483F0872
:1066B0001101100120010120721B10310152000153
:1066C000100708020020F80300200111C301000197
:1066D00012B818210422000150026CDC02000150A3
:1066E000036C030020030D1003395E00008104F3E6
:1066F00001010001200228040020171200010002FD
:10670000080200205200015200011200010002089C
:0367100000000086
:109AD80038B504460D4614F00FF9084821680160AE
:109AE80061684160A168816011F049FD11F039FD9C
:109AF8002846BDE832400AF08DB900BF9C470020D7
:109B08004549010005830100B3350100678C010058
:109B18003D2A0100CD8E0100ADC40000CBD4000069
:109B28007B9F000009006E1902000000B4BC010010
:109B380002000000B0BC010006040000CD84010052
:109B48001D040000E3840100010C0000F7840100FB
:109B5800630C000003850100030C00000F85010061
:109B68002D0C000019850100310C00002F85010023
:109B7800330C00003B850100350C000069850100AD
:109B880001100000AF85010002100000B985010036
:109B980003100000C3850100091000005B8A010062
:109BA80005140000CD85010001200000E1850100B9
:109BB80002200000ED85010003200000F785010068
:109BC8000520000001860100062000000D86010026
:109BD8000820000045860100092000005386010086
:109BE8000A20000061860100072000006D86010040
:109BF8000B200000778601000C200000A3860100DE
:109C08000D200000B18601000E2000002987010008
:109C18000F20000033870100102000003D8701005D
:109C2800112000004787010012200000558701001D
:109C3800132000006387010014200000BF87010083
:109C480015200000CB87010016200000DF870100E7
:109C580017200000F3870100182000001588010074
:109C6800192000001F8801001A2000003D8801000B
:109C78001B200000538801001C2000006788010099
:109C88001D200000718801001E2000007D88010051
:109C98001F2000008D8801007B0C000079850100E1
:109CA8007C0C00008F8501002020000097880100AF
:109CB80021200000F388010000FC00000989010050
:109CC80001FC00001589010016FC00002189010033
:109CD80019FC00002B89010002FC0000A589010085
:109CE80003FC0000B189010004FC0000BD890100EB
:109CF80005FC0000C989010006FC0000EB89010091
:109D080007FC0000F78901001AFC0000038A010023
:109D180008FC0000658A010009FC0000738A010044
:109D28000AFC00007D8A01000BFC0000898A010002
:109D38000CFC0000938A01000DFC00000F8A010052
:109D480011FC00003789010012FC00004389010062
:109D58000FFC00009F8A010010FC0000AB8A010084
:109D680013FC00005189010014FC00006589010002
:109D78001EFC00007B8901001FFC00008789010090
:109D880020FC0000958901001BFC0000238A0100CB
:109D98001CFC00003B8A01001DFC00004F8A0100EA
:109DA800FFFF00000000000000613100B09D0000CE
:109DB800010000000000D0020A05000000000000B9
:109DC8000201000000000000100000000000000078
:109DD800EC0000210000000000000000D89D0000F9
:109DE800BC9D000000000000C09D0000C49D000054
:109DF800C89D0000CC9D0000D09D0000D49D0000AF
:109E0800A0460020DFF800F0A1940010DFF800F071
:109E180041950010DFF800F071950010DFF800F0B0
:109E2800D1950010DFF800F03D970010DFF800F042
:109E380065970010DFF800F029980010DFF800F0AF
:109E4800F5980010DFF800F0C9990010DFF800F06D
:109E5800F9990010DFF800F0159A0010DFF800F00B
:109E6800319A0010DFF800F0859A0010DFF800F052
:109E7800A19A0010DFF800F0F59A0010DFF800F062
:109E8800159C0010DFF800F08D9C0010DFF800F042
:109E9800099D0010DFF800F0459D0010DFF800F084
:109EA800D19D0010DFF800F02D9E0010DFF800F0C3
:109EB8004D9E0010DFF800F06D9E0010DFF800F0F6
:109EC8008D9E0010DFF800F0AD9E0010DFF800F066
:109ED800CD9E0010DFF800F0ED9E0010DFF800F0D6
:109EE8000D9F0010DFF800F0499F0010DFF800F028
:109EF800699F0010DFF800F0D19F0010DFF800F034
:109F080011A00010DFF800F031A00010DFF800F019
:109F180075A00010DFF800F0F1A00010DFF800F0E5
:109F280009A10010DFF800F0B5A10010DFF800F07B
:109F3800318D001010B5DFF8AC4C207002F086FAB5
:109F4800207802F03AFC207803F090FA04F10C0231
:109F58001021022004F05EFC04F11C0210210320F1
:109F680004F058FC221DBDE810400421042004F030
:109F780051BC2DE9FE4388465FEA0841DFF8640CCE
:109F880077D5007804F06AFD05006FD0DFF8587CBB
:109F9800DFF8584C39680126002918BF11F1010F64
:109FA80005D0207804F0FBFC4FF0FF3038602878AB
:109FB80002284AD0032835D0812804D082282DD001
:109FC800932847D04AE000208DF808608DF80900F2
:109FD800AE88AF79AC78B00A3F2807D1C6F3C21073
:109FE80020B100F054F800F059F803E000F04FF801
:109FF80000F0A3F88146284604F0C2FC9DF808004A
:10A00800A0B3DFF8EC0B01904B469DF809000090D7
:10A018003A463146204600F0DBF927E0284600F0B2
:10A028002BFC1EE0EF682889FFF7ECFEE86040B1E2
:10A038002A89394604F043FC2078294604F0AFFC0D
:10A048000026384604F071FF0CE02078294604F019
:10A05800A6FC0BE0284600F0DBFC02E0284601F0F5
:10A068000FFD064616B1284604F08AFC88F4004025
:10A078000BE05FEA484107D5021D0421042004F0E3
:10A08800D9FB88F4804000E00020BDE8FE8302ABE5
:10A098000DF10902294630467047000038B500F036
:10A0A8007F04C00900F00700401E04280D4642D86E
:10A0B800DFE800F0030C32373C00122C3BD12A7C3D
:10A0C800E9682889BDE8384004F0A7BF2889E9680D
:10A0D800012C1DD00B2C17D00D2C11D0132C0BD00C
:10A0E800192C05D01E2C26D1BDE8324005F0A2B8A7
:10A0F800BDE8324005F06FB9BDE8324005F058B907
:10A10800BDE8344005F026B9BDE8344005F014B97F
:10A11800BDE8344005F0BDB81A462046BDE83840D1
:10A1280019E2204601B0BDE83040C9E2204601B03E
:10A13800BDE8304086E1012032BD0B4640F21D41AA
:10A14800401A00F09A8040F2E471401A00F09880BA
:10A15800801E00F09B802A3800F09A80363800F084
:10A16800928040F29E31401A00F09780401E00F025
:10A178009680401E00F09580801F00F094804FF478
:10A188007F71401A00F0918040F6FC31401A00F0CF
:10A198008F80801E00F08F80001F00F08E800838AE
:10A1A80000F08D80401E00F08C80401E00F08B80F7
:10A1B800401E00F08D80801E00F08F80401E00F051
:10A1C8008F80401E00F08F80401E00F08F80401F5F
:10A1D80000F09080401E00F09480401E00F08C80BB
:10A1E800401E00F092804DF6E231401A00F08F8058
:10A1F800401E00F09080C01E00F09180401E00F0CC
:10A208009280401E00F09280401E00F09780401E11
:10A2180000F09A80401E00F09980401E00F09A805D
:10A22800401E00F09980401E00F09980401E00F00A
:10A238009980C01E00F09880801E00F09980401E12
:10A2480000F09980401E00F09B80801E00F09C80EA
:10A25800401E00F09E80801E6CD0401E00F09F8043
:10A26800401E00F0A180401E00F0A180801E00F07A
:10A27800A280401E00F0A580A8E01889FFF7C6BD9F
:10A288009868FFF7C7BD986805F00ABA05F022B9C3
:10A2980059891889C9B2FFF7C1BD05F069BA05F037
:10A2A8002AB9FFF7BFBDFFF7C1BD188905F08CBA01
:10A2B800986805F041BAFFF7BDBDFFF7BFBDFFF7CE
:10A2C800C1BDFFF7C3BD1889D968C0B2FFF7C2BDC9
:10A2D8001889D968C0B2FFF7C1BD9868FFF7C2BD39
:10A2E8001889FFF7C3BD188905F0B3B9D96898680C
:10A2F800FFF7C0BDFFF7C2BD9A7A597A187A05F000
:10A30800BDB91889C0B205F0C2B9FFF7BBBD18893D
:10A31800C0B2FFF7BBBD1889C0B2FFF7BBBDD96893
:10A328009868FFF7BBBD9868FFF7BCBD1889C0B235
:10A33800FFF7BCBD1889C0B2FFF7BCBD59891889A1
:10A34800C9B2C0B2FFF7BABDFFF7BCBD1889C0B229
:10A35800FFF7BCBDFFF7BEBD9868FFF7BFBD188902
:10A36800FFF7C0BDFFF7C2BD1889C0B2FFF7C2BD75
:10A378001889FFF7C3BD59891889C9B2FFF7C2BD4B
:10A38800D9681889FFF7C2BD18895989C0B2FFF783
:10A39800C1BD59899A891889C9B205F0CBB91889FC
:10A3A8005989C0B2FFF7BABD188905F0B1B9188943
:10A3B800C0B205F09AB959891889C9B2C0B2FFF775
:10A3C800B1BD1A69D968986805F09FB8012070472F
:10A3D8002DE9F843089C804604F10C000F46154609
:10A3E800994680B204F0BAFA060016D08020307080
:10A3F80086F8019040F27F607080B780B57106F1F1
:10A408000C00F471B0602246099904F058FA3146FC
:10A418004046BDE8F44304F0C2BABDE8F183002227
:10A42800831E012B02D99B1E02D004E0102900E0F4
:10A43800042904D002E08038102800D302221046F4
:10A448007047000070B5401E052882B00C461546BE
:10A45800DFF8546C42D8DFE800F0030C15191D3002
:10A4680000F03EF880B9E2683146284604F0D2F997
:10A4780076BD00F035F838B9E2683146284604F070
:10A48800D9F976BD05F0E5F9022076BDA06800F09F
:10A498002CF876BDDFF8143C1B68083300221B68D3
:10A4A800002100209847B071010AF171010C000EDB
:10A4B80070723172042028700EE04FF6FF70ADF80C
:10A4C800000005F0E1FEADF800000222022028702D
:10A4D8006946B01D04F0F3F9002076BD012076BD71
:10A4E800257A667A3146284699E770B1DFF8C01BAD
:10A4F8000160DFF8C01B09888180912181717F216B
:10A5080001810C214181002070470220704738B535
:10A51800012815461C4602D0022809D00DE0049BEC
:10A528000A462146284601B0BDE8304002F0BEB8D0
:10A538000846BDE8324006F0E7B90846BDE83240B3
:10A5480006F0F0B90B4601281146184608BF02F07C
:10A55800E9B806F0FEB938B50C460346E168227C36
:10A568002089022B1D462ED0042B4FD0062B33D02A
:10A57800082B47D00A2B51D00C2B57D00E2B59D073
:10A58800102B24D0122B61D0162B63D01B2B00F07C
:10A5980085801D2B00F08680302B18BF322B22D0EF
:10A5A800342B3FD0362B49D0382B4BD03A2B5BD0AD
:10A5B8003C2B67D03E2B69D0402B6BD0422B49D027
:10A5C800432B75D07AE0BDE8384002F0FAB8A17A9A
:10A5D800BDE8344002F00BB91346A27A01B0BDE8D9
:10A5E800304002F02AB96189A289A37B302D04D1B9
:10A5F80001B0BDE8304002F051B901B0BDE83040CB
:10A6080002F059B9BDE8384002F06DB913464A88DE
:10A61800098801B0BDE8304002F068B9BDE83840AB
:10A6280002F082B9BDE8384002F07FB9BDE8384091
:10A6380002F07EB9BDE8384002F07BB9BDE834408D
:10A6480002F08DB9BDE8344002F097B9BDE8384052
:10A6580002F0ABB9162D03D1BDE8384002F0A6B917
:10A66800BDE8384002F0EDB9E17A0B0008D00629C0
:10A6780006DA009201230A46E16802F098F932BD31
:10A68800022032BDBDE8384002F0D8B9BDE83840F4
:10A6980002F0D5B9BDE8384002F0D2B9BDE838407B
:10A6A80005F0F8BA637C01B0BDE8304005F0BCBAEB
:10A6B800A289618903F082FE002032BD012032BDEB
:10A6C8002DE9FC410F4615460024DFF8DC69A8B3E4
:10A6D80003285AD004283CD005283ED0062844D068
:10A6E800072847D008284CD009283AD00A2851D042
:10A6F8000B285DD00C2874D00D2800F098800E2807
:10A7080069D00F285ED0102857D0112848D01228B9
:10A718004AD030286FD0312876D0322866D03328F6
:10A7280000F08A80342800F08B80352800F095806E
:10A73800362863D0372800F0968098E07869019031
:10A7480038690090FB68BA7A797A387A06F050F955
:10A7580085E0B86806F082F981E0387A06F0C3F936
:10A768007DE0B86806F024FC79E0F968387A06F0EC
:10A7780055FD74E0FB68BA7A797A387A06F097FD65
:10A788006DE0387A06F0C7FD69E0F968387A07F0B5
:10A79800A0F864E03A7B7989387A07F0F7F95EE047
:10A7A800B86807F030FA5AE0B86807F060FA56E07F
:10A7B800F968B86807F0C8FA51E0B97A388907F03B
:10A7C80011FB4CE0387C0090FB68FA7AB97A38893A
:10A7D80007F057FB43E0FA68B97A388907F090FA2E
:10A7E8003DE03989F86807F00CFB38E0F968B8688B
:10A7F80007F0AAFE33E038897989262831D028283D
:10A808002FDA07F01BF82AE04FF6FF78ADF8008042
:10A818003889FF2825DA262823D0282821DA07F0C6
:10A828001AF84045ADF800001BD002200EE0B97AB6
:10A83800388907F0E1FE12E0B86806F092FD0EE0F4
:10A84800387A06F0E3FD009058B1042028700246DB
:10A858006946B01D04F033F80AE006F0FCFD044632
:10A8680006E0022404E000200224287000E001240D
:10A878002046BDE8F68100002DE9F04F044683B07C
:10A88800A688A07994F80280DFF81C780025042EA9
:10A898004FF0010A814622D8DFE806F0030A3D613D
:10A8A8007D001028AB461AD1207A07F04FFF54E0FC
:10A8B8000428AB4651D0102829D0112820D01228BE
:10A8C8001BD0132818BF14280CD0152818BF162819
:10A8D80043D0172804D018280CD0192805D07EE0BA
:10A8E8000A2011E04FF0020B7AE0E168208907F0B6
:10A8F800CAFF72E008F02CF806E008F03DF803E023
:10A90800A17A208908F00DF8B871012568E0207A4D
:10A9180008F082F821E010380528AB465FD8DFE858
:10A9280000F01916120D0903E268A17A208905F0D2
:10A9380021F952E0A06801F092FD0EE0A17A208989
:10A9480001F087FD09E0207A01F037FF05E001F00A
:10A95800F3FE42E0207A01F079FDAA4640E0AB46DA
:10A96800A8B1042804D0052806D006280AD036E065
:10A97800A06808F028FA33E02089E168C0B208F03E
:10A98800FBF92AE000F03EF808F0B6F925E0A068E7
:10A9980008F00DFA21E0062821D8DFE800F01B2096
:10A9A800140F20040A002089E168C0B202F024FED6
:10A9B80013E000F027F802F0F0FD0EE0E1682089CE
:10A9C80002F0C9FD09E02369A27BA189A06802F011
:10A9D80097FD02E0A06802F06CFE834600E0D346D3
:10A9E800204603F0CDFFBAF1000F08D0B81D019042
:10A9F80000955B464A4631464046FFF7E9FC002091
:10AA0800BDE8FE8F61892089E268C9B2C0B270478B
:10AA1800F0B58BB0044600208DF80000606810F88F
:10AA2800011B8DF80410C31C00F0FDFFADF80610E3
:10AA3800BDF8067081788DF80810F809401E0428C2
:10AA4800039342D8DFE800F0032B31363B00187837
:10AA58005A78644E00EB022507F07F000A2802D0DE
:10AA680012280ED031E08A1E92B2991C04A805F073
:10AA780003FE07002AD1327804A9A8B204F0C1FA6B
:10AA880021E08A1E92B2991C04A805F0CAFD0700AD
:10AA98001CD1327804A9A8B204F0BFFA13E001A9C6
:10AAA80007F07F0000F0A6F80DE000F02DF800F0A8
:10AAB80054FB08E000F028F800F083FD03E000F004
:10AAC80023F800F027F8074600E00127204603F0A6
:10AAD80057FFDFF8D4257F2010709770062050703C
:10AAE800BDF80600D070000A40F0FC0010719DF817
:10AAF800000050719DF80000811DC9B2FF20FFF7CA
:10AB080015FA00200BB0F0BD6A4601A907F07F00D6
:10AB1800704700002DE9F0411446401E84B000251E
:10AB280003282570DFF8806557D8DFE800F00217A2
:10AB380034388F6897F801803D78B8F1320F2CDAF5
:10AB480041462846FFF76BFC38BBB21D41462846F4
:10AB580003F060FE050041D178783CE08C682678E7
:10AB6800657829463046FFF75AFCB0B9A21C294639
:10AB7800304603F05FFE042E05462FD1A078E17819
:10AB880000EB0120217900EB0140617900EB0160C5
:10AB98001449486022E004F05CFE02251EE0684685
:10ABA800FFF7A3FC0098B0717573F5730098000A5D
:10ABB800F0710098000C3072BDF804007072000A41
:10ABC800B0729DF80600F072BDF808003073BDF849
:10ABD8000A00B0730A20207000E00125284604B05E
:10ABE800BDE8F081084700206C430020DC480020C5
:10ABF8003A4700202DE9F04F0C4687B02179022909
:10AC08004FF000084FF0400BB8BF4020C0F2F5806D
:10AC1800A768DFF814A93B787A78DFF81069401E36
:10AC28001D2803EB02254FF6FF7900F23982DFE891
:10AC380010F01E00290034003F004A005A00770037
:10AC48008700A800BA00C400E700F3000C011C014B
:10AC58003201490159018601370237029001B801D2
:10AC6800CE01F90137020302370215022D0200F066
:10AC780035FA08F001FA002865D101A9A8B204F054
:10AC880008FBC7E000F041FA08F006FA00285AD19C
:10AC980000F02EFA01F095FDBCE000F01FFA08F074
:10ACA80008FA00284FD101A9A8B204F0FBFAB1E0D4
:10ACB80000F02BFA08F009FA002844D100F001FA54
:10ACC80001F014FEA6E000F00EFA5FEA00082BD0AF
:10ACD80000F0FEF908F00AFA00282BD101A9A8B261
:10ACE80004F0ECFA5BE000F010FA08F02EFA002805
:10ACF80029D100F017FA002800F0D480BDF804002C
:10AD0800012804BFBDF80600484540F0CB80BDF8D7
:10AD18000C2033780499D2B2A8B201F08EFD79E004
:10AD280000F0E1F95FEA000864D000F0D1F908F01A
:10AD380031FA00285BD101A9A8B204F0D7FA2EE0B5
:10AD480000F002FA002855D19DF80830DFF8580CB9
:10AD580000F0E3F920B100F0B4F901F09FFD59E0EB
:10AD68009DF80830DFF8440C00F0D7F920B100F066
:10AD7800A8F901F0A0FD4DE000F0BAF901F0D5FD09
:10AD880048E000F0B0F95FEA000833D000F0A0F91D
:10AD980008F044FA58BB01A9A8B204F0B7FA5FEA70
:10ADA800000B24D126E000F0B0F908F049FA08BBFE
:10ADB80000F09EF901F0B8FD2CE0032902DB00F059
:10ADC80092F980462079022802D0B8F1000F11D0FC
:10ADD80000F07FF908F043FA30B901A9A8B204F0ED
:10ADE800ABFA5FEA000B05D0B8F1000F02D040467D
:10ADF80005F0AFFD584601F0F6FA07B0BDE8F08F50
:10AE080000F083F908F054FA0028F3D100F070F943
:10AE180001F08EFD8346EDE7032902DB00F063F9BC
:10AE280080462079022802D0B8F1000FE2D000F065
:10AE380050F908F051FA0028D6D101A9A8B204F0B7
:10AE480089FA5FEA000BCFD1D4E700F04CF95FEA4A
:10AE58000008CFD000F050F908F049FA0028C6D110
:10AE680000F046F901F065FD99E7032902DB00F0DF
:10AE78003AF980462079022802D0B8F1000FB9D0FB
:10AE880000F027F908F045FA0028ADD101A9A8B2C9
:10AE980004F06EFAD5E700F057F90028AAD100F0BF
:10AEA80041F910B94FF0020BA4E7BDF804000128DE
:10AEB80004BFBDF806004845F4D13178A8B201F0C6
:10AEC80096FCA7E700F00FF95FEA000892D000F0BF
:10AED800FFF808F028FA002889D101A9A8B204F0DF
:10AEE80056FA5CE70B1FF978B8789BB23A1D01F067
:10AEF80089FA5FEA0008E9D001A800904246207963
:10AF0800F978031FB8789BB208F0AAF90028E3D1B2
:10AF18009DF80D0020B900F0EBF801F046FD0AE0BD
:10AF28009DF80C00002801A9A8B202D101F017FD74
:10AF380001E001F022FD83465FEA0B008CE000F09F
:10AF4800CDF808F0A3F900282AD1A8B204F030FA05
:10AF580060E700F0C8F85FEA000821D000F0CCF8FC
:10AF680008F0F8F9002809D1B06818B93C2003F0B6
:10AF7800CFFFB060B06810B94FF0130B37E77178A6
:10AF88000B46052BA8BF4FF0020BF7DA491C71706E
:10AF98000C22534301A9184403F091FC4FF0000B15
:10AFA80028E700F0A0F85FEA0008F9D000F090F870
:10AFB80008F0F3F90028E1D101A9A8B204F0FEF9DC
:10AFC8005FEA000BDAD103980028D7D012E700F027
:10AFD8009CF808F0FFF90028F8D1B16800293FF47F
:10AFE80061AF30789DF804300090A8B2727801F013
:10AFF800DEFC5FEA000B10D0002408E00C2161435E
:10B008000844806808B105F0A4FC641CE4B27178B7
:10B01800B0688C42F2DB03F088FFC6F8088086F837
:10B028000180E7E600F05AF808F0DDF90028F8D1C9
:10B03800A8B204F0D0F9EDE600F03EF85FEA0008A7
:10B04800EFD000F077F8002898D1BA7801A9A8B213
:10B0580004F020FE5FEA000B90D112E000F02CF81B
:10B068005FEA000811D000F065F8002807D13378AE
:10B07800BA7801A9A8B204F0D7FD5FEA000B7FF403
:10B08800B6AE029800283FF4AFAEB3E600F026F85B
:10B0980008F0CEF90028F8D1A8B204F0CBF8B9E648
:10B0A8004FF0010BA6E6000034470020644300205F
:10B0B800020202002E9B0000C91E89B2F81C01F092
:10B0C8009FB93378BDF80620BDF80410A8B27047C0
:10B0D8002079811E01AA89B240467047891E01AABB
:10B0E80089B2B81C7047891E89B2B81C01F088B9AA
:10B0F800327801A9A8B2704701A800904246207989
:10B10800831E9BB200210020704701A800908B1E6F
:10B118009BB2BA1C0021002070470DF109020221E0
:10B1280008F0CEB99DF808300DF109020221504609
:10B1380008F0C6B901A8009042462079C31E9BB208
:10B148000021002008F05EB901A800908B1E9BB278
:10B15800BA1C0021002008F042B82DE9F04F0F4634
:10B1680089B0397902294FF000094FF04008B8BF7B
:10B178004020C0F28181BE6833787478DFF8AC5320
:10B1880003EB04242B780228824636D004286DD09D
:10B19800062842D008285ED00A2876D00C2800F06D
:10B1A80088800E2800F08E80102831D0122800F0F8
:10B1B800C38016281ED01B2800F082811D2800F0AD
:10B1C8009581302818BF32282ED0342866D03628EA
:10B1D80000F08B80382800F099803A2800F0D7805A
:10B1E8003C2800F04C813E2800F05381402800F0B4
:10B1F8005981422800F0AE8092E100F0B5F907F0DD
:10B208004BFF002870D100F099F901F0DAFA3EE11D
:10B218001946A0B201F0EBFA39E18A1ED2B2B11C8C
:10B22800A0B201F00AFB32E1881E04285CD1B07894
:10B23800F178727900EB0121307900EB0222BAF142
:10B24800300F92B289B2A0B202D101F027FB1EE101
:10B2580001F031FB1BE100F06BF9FFF77AFF0028E2
:10B2680042D100F06BF901F03EFB10E100F07CF9EF
:10B2780007F02BFF002837D12B78BDF80E20BDF83A
:10B288000C10A0B201F032FB01E100F087F90028B0
:10B298002AD100F053F901F047FBF8E000F048F933
:10B2A800FFF757FF00281FD100F048F901F03DFBD8
:10B2B800EDE000F06AF9002816D100F03FF901F03E
:10B2C80037FBE4E000F043F95FEA00090CD000F036
:10B2D80053F908F00CF8002854D100F02FF901F0C8
:10B2E80028FB002880464DD1C3E000F030F95FEA22
:10B2F8000009F9D000F030F9002007F0B1FF00286C
:10B3080040D103A9A0B201F02AFBEBE08B1E9BB24F
:10B31800B21C0121012001F075F85FEA0009E3D0B1
:10B3280000F01AF9012007F09BFF00282AD103A991
:10B33800A0B201F022FBD5E000F009F95FEA0009AC
:10B3480024D000F034F900281CD100F0F7F801F0FF
:10B358002CFBC7E000F0FBF85FEA000916D000F00C
:10B368000BF907F0F7FF00280CD12A78BAF1160F6D
:10B3780003A9A0B202D101F019FB01E001F061FBC1
:10B388005FEA000872D1059800286FD071E0881E26
:10B3980001286EDBB078019010B94FF0020868E020
:10B3A8000628FADA0C21484303F0B2FD029010B9DE
:10B3B8004FF013085DE001980C2101FB00F20298A0
:10B3C800002103F0AEFAF61CCA460AE0761CCDF856
:10B3D80000B004233246002107F0BCFFF6190AF139
:10B3E800010A0198824516DA02980C2101FB0AF13C
:10B3F80000EB010B307804270028E7D016F8010B82
:10B40800071DFFB23946304600F0FAFF5FEA00092F
:10B4180012D14FF01308019882450AD12878019A71
:10B42800029900900123D2B2A0B201F0C0FA80467E
:10B43800C8B14FF0000A10E0CDF800B03B464A46CC
:10B4480000210020C8E70C2101FB0AF108448068AC
:10B4580008B105F07EFA0AF1010A019882450298BE
:10B46800F1DB03F062FDB9F1000F02D0484605F0A8
:10B4780070FA404600F0B7FF09B0BDE8F08F00F061
:10B488008DF80028F5D100F059F801F0D7FA804678
:10B49800EFE700F07AF80028EBD100F04FF801F060
:10B4A800CEFAF4E700F053F85FEA0009E1D000F0C3
:10B4B8007EF80028DAD100F041F801F0C1FA11E075
:10B4C80000F040F85FEA0009D3D003A800904A468C
:10B4D8003879FFF733FE0028C8D1B27803A9A0B2A3
:10B4E80004F0D8FB00288046C0D115E000F02AF807
:10B4F8005FEA0009BDD003A800904A463879FFF7F3
:10B508001DFE0028B2D12B78B27803A9A0B204F0AE
:10B518008BFB00288046A9D104980028A3D0A8E76F
:10B528004FF00108A5E70000B8BC0100084700205B
:10B5380003A800908B1E9BB2B21C70472A7803A9FF
:10B54800A0B27047C91E89B2F01C00F059BF891E0D
:10B5580089B2B01C00F054BF03A800904A4638795D
:10B56800831E9BB20121704703A800908B1E9BB2DB
:10B57800B21C00210020704703A800904A46387981
:10B58800831E9BB200210020704703A800908B1EE9
:10B598009BB2B21C0021002007F08ABE03A80090CD
:10B5A8008B1E9BB2B21C0021002007F049BE03A8E5
:10B5B80000904A463879831E9BB20021002007F08C
:10B5C8004FBE2DE9F043ABB0DFF84C9A8D680346C7
:10B5D80099F80000904600272C1DAE1C002B48D07F
:10B5E800032B00F0C280042B00F08080052B00F0B4
:10B5F8008880062B00F09880072B00F0AD80082B80
:10B6080000F0B080092B00F07F800A2B00F0BD808D
:10B618000B2B00F0D2800C2B00F056810D2B00F084
:10B6280088810E2B00F033810F2B00F00B81102B3B
:10B6380000F00381112B00F0B180122B00F0B480D0
:10B64800302B00F05081312B00F05A81322B00F062
:10B658004481332B00F07281342B00F08E81352B1E
:10B6680000F09281362B00F09381372B00F0928105
:10B6780095E12C7810220021304603F027FC28B9E8
:10B688001022314609F10C0003F019F910220021AB
:10B6980005F1120003F01AFC30B9102205F112016D
:10B6A80009F11C0003F00BF905F1220000F0BBF9C9
:10B6B8008278C07801EB024111EB006018BFC9F82D
:10B6C800040009F10400019009F10C0309F11C00C0
:10B6D800009021466A7899F8000005F089F9074634
:10B6E80099F80010262006F0A9F859E18DF8000015
:10B6F80028788DF8010000F05BF9684605F0AEF98E
:10B7080044E105F0F0F941E18DF8000006222878BF
:10B718008DF80100E91C00F04BF901A803F0CFF8FF
:10B72800684605F045FC31E128788DF800000622CE
:10B7380068788DF8010031460DF1020003F0BFF87A
:10B74800B0798DF808006946F0798DF8090099F804
:10B75800000005F063FD19E16A782978334605F0A1
:10B76800A6FD13E105F0D7FD10E10024CDE9004462
:10B7780006226946681C03F0C6F8012818BF6C1C2D
:10B788002878214606F0A5F800E129786B78327808
:10B7980001EB032189B206F0F9F9F7E000F04FF95F
:10B7A800684606F030FAF1E000F049F9A8788DF81B
:10B7B8000A00684606F05BFAE8E0A422002102A825
:10B7C80003F0AFF82878697800EB0120ADF808009D
:10B7D800102230788DF80C00E8788DF80D00254699
:10B7E80029460DF10E0003F06AF815F8930F299910
:10B7F8008DF8A100490868788DF8A800A87800F0AD
:10B80800DEF82990E878002812D0287901998DF877
:10B818000000490868798DF801006F46A8798DF80D
:10B828000200E8798DF80300287A00F0C8F8019042
:10B83800394602A806F088FAA8E000F0F9F806F000
:10B84800D1FAA3E028786978367895F8038000EB78
:10B8580001271022214601A803F031F804F1100055
:10B8680000F0E1F8ADF81410851C082229460DF106
:10B87800160003F024F8287A8DF81E0001AB012089
:10B88800009042463146B8B206F0FBFA7EE02878CE
:10B898006978367800EB0124ED1C102229466846A9
:10B8A80003F00DF815F8100F697800EB0120A9785E
:10B8B80000EB0140E97800EB016004906A463146EC
:10B8C800A0B206F01DFA61E02878697800EB012043
:10B8D80081B2304606F095FA58E005F11001284685
:10B8E80006F032FE52E0287869783278262801EB93
:10B8F80002214DD028284BDA89B205F09FFF45E098
:10B9080029784FF6FF74FF29204608DA262906D041
:10B91800282904DA084605F09EFFA04200D1022734
:10B92800022188F80010DFF8F41688710012C87137
:10B9380036E000F07DF806F05FFE27E06C7804F151
:10B94800080080B203F0E4FA5FEA000813D0287810
:10B9580088F8000088F8014008F10800C8F80400D9
:10B968002246314602F0ABFF404605F0FAFC0700DC
:10B9780016D0404605E0132712E0287805F046FD6A
:10B9880030B103F0D2FA0BE005F065FD074607E099
:10B99800022705E00020022788F8000000E00127C0
:10B9A80038462BB0BDE8F083C0BC0100C4BC010020
:10B9B80068788DF8020030788DF80300704700F041
:10B9C800010242EA4101420821F0020102F00102AB
:10B9D80041EA4201820821F0040102F0010241EA31
:10B9E8008201C20821F0F80102F0010241EAC20115
:10B9F800020921F4807102F0010241EA02214209A0
:10BA080021F4007102F0010241EA4221820921F485
:10BA1800806102F0010241EA822121F47841C009E3
:10BA280041EAC02070470178427801EB0221704753
:10BA380028786A78317800EB022080B2704728783D
:10BA4800697800EB0120ADF800007178307800EBE0
:10BA58000120ADF802006178207800EB0120ADF8F4
:10BA68000400A01C0178427801EB0221851CADF886
:10BA780006102878697800EB0120ADF808007047B7
:10BA88007CB504460020ADF8040001208DF80600BE
:10BA98002C22DFF88C550021284602F042FF20783E
:10BAA8000026A0283DD0A22814D0B0283ED0B12826
:10BAB80042D0C22809D0D0285CD10DF106000090F0
:10BAC80000F070F800F074F834E000F06BF800F063
:10BAD800E8FA2FE060796388627840F4906128463C
:10BAE80000F078FC06466078C0B96179A819012988
:10BAF8000ED00B2902D0132905D00FE004F108015C
:10BB080004F0C6FD08E004F1080104F0A7FD03E015
:10BB180004F1080104F030FD8619F6B28DF80460CE
:10BB280027E000F03FF800F000FB03E000F03AF8EF
:10BB380000F03AFB06461DE06078002804BF207933
:10BB480000280AD1E088A8710426E088000AE87174
:10BB5800208928722089000A6872207963886278AF
:10BB680040F4B061284600F035FCB01D6E718DF8C8
:10BB780004002E469DF8060010B1204602F000FF92
:10BB88009DF8040020B101463246FF20FEF7CEF9A9
:10BB980036B19DF80500012804BF304603F0C5F909
:10BBA800002076BD0DF1050301AA294620467047FD
:10BBB8002DE9F44F0C460A99054601200870002724
:10BBC800A87800261128984649D8DFE810F0120016
:10BBD80049008C00940096009D00BC00D400DB0056
:10BBE800E7001601FA00E701FA01A201B0012002FC
:10BBF800C80027700620607006226878DFF818648D
:10BC0800A070E91CE01C02F05AFE688960721022DC
:10BC18006889000AA07206F10C01287BE07204F121
:10BC28000C0002F04CFE102206F11C0104F11C006D
:10BC380002F045FE687880B906F10C021021022056
:10BC480002F0F8FD06F11C021021032002F0F2FDBB
:10BC5800321D0421042002F0EDFD26462C27D6E1F2
:10BC68006878B0BBE878010038D0C000071D00F044
:10BC7800DFF906002BD00120307006F104090620F8
:10BC880070704FF0000B6878B070E878F070D5F8F5
:10BC980004A013E09AF8000009F8010B06229AF8AC
:10BCA800010009F8010B0AF10201484602F007FEFB
:10BCB80009F106090BF1010B0AF1080AE9785FFAA4
:10BCC8008BF08842E6D3012088F8000001E01320B9
:10BCD8006870687810B9E87800280BD1012000F066
:10BCE800CFF9002003E0022000F0CAF9E878E070FC
:10BCF800264604278BE1032000E0042000F0BBF96E
:10BD080003276878A07082E1052000F0BFF91427A6
:10BD1800201D02F0D4FD6889A0726889000AE072CB
:10BD2800287B2073E8896073E889000AA073288A51
:10BD3800E073288A000A2074688A6074688A000A96
:10BD4800A074287DDDE006202070607026466878A3
:10BD5800A070062700F066F9A879607157E11220F3
:10BD680000F089F90D2700F06AF9A889E072A8891E
:10BD7800000A20734BE1072000F07DF90B2700F043
:10BD88005EF944E1082000F071F9291D6878A07077
:10BD9800E878E070201D02F092FDFCE0092000F038
:10BDA80075F90E27201D02F08AFDE868A072E86880
:10BDB800000AE072E868000C2073E868000E6073FF
:10BDC80025E10B2000F052F9E91C6878A07026469E
:10BDD800E01C02F074FD6889607204226889000A18
:10BDE800A07205F11001287BE0721127687B20738F
:10BDF80004F10D0002F063FD09E16B2003F088F8FF
:10BE08006B27060000F07F80012088F800006B2275
:10BE18000021304602F085FD0A20307006F1220428
:10BE2800062070706878B070A888F070A888000A3A
:10BE38003071A8797071A868C0B10120B071102262
:10BE4800A868807EF07106F10800A96802F037FD45
:10BE5800A868008A30760822A868008A000A7076E6
:10BE680006F11A00A968123102F029FD2869C8B143
:10BE78000120207010222869807E6070A41C296926
:10BE880000F0DAF82869008A207408222869008AF4
:10BE9800000A60741234286900F1120100F0CCF82D
:10BEA800083400E01C34686990B1012004F8010BE3
:10BEB8001022696900F0C0F86869103400F11101B6
:10BEC800062200F0B9F86869007CA071E41D00E062
:10BED8001834E868002815D0012004F8010B102256
:10BEE800E96800F0A9F8E86800692074E868006962
:10BEF800000A6074E8680069000CA074E8680069CA
:10BF0800000EE07483E00A20207006206070132081
:10BF180004E00E202070062060706878A070264625
:10BF2800A888E0700527A888000A20716FE00F2014
:10BF380000F0A6F800F076F8287A6071687AA071A7
:10BF4800A87AE071E87A2072E86800F00101C0F38D
:10BF5800400202B102221143C0F3800202B104225E
:10BF68001143C0F3C00202B108221143C0F30022FA
:10BF780002B110221143C0F3402202B12022114322
:10BF8800C0F3802202B140221143C0F3C02000B1A7
:10BF980080200843607226460A2738E00C2000F00B
:10BFA80065F8A91D6878A0702646A888E0700C2757
:10BFB800A888000A2071601D02F081FC287BE072CD
:10BFC80025E0287B00F10D0700F032F806001CD0B0
:10BFD8000D203070062206207070691D6878B070D8
:10BFE800E878F07028793071701D02F068FCE87A02
:10BFF800F072287B30732A7B296906F10D0002F064
:10C008005EFC012088F8000001E0132068700098A9
:10C0180007703046BDE8F28F0847002034470020FB
:10C028006C470020A888E070A888000A2071704733
:10C03800FFB2384602F06CBF204602F040BC687878
:10C04800A070A888E070A888000A2071E88860714C
:10C05800E888000AA0712889E0712889000A2072FE
:10C06800688960726889000AA07270472070062289
:10C078000620607070472070264606206070704762
:10C088002070062060706878A070704720700622C3
:10C0980006206070291D6878A0702646E878E07050
:10C0A80070472DE9F84304469046A0781E460027BD
:10C0B800002510B101281AD02AE0632002F028FFD9
:10C0C8006327050022D0102000F027F805F1230986
:10C0D800E81C02F0F4FB202204F12301484602F098
:10C0E800EEFB202204F1430109F1200009E023209E
:10C0F80002F00EFF2327050008D0112000F00DF8EC
:10C10800E81C02F0DCFB0120307001E013206070B5
:10C1180088F800702846BDE8F2832870202206209F
:10C128006870E11C6078A87070472DE9F0470446F4
:10C138009A46657800208AF800008846A08900F1B0
:10C148000907BFB22D2F91460CDBFFF772FF0600DF
:10C1580003D001208AF8000005E0A08946463F1A6E
:10C16800132500E0464663882A464FF49E61304610
:10C1780000F030F9A0887071A088000AB071A08919
:10C18800F071A089000A3072A16841B125B9A2896D
:10C1980006F1090002F093FBA06804F0DAFB89F8C5
:10C1A80000703046BDE8F0872DE9F44F05460027BA
:10C1B800994695F801B00024BBF1000F18BFBBF1F8
:10C1C800160F0E46A24689F8004035D12879012875
:10C1D80033D0022836D0032839D004283CD005288B
:10C1E8003FD0062842D0072849D0082873D009280C
:10C1F8004AD00A284DD00B2850D00C2853D00D28EF
:10C2080056D00E2859D00F285FD0102863D0112897
:10C2180066D012286BD0162878D017287BD018281B
:10C2280000F082801B2818BF1D2800F083807E281C
:10C2380000F089807F2805D08AE000F0C7F806F072
:10C2480012FF75E000F0C2F806F025FF70E000F07C
:10C25800BDF806F026FF6BE000F0B8F806F034FFF2
:10C2680066E000F0B3F806F035FF3DE000F0AEF808
:10C2780006F05EFFD5F814A00627841F68E000F0DA
:10C28800A5F806F083FF24E000F0A0F806F0C5FF4B
:10C298002AE000F09BF806F0D2FF49E000F096F89B
:10C2A80006F0DBFF15E000F091F806F0F4FF3FE040
:10C2B80000F08CF807F00EF80BE000F087F807F0B4
:10C2C80012F8D5F808A0044642E000F07FF807F01D
:10C2D8001EF8044634E000F079F806F068FF27E01D
:10C2E80000F074F807F016F80127441E28E0287CAF
:10C2F800B07105F10801687CF071042706F10800A7
:10C3080006F0C3FFD5F80CA0841E21E000F05EF80B
:10C3180007F01FF803E000F059F807F02FF804279A
:10C32800D5F810A0041F13E000F050F807F04EF8FD
:10C3380007460DE000F04AF807F05AF80227841E75
:10C34800D5F80CA004E0287AB0710227687AF07159
:10C35800FFB2E4B2E019801D2D2817DBE019801D1B
:10C3680080B202F0D5FD5FEA00080AD0012089F802
:10C37800000067B13A46B11D08F1060002F09FFAC5
:10C3880005E0B04600244FF0130B00E0B046BAF1C8
:10C39800000F0AD034B108EB070022465146801D31
:10C3A80002F08DFA504604F0D4FA28796B8840F4EC
:10C3B800A0615A46404600F00DF8E01988F80500DB
:10C3C800801D009908704046BDE8F28F05F108010C
:10C3D800B01D704701708270090A4170C370190A54
:10C3E800017105207047052804D00C2806D00F28B5
:10C3F80002D0704741207047422070474320704761
:10C40800002209E010B504001046BDE810401ABF2C
:10C4180000290C220022194670B504460D46501911
:10C42800401C80B204F070FA48B14FF0FF3104F0BC
:10C43800B5FA06462A46214602F041FA304670BD52
:10C448008249086070478149486070478049087090
:10C458007047032290FBF2F080B202F002BE01782E
:10C46800B02904BF417800290CD10179122903D1E0
:10C47800417C012906D101E01B2903D14088012113
:10C4880002F00CBE704710B5724C607006F074FA7A
:10C49800401C20700421607802F066FDBDE8104061
:10C4A80003F0D8B938B50C46200411D5694840784E
:10C4B80002F0D4FA050008D02878A02804BF28463E
:10C4C80000F008F8284602F05BFA84F4004032BD18
:10C4D800002032BD30B587B0044601208DF8000039
:10C4E80001A9204606F092FD05002AD19DF8061004
:10C4F8005648C9070AD54368180005D060886A46B7
:10C5080001A9984705461CE006251AE003681800AB
:10C5180006D060886A4601A99847050001D110E055
:10C5280006259DF8050060B99DF806008DF81000F5
:10C538008DF814500020ADF8120004A9608802F0AC
:10C54800A8FE9DF8000000281EBFA068002804F07F
:10C5580000FA45B99DF80600122806BF9DF8051097
:10C5680001291B2803D06088012102F097FD07B03C
:10C5780030BD2DE9F0410446FF2C0D46164698467D
:10C588001FD0202002F0EAF9070018D0B020387038
:10C598007E707D8087F80480069929B1182207F1FA
:10C5A800080002F08CF904E0182207F1080002F0F4
:10C5B800B8F93946204602F0F2F9002002E01320CB
:10C5C80000E00220BDE8F08110B54FF47A746243B0
:10C5D800BDE8104007F025B810B504001EBF20784C
:10C5E800FF28FE2803D007F056F8FF20207010BD62
:10C5F80080B5009313460A46014615480078FFF7B0
:10C60800B8FF02BD30B583B004460D4606F094FF6E
:10C6180050B901A80090ADF804507F230C48007869
:10C6280000222146FFF7A5FF37BD00B583B07E2362
:10C638008DF804108DF8052001A90091002201460B
:10C6480003480078FFF795FF07BD00000C4800205D
:10C65800F8460020D8480020052923D006291BD0F9
:10C66800072918BF09291DD00B2918BF0D2919D072
:10C678000E2913D00F291CBF1129122912D01629EF
:10C6880018BF17290CD01B2918BF1D290AD05229F9
:10C6980018BFD22906D007E0C06870470068704705
:10C6A80080687047406870470020704770B505295A
:10C6B80014461D4616D0062912D0092918BF11297B
:10C6C80010D0122912D0162918BF17290CD01B29EF
:10C6D80018BF1D290AD0522918BFD22906D007E051
:10C6E800072606E0022604E0052602E0032600E00D
:10C6F80001264FF6FF72944203D106F032FF841BE5
:10C7080002E0D22908BF0C34301980B204F0FCF8DA
:10C7180038B105B12C807142BDE8704009B204F00F
:10C728003DB970BD80B5FFF797FF18B1BDE802406D
:10C7380004F00FB901BD00002DE9F041DFF8945B6A
:10C74800DFF8948B28782824604302F0E1FBC8F8CE
:10C75800000008B913202EE00027FF260FE01880FC
:10C768001822002098705E721E72987283F8240056
:10C77800002103F10C0002F0D4F87F1CFFB22878E6
:10C7880087420BDAD8F8000004FB07F14318002FA2
:10C798000CBF4FF6FE704FF6FF70E0E70FF2D14086
:10C7A800FFF751FE0FF6E93002F09EFC0FF63D4010
:10C7B80005F0F9FF0020BDE8F081DFF8201B0870C4
:10C7C8007047F0B583B000F0BDF907000DD12946D8
:10C7D800204602F08CFC070007D10198DFF8003BE7
:10C7E80000960322294600F02CFD3846FEBD70B5A0
:10C7F80088B004460120ADF808000D464FF6FF70DA
:10C80800ADF80A0001A902208DF80C00002000F004
:10C818007CF900F036FD06000CD102A9204602F092
:10C82800C3FC060006D10198DFF8B83A009511223A
:10C8380000F069F9304608B070BD2DE9F0411646A0
:10C84800022E18BF102E88B080460D461F4622D1F2
:10C858000DB301A900F015FD0446E8B90120ADF8B3
:10C8680008008DF80C604FF6FF70ADF80A003246EC
:10C8780029460DF10D0002F022F802A9404600F009
:10C88800E1F8044640B90198DFF85C3A00970722BE
:10C8980000F039F900E00224204631E100B587B004
:10C8A80000F01BF88DF80510ADF8022028218DF84E
:10C8B800061000220CE000B587B000F00EF8ADF8C5
:10C8C800022003218DF80510002228218DF806107A
:10C8D800694600F0E0F807B000BDADF8001002218D
:10C8E8008DF80410704713460122D4E070B584B067
:10C8F8000446ADF80410ADF806201D4602A900F064
:10C90800C0FC06000DD101A9204602F003FC060078
:10C9180007D10298DFF8D4390095052201A900F063
:10C9280090FC304604B070BDF6E013460022B2E039
:10C938000DE1F0B583B000F005F907000DD12946E7
:10C94800204602F01FFC070007D10198DFF8A03944
:10C9580000960F22002100F074FC3846FEBD38B561
:10C9680000F019F8172807D0287A002804BF687A39
:10C97800012800D114E0022032BD38B500F00BF8D0
:10C98800172807D0287A012804BF687A012800D11F
:10C9980006E0022032BD0D460446694600F071BC2F
:10C9A8002946204602F00CFC32BDE6E008E12DE9FC
:10C9B800F0410E0086B0804617461D4639D0380033
:10C9C80037D0404606F0CDFDC0B20021C9B20C23D5
:10C9D8004B433344421F9B889A4201DA1B202AE0CA
:10C9E800491CCAB2BA42F1D301A9404600F049FC39
:10C9F80004001FD1B0680090B3887288318840461F
:10CA080000F012F9040015D100208DF811008DF8FE
:10CA1800107001208DF8080003968DF81250172227
:10CA28000C98DFF8D038009002A9019800F009FCB2
:10CA380000E00224204606B0BDE8F0816CE086E004
:10CA48009BE0BDE030B50D4685B02A790446002349
:10CA58000621FFF72BFE0390C8B12888ADF8000027
:10CA6800691D688800F056FB002000F04DFB2A790C
:10CA78000398ADF8082001F022FF6946204602F02D
:10CA880053FB040004D0039803F063FF00E0132471
:10CA9800204605B030BD2DE9F04188B00D4604466A
:10CAA80090461F4601A900F0ECFB064638BB5FEA3A
:10CAB80008000FD02888ADF8080002A96888ADF8EA
:10CAC8000A0002208DF80C00032000F01EF802F086
:10CAD8003DFB03E02946204602F038FB06000ED154
:10CAE800162229460DF10A0001F0E9FE0198DFF847
:10CAF80008388DF808800097092200F004F83046BD
:10CB080008B0BDE8F08102A99BE38DF80D0028204C
:10CB18008DF80E0020467047F0B583B000F012F88B
:10CB280007000DD12946204602F01CFB070007D15B
:10CB38000198DFF8C83700960B22002100F081FB2E
:10CB48003846FEBD0D460446164601A999E3F0B5E0
:10CB580083B0FFF7F7FF07000DD12946204602F002
:10CB680007FB070007D10198DFF8943700960D22DC
:10CB7800294600F066FB3846FEBDF0B50D4683B089
:10CB88000446287A002804BF687A0028164614D17B
:10CB980001A9204600F075FB07000FD12946204661
:10CBA80002F00EFB070009D10198DFF8583700960C
:10CBB8001322002100F045FB00E002273846FEBDA5
:10CBC800F0B587B00D460746144601A900F059FB99
:10CBD800060026D1384606F0C4FCAB88401F8342C5
:10CBE80003DB384606F0BDFC431FA86800906A883E
:10CBF80029889BB2384600F017F8060011D10020AA
:10CC08008DF808000C22294603A801F058FE688810
:10CC1800DFF8E036ADF81800009417220198FFF706
:10CC280072FF304607B0F0BDFEB50D4616461F46EA
:10CC3800044600233A461621FFF738FD029098B1C2
:10CC48000899ADF80050ADF80260ADF804703A46A6
:10CC580001F035FE6946204602F0D6FA040004D0F9
:10CC6800029803F076FE00E013242046FEBD000083
:10CC78002DE9F0430E4687B08046307817460024E9
:10CC880060B97078012809D0B0781B2818BF1D2812
:10CC98003CD1DFF848562978FF2901D1062091E0D8
:10CCA8001D2812D1404600F000FB04000DD0A27AE6
:10CCB80010000AD010062ED4B1784046FFF7B5FC14
:10CCC800A07A40F08000A07225E001A80090B38807
:10CCD800B2687178307806F095FB0028814670D1EB
:10CCE80001A800900022B37828784146FFF741FC5C
:10CCF8000028814665D1029808B100203870B078C4
:10CD08001D285ED1002C5CD0A0725AE0404600F08D
:10CD1800CCFA040001D1002054E0B07801281DD1DC
:10CD2800B188B06801AA06F0A7F95FEA000948D1FE
:10CD3800A078052818BF072808D009281CBF0D2887
:10CD4800112803D0172817D12069A8B1B27801ABF0
:10CD58002146404600F037F8387032E0A178884222
:10CD680007D16368180004D0B188B06801AA984751
:10CD7800DBE74FF0040924E0DFF88C25607A1278AD
:10CD880090420FD001A900910022B3784146FFF7E5
:10CD9800F0FB814630B9B17801A8FFF75DFC08B116
:10CDA80000203870A078032808D1A189BDF80400B4
:10CDB800814288BF01464046FFF724FC204600F028
:10CDC800AFFA484692E12DE9F8450D468246A87823
:10CDD800052816461F464FF0010847F230540BD07D
:10CDE80007280FD0092834D00D2839D011285AD057
:10CDF800172800F080808DE03A463146284600F03A
:10CE0800B0F82BE0072E19D195F82400EA89401CC8
:10CE180085F824003988786800EB810010F8041D33
:10CE2800407801EB002081B2914210D2401CA881C9
:10CE380005F10C012888FFF705FE56E038790A2825
:10CE480028D195F82400441EA441E40F23E00024CF
:10CE580021E03A463146284600F0B3F804461AE085
:10CE68000D2E14D195F82400401C85F8240028883C
:10CE780006F077FB3988401E8142E8DBE88908180C
:10CE8800E88105F10C01288802F072F92DE0387963
:10CE98000728D6D00124002C08BF012E3BD13879B1
:10CEA8000A283DD14CE0112EC8D138887988401E17
:10CEB800484395F82410491C85F8241080B27968F5
:10CEC80008448178C07801EB002080B24FF6FF71EA
:10CED8008842BCD0401CA88180B2E9898142B6D37F
:10CEE800288805F10C0102F05FF9287A214606F03E
:10CEF800A0FB162414E0287B01283A463146284630
:10CF080002D100F04AF901E000F00FF90446012CC3
:10CF1800C1D023E00124092E04BF388800280ED090
:10CF280000973346687A00225146FFF722FB30B952
:10CF380031463846FFF790FB08B14FF0000844B976
:10CF4800002000901A22AB78687A5146FFF711FB4F
:10CF580001E0162C02D0284600F0E2F94046BDE870
:10CF6800F28510B50529044621D100F0C2F85168B0
:10CF780010889278012A03D101EB8000001F03E09A
:10CF8800122250430844123801784078E28901EBB4
:10CF9800002080B2904212D2401CA08104F10C0102
:10CFA800208802F0B7F800F0AAF8162010BD107912
:10CFB8000A2802D194F8240008B9012010BD0020E5
:10CFC80010BD2DE9F043092987B0044615463CD128
:10CFD80028886988401E484394F82410491C84F81E
:10CFE800241080B269680A5C0844407802EB002685
:10CFF800207B012854D128886988002748431FFAD4
:10D0080080F82F80B946C1454ADA6888A17C431F59
:10D0180068684844421D9BB204F1130006F050FAB8
:10D0280070B1B94506D068686A8800EB09013844D0
:10D0380001F045FC6888C7192888401CBFB22880C1
:10D04800688848445FFA80F9DDE728790A2803D11F
:10D0580094F82400002848D1A37CAC4800F060F87C
:10D06800002837D1A37CAA4800F05AF8002831D10B
:10D07800A37CA84800F054F800282BD1A37CA6482C
:10D0880000F04EF830BB2879022818BF052804D0D4
:10D0980008281CBF0F280C281CD100F02AF86E881D
:10D0A800B6B24FF6FF7086421FD0218A8E421CD23C
:10D0B800217B701C0129E0810ED1ADF80000694682
:10D0C800208A00F027F8032000F01EF8208802F0DC
:10D0D8003DF806E0012009E0208804F10E0102F085
:10D0E80035F800F00CF8162000E0002007B0BDE885
:10D0F800F08394F82400401C84F824007047207AB8
:10D1080047F2305106F095BA8DF8050028208DF8C1
:10D1180006007047ADF8020002208DF80400704741
:10D1280004F11302022106F0CBB9F0B50E46172E12
:10D1380083B0044647F2305522D1208806F011FA10
:10D14800A18BA38A421F5118A183A28B618A511A0D
:10D1580089B2994212DAA0F1050C5F1ABC45B4BF36
:10D16800431F5B1AA069084400909BB2218A20885B
:10D17800FFF75AFD20B900F060F80CE0012000E04C
:10D18800002000F054F8012E01D10120FEBD00F06E
:10D1980054F800F047F81620FEBDF0B50E460446D8
:10D1A800172E83B0104647F230552ED1627D216983
:10D1B8000C277A438B1802881988914202BF598834
:10D1C8004288914202BF8288998891421DD1816824
:10D1D800986801F098FBC0B1607D227D401CC1B207
:10D1E800914260750FD22169C0B278430F18B868B0
:10D1F8000090BB887A8839882088FFF715FD20B908
:10D2080000F01BF80CE0A07D00E0002000F00FF813
:10D21800012E01D10120FEBD00F00FF800F002F848
:10D228001620FEBD1920A0703C48606070478DF83C
:10D23800040001A9208801F0F7BF207A294606F0EA
:10D24800F8B92DE9F041069CFF2C05460E46174615
:10D25800984614D005F108031E2229460FF24D10F6
:10D26800FFF7B2F96C72AF70C5F804803EB1314671
:10D2780005F10C00BDE8F041182201F020BBBDE823
:10D28800F08110B50C4600F010F860B104B12060D0
:10D29800007AFE2801D1172010BDFF2801D10020F7
:10D2A80010BD162010BD022010BD10B50A4A126824
:10D2B800002100E0491C074C2478CBB2A34207D2D6
:10D2C800C9B228234B43D45A8442F3D1D01810BD95
:10D2D800002010BDD848002014480020F94600203E
:10D2E800BB3001002F3301009D310100F5300100F2
:10D2F8001B330100A333010025320100673201000E
:10D30800E132010095320100D9480020B8BC010083
:10D31800BCBC0100C0BC0100C4BC0100EF3301006B
:10D32800F8B5044604F10800FFF756F9A51C04F106
:10D3380010062878172818BF19281AD1A87A0128A2
:10D3480013D13068A8B1002708E00C2179430844BC
:10D35800806808B103F0FDFA7F1CFFB231793068AC
:10D368008F42F2DB01F0E1FD03E0B06808B103F0A1
:10D37800F0FA002028701822FF20E8710021002010
:10D38800307504F10C00BDE8F84001F0CABA00009D
:10D3980010B50C46FFF789FF30B1817A4A1C9442D8
:10D3A80004BF01F08001817210BD000010B582B089
:10D3B80004001CBF207AFF2816D000200090A37814
:10D3C8002188607A1722FFF7D4F8A078182806D1A8
:10D3D80000208DF800006946208801F025FFFE2016
:10D3E80020722046FFF79CFF13BD000070B504466D
:10D3F8004FF6FE70844282B037D008004FF6FF76B1
:10D408000AD12046FFF751FF78BB3046FFF74DFFA2
:10D4180005002AD0048073BD012906D12046FFF7F4
:10D4280044FF050021D02E800BE002291DD10121E7
:10D43800204605F076FAC0B92046FFF736FF05000A
:10D4480013D0287AFF280ED0FE2807D0002000909D
:10D458001422AB78687A2146FFF78BF82846FFF745
:10D468005FFFFF2028720020A87273BDDFF8581CE8
:10D478000870704738B5DFF8544CDFF8545C2076F4
:10D488002878C00001F044FDE061C8B1002108E03F
:10D498004FF6FF7220F8312000EBC10300225A60DA
:10D4A800491C2A789142F3DB052000F0AFF8207E72
:10D4B80002F072FABDE83240DFF8180C05F073B9D3
:10D4C80031BD38B50C46200418D5DFF8000C007EB5
:10D4D80001F0C4FA05000ED02878B02808D12846F3
:10D4E80000F0FDF820B1297905F10800FFF71AF9D5
:10D4F800284601F045FA84F4004032BD002032BDD0
:10D508007CB506001C460DD0ADF800108DF8022041
:10D518000196684602F0D2F905001AD1CCB1768995
:10D52800300001D1022514E00C2001F0F1FC08B90B
:10D5380013250EE00021016086808460DFF8981BC7
:10D548000A6812B9086004E00A4611680029FBD18C
:10D558001060284676BD30B50C46DFF87C1B0546C2
:10D56800086883B0002201E00246006898B1838809
:10D57800AB42F9D10368002A0CBF0B60136001F0BD
:10D58800D4FC6946284602F0E7F9010002D10CB143
:10D59800019921603EBD01203EBD70B550BB0129F7
:10D5A80026D1DFF8280BC169002300E05B1CDFF8F7
:10D5B800204B2478A34217DA31F833404FF6FF7531
:10D5C800AC42F3D0002400E0641C467EE5B2B542CC
:10D5D800ECD201EBC305E4B26D680C266643AD5B83
:10D5E800002DF1D0012070BD1078BDE870400DE02D
:10D5F800182070BD022070BD0022002803BFDFF88C
:10D60800CC0A407E08700222104670472DE9F84384
:10D61800DFF8B87A0446002078760C25F869DFF838
:10D62800B06A406805FB04F870B101F07EFC002088
:10D6380006E0F969C0B201EBC00100224A60401C53
:10D648003278C1B29142F4D3307808FB00F080B24E
:10D6580001F05EFC5FEA000928D0307808FB00F290
:10D668000021484601F05DF900200FE0516805FBF4
:10D678000CF34FF0000E21F803E019440CF1010CF3
:10D68800C1F808E0A445F1DBC144401C3278C1B2BE
:10D69800914208D2F969C0B201EBC0024FF0000C08
:10D6A800C2F80490EEE77C76002000E01320BDE885
:10D6B800F28301460020C90705D500231022012165
:10D6C800DFF8180C1CE77047DFF80C1A096821B15D
:10D6D8008A888242FAD188687047002070472DE90D
:10D6E800F04186B004460020ADF8100001208DF806
:10D6F8001200DFF8D859286A38B901F0E0FC01F0C7
:10D7080007FC0028286200F0E28018220021284641
:10D7180001F007F92079461C02284FF6FF7817D048
:10D7280006282CD008282FD00A2833D00C2857D008
:10D738000E2800F08B80102800F08D80122800F051
:10D748008F80162800F09380182800F09780BBE09F
:10D7580001F0B5FC28802946608801F0A3FD002867
:10D768002189288804D0814228BF01462980A0E069
:10D77800814228BF01466088FEF744FFA4E004A95F
:10D78800204600F0AEF87DE004AA0021204600F013
:10D798002CF977E000F0A0F8070052D0608805ABBC
:10D7A80042460B21FEF782FF03006B6024D02079EC
:10D7B800BDF81620039000953946BDF81400029074
:10D7C8000020019000F026FA070004D1608829465D
:10D7D80001F0B2FD29E0162F686808BF00272BE08A
:10D7E80000F07AF807002CD0608805AB42460D217E
:10D7F800FEF75CFF686020B92089ADF8100011279A
:10D8080045E02179BDF8162003910346BDF81410B0
:10D818000291618901910095394600F0FBF90700F2
:10D8280006D16088294601F095FD002841D12AE0FB
:10D83800162F686808BF002703F08BF8380001D15D
:10D8480021E001272089ADF810001CE004A920463A
:10D8580000F06EF916E004A9204600F0E9F911E09D
:10D868000DF1120204A9204600F086FA0AE00DF133
:10D87800120204A9204600F0C0FA03E004A92046D9
:10D8880000F029FB0746380011D0162F11D0607818
:10D8980014280CD0207928702F712946BDF8100063
:10D8A8006880608801F0F5FC08B1012601E0162FB8
:10D8B8000AD160882B46F2B21621FEF799FE18B1FC
:10D8C800F1B22846FEF72EFF2046FEF7C8FD9DF868
:10D8D800120006B0BDE8F08120890DF1160102F0B2
:10D8E800D3B82DE9FA47044686B06088DFF8DC57DC
:10D8F80005F037FE80460DF1120000F0D4F800273D
:10D9080081464FF0FF0AB9F1000F5BD009E0BDF87E
:10D9180010304354BDF81000696892B2000A885468
:10D92800571CBFB2A8F1050087424BDA2079039053
:10D938000026A8F1070080B20290019605F11A00AE
:10D9480000902B6ABDF812206088494600F0CCFB95
:10D95800002802BF6A8B208A904214D1296A606924
:10D9680000F0D1FF78B1686858B900F055F907217F
:10D97800FEF79CFE686020B906992089088011206E
:10D9880030E0B9F80A60BDF81220618904AB484656
:10D9980002F0A0F8002E8146B5D06868C655781CFC
:10D9A8006A6880B231121154411C4A1C6868B9F186
:10D9B800000F89B2ABD100F801A092B2686800F8F4
:10D9C80002A0571CB8B248B13F04B80C28802946B9
:10D9D800608801F08BFC28B1162003E006992089A5
:10D9E80008800A2008B0BDE8F0872DE9F043044616
:10D9F80085B060888846914605F0B3FD851EADB2B6
:10DA0800DFF8C87601E0401C2081A81E39898842C9
:10DA18002FDB5FEA08002CD104A800F044F80600C8
:10DA280027D070892081BDF81020317A608801F0F4
:10DA3800B7FF5FEA00081CD120793B6ABDF81020C7
:10DA480003903146A81E80B200F0EBF800F0E2F82F
:10DA58005FEA00080DD173897A8B396A608800F013
:10DA68002AF85FEA000804D120894FF6FF7188423E
:10DA7800C9D1388901000AD0798890FBF1F0388043
:10DA88003946608801F042FC50B1162008E05FEA90
:10DA980008002089A9F8000008BF4FF00A0840468E
:10DAA80005B0BDE8F0830090237B6189208904F1EB
:10DAB8000D0201F0BABF2DE9F8468246894615469F
:10DAC8001E4605F04EFDDFF804460746208990B94A
:10DAD80000F0A3F809215046FEF7E8FD606008B998
:10DAE800112023E0A81C60803A1F208901466B188A
:10DAF8009A4206D203E06088A91C8842F4D001202B
:10DB080014E0401C2081606846542089411C218112
:10DB1800310A62681154606823892A4649461844C4
:10DB280000F0CDFE2089281820810020BDE8F2866B
:10DB38002DE9F047044686B06088DFF890750D46F9
:10DB480005F00FFD0026A0F10109A0F1010814E07D
:10DB58003888798B0346C9188845BCBFA9EB0000F3
:10DB6800788378687A8B396A184400F0A8FE388878
:10DB7800798B0818761C3880B6B2A0898642BCBF5B
:10DB88003888404534DAA06810F8162000EB4600C3
:10DB980004A9407802EB002080B201F075FF010073
:10DBA80009D14FF0010A00F02BF8786808B102F0AB
:10DBB800D0FE5046DDE02079BDF8102003901FFA12
:10DBC80089F000F02EF83B6A00F024F8002882461D
:10DBD800E9D178680028BBD100F01EF80F21FEF7C4
:10DBE80065FD00287860B3D100F00AF81120E1E75C
:10DBF8006088394601F0BCFB0028DBD01620D9E745
:10DC0800A06810F8161000EB4600407801EB0020E1
:10DC180028807047608867E2608800234FF6FF72AB
:10DC2800704702900020019007F11A000090704799
:10DC38002DE9F047044686B06088DFF8905489469D
:10DC480005F08FFC059004F10D0204A80090237BD9
:10DC58006189208901F0E9FE0026B24607464FF0A7
:10DC6800FF0810E0696801F8068080B2696801F869
:10DC78000080461C68686A8B296AB6B2801900F071
:10DC88001EFE688B8619B6B2FFB1BDF81020397A2E
:10DC9800608801F085FE5FEA000A13D12079BDF89B
:10DCA8001020039039460598801F80B2029000200A
:10DCB800019005F11A0000902B6AFFF7ABFF5FEAAD
:10DCC800000A10D07889A9F80000002E48D068888A
:10DCD80096FBF0F028802946608801F058FB002860
:10DCE80047D0162045E07EB9FFF796FF1121FEF7D1
:10DCF800DDFC686020B97889A9F80000112038E0B7
:10DD0800688B001D688009E0688B6988021D914254
:10DD1800DDD10599891F80198142D8DB6968788926
:10DD2800885579896A68701C80B2090A1154461CA2
:10DD3800BDF8102061890DF11203384601F0CAFEC2
:10DD48000746701C002FB6B28CD06A68BDF8121056
:10DD5800915580B2BDF812106A68090A115488E713
:10DD68005FEA0A002089A9F8000008BF4FF00A0AF4
:10DD7800504606B0BDE8F087FEB504460D4620893A
:10DD8800164602A901F080FE07002ED0387A8006D8
:10DD98000BD5BDF8080000F0A1F903000BD060888E
:10DDA800122239469847070020D1607C002814BF0A
:10DDB8005220207901E00E2718E001900020009001
:10DDC8006389E2682189608800F08AFA070007D130
:10DDD800607C68B9608801F0EBFA48B11620FEBD96
:10DDE800162F03D10027377002E0012720892880E9
:10DDF800607C00B100273846FEBD2DE9F04104469D
:10DE080082B00D4660889046012104F08AFD002703
:10DE180018B9142060700E205BE02089694601F073
:10DE280033FE060051D0307A80060BD5BDF80000CD
:10DE380000F054F9030013D0608812223146984745
:10DE4800070043D16688304600F008F928B94FF634
:10DE5800FF7000F003F9A0B3068000219B4E02E09A
:10DE68000E2733E0491C737ECAB29A4229D242680F
:10DE7800C9B20C234B4313441A88002AF2D10C224E
:10DE880004F10801184600F01AFD002088F8000087
:10DE98000C2204F10801304600F011FDA2896088C7
:10DEA80000231721FEF702FCB06060B1A289216946
:10DEB80000F005FD6088314601F080FA40B1162077
:10DEC80007E0092702E0112700E0012720892880C0
:10DED8003846BDE8F6812DE9F043044683B06088F2
:10DEE800894600F0BBF800265FEA00084CD0207A8B
:10DEF800012845D1414604F1080000F051F8A0B1CD
:10DF0800D8F804701820019078880090BB88BA6807
:10DF18003988608800F0E4F90646162E02D1002000
:10DF2800B8602DE060B3388828E000270EE0019043
:10DF380068880090AB88AA68608800F0D1F9064626
:10DF4800162E18D10020A8607F1CFFB25F48407EC3
:10DF5800874215DAD8F804100C227A430A44154689
:10DF680029880B000CD07B1C83421DBF9089002898
:10DF780016201820DBE7002EE6D02888A9F8000034
:10DF8800404600F080F82EB9608801F024FA20B1EC
:10DF9800162003E0162E08BF00263046BDE8FE8393
:10DFA8002DE9F84F0C460020002700264FF00C0BF7
:10DFB80046490DE0984202BFBCF8025093B2AB420A
:10DFC80024D1BCF80430DF19BFB29A1892B2761C7B
:10DFD8004B7E9E420FDA63680BFB06FC9C44BCF840
:10DFE800003043B10028E5D1BCF80470BCF8022029
:10DFF8001846BA18EAE7022E2DDB38004FF0000960
:10E0080004D002F08FFC5FEA000801D1002023E071
:10E01800CA461AE00BFB0AF14518A96859B1AA8843
:10E0280008EB090000F04BFCA88848441FFA80F967
:10E03800A86802F08EFCBAF1000F04D00C2200216F
:10E04800284600F06EFC0AF1010AB2456068E1DB7F
:10E05800C0F8088087800120BDE8F28F10B51B4A00
:10E06800D269002100E0491C194C2478CBB2A342A4
:10E0780007D2C9B232F831308342F4D102EBC10081
:10E0880010BD002010BD70B5044600250BE0B06837
:10E0980008B102F05EFC0C220021304600F041FC81
:10E0A800002030806D1C0949497EE8B2884207D2B9
:10E0B8006068EDB20C216943461830880028E6D123
:10E0C8004FF6FF70208070BDF7460020E44700201F
:10E0D8002048002071E300000848002080B5FFF7C1
:10E0E800F3FA00B1806802BD2DE9FE4F0D46804667
:10E0F800287AC00693461E464FF0000A0CD55846AB
:10E10800FFF7ECFF030000F0E4800A2229464046AE
:10E1180098470028824649D128780C9F0D9CDDF845
:10E128003890022816D100F018F94FF42051401AFF
:10E13800012810D9801E3AD0401E14D0FD3876D060
:10E14800401E00F07D80401E6AD0401E6FD0401EE9
:10E1580000F09180A7E0002C2AD1E8680178398086
:10E168000278416883E0002C22D101203880002108
:10E17800E868007830706889401C80B201F084FC3F
:10E18800398860B10278921C5118398041897170C0
:10E198004189090AB17002784168F01C68E0081DDD
:10E1A800388004220021701C00F0BBFB93E0002C97
:10E1B80062D1E8680488042038803470200A7070BE
:10E1C8000DF10201204601F05FFC05001ED0EC684D
:10E1D800BDF802204FF6FF786B46414601F07AFC05
:10E1E80040B92B786A688348022105F069F908B9B3
:10E1F800ADF80080207802280AD161680222301D1B
:10E2080000F05DFB3888801C388001E0ADF80040E4
:10E21800BDF80000B070BDF80000000AF0705AE0C8
:10E2280054BBE8680168404605F0CAFA02E01CBB26
:10E23800E8680088022139803070000A70704AE06E
:10E24800E86800F03AFB82B2A242B8BF4FF0070A72
:10E2580041DB944208BF002206D009EB0401914239
:10E26800B2BF4A46121B92B23A80E968214430464E
:10E2780000F025FB2FE014B14FF00B0A2BE0E86803
:10E288000721398001783170417871704188B17007
:10E298004188090AF17001793171C1887171C088AA
:10E2A800000AB07117E05846FFF70EFA00281CBFA5
:10E2B800D0F800C0BCF1000F0BD00F980290CDF839
:10E2C800049000943B46324629464046E047824641
:10E2D80001E04FF00E0A5046BDE8FE8FF4450020DD
:10E2E8002DE9FE438046894617461E4602A9484640
:10E2F80001F0CAFB05002CD0BDF80800FFF7E4F9CF
:10E3080000281CBFD0F804C0BCF1000F1FD00A9829
:10E318000B9C0090019433463A4629464046E04714
:10E328000646B8B9FE2C15D02878022812D100F07C
:10E3380014F842F6021188420CD13878797800EB4B
:10E34800012082B24946404600F038F802E00E2625
:10E3580000E001263046BDE8FE8368680178407811
:10E3680001EB002080B270477CB50129044605D036
:10E37800022922D1012104F0D4FAF0B92046FFF78E
:10E388006DFE08B1FFF77FFE01A800904FF6FF75FC
:10E398000223194A2946012001F047FB0BE0F068E7
:10E3A8000168204605F0F2F9BDF80420002329464B
:10E3B800304601F08FFB0600F1D173BDF8B50F4F61
:10E3C80004463878FF280D46164611D00A2000F07A
:10E3D800C5FA68B1B1210170448000214170017112
:10E3E800C580068101463878BDE8F44000F0D7BA08
:10E3F800F1BD0000BCBC0100C8BC0100F74600200C
:10E40800002010B5DFF8F0436070207082B000F093
:10E41800E8F8002100F0E2F80098B0F5801F02D17A
:10E4280000F0C7F80BE020B900F0C3F800F001F9DC
:10E4380005E000F0A1F800F08FF804206080607813
:10E4480016BD13B5DFF8B003BDF8021040881C46AE
:10E45800C9B200F0CBF8010009D0DFF8A003049A94
:10E468000003A3B2000E05F0C7F9002016BD012075
:10E4780016BD2DE9FB43DFF8806382B00020707081
:10E488001746BDF80A90708898465FFA89F100F03F
:10E49800ADF80446B8B1002501E0641C6D1CEDB26E
:10E4A800B9B28D420CD2D5480003012301AAA1B20A
:10E4B80000F094F89DF8040018F805108842ECD094
:10E4C800B8B285423ED0BFB2F81C411000EB917043
:10E4D800801087007088BFB23818001DB0F5805FC3
:10E4E80003DD00F041F800F0A4F874884FF6FF70DF
:10E4F800ADF800003D1947F4004000F027F8BDF8DA
:10E508000200C0F30E0000F021F8BA05120E4146D1
:10E51800204600F016F95FFA89F141F40040ADF8A1
:10E52800000000F015F8BDF80000C0F30E00ADF8CB
:10E53800000000F00DF87078010004D17088391DD2
:10E5480008187080002005B0BDE8F083ADF802001F
:10E5580001226946A8B2F4E080B54FF4801000901B
:10E5680001226946002004E080B5002000900122C5
:10E57800694600F0E6F801BD70B5A148006880471B
:10E58800044600F023F905469C4800030021000ECC
:10E5980005F053F905F05CF90646284600F00EF937
:10E5A8000EB100F006F92046BDE8704095490968AB
:10E5B800084710B582B040F6FC7400F012F8214606
:10E5C80000F00CF8009810F1010F03D1241FA4B239
:10E5D800042CF2DA8849201D488013BD000E05F08E
:10E5E8000BB98648000304236A46704738B50C46C1
:10E5F800051F00E02D1FADB2042D18DBFFF7F1FF5A
:10E608002946FFF7EBFFBDF80010BDF80200A14254
:10E6180003D1C0B2281A80B232BD0104EAD4011D68
:10E628008D42A8BF281AE3DA002005F030F900204F
:10E6380032BD2DE9F04F83B000F0C8F86E4FDFF817
:10E64800BC9183467888041F4FF0FF080025A4B2C8
:10E658004FEA193A2DE04FF088508119042201A899
:10E6680005F024F9BDF804005FFA88F188421BD050
:10E67800BDF80600301A061FB6B2301F40F6FC710E
:10E688008842E8D3BDF802004FF088514A19031DAB
:10E69800211A9BB289B25FFA8AF005F0ADF8BDF88D
:10E6A80002004019051DADB2BDF80200201A041F72
:10E6B800A4B2042C2ADB04236A4621465FFA8AF0B6
:10E6C80005F09AF8BDF800004FF6FF71884218BFB0
:10E6D800002810D1BDF80200010448BF241FE7D468
:10E6E800001D8442E0DA002005F0D1F8584600F019
:10E6F80065F8002023E00004D6D4BDF800005FFAD6
:10E7080088F18842D0D080462E1FB5E7FFF734FF46
:10E7180045B12A464FF0885109F1040005F088F800
:10E72800FFF71AFF584600F049F8787828B9281DED
:10E738007880C5F5805080B201E000207880BDE87F
:10E74800FE8F2DE9F04705462C480E46040B82B093
:10E7580017462946E0B205F070F881462848006857
:10E768008047804600F032F88246BA003146484673
:10E7780005F05EF8504600F021F801E02D1D361D29
:10E788003846471EC0B270B104236A46A9B2E0B247
:10E7980005F032F804223146684605F0C3F800282F
:10E7A800ECD000F006F84046164909688847BDE8ED
:10E7B800F3871148012141700170704728B1124A4E
:10E7C80012481268526801211047704738B50F4C3B
:10E7D800204605F0D9F80546C0B250B10A4A126879
:10E7E8005268002120469047204605F0CDF80028C1
:10E7F800FAD1E8B232BD0000F046002000E0010086
:10E80800A0470020A4470020D80100100040034082
:10E818000020F5E5E0B5ADF806000B460020ADF8A0
:10E8280008008DF804000092DDE901010022FFF7DD
:10E8380008FE0EBD82B01346ADF802000A4600205D
:10E84800ADF804008DF80000DDE9000102B010E623
:10E8580000B583B00821ADF8001001900B21ADF888
:10E8680002106846DFF88416096888470EBD1FB590
:10E878008DF806100824ADF800408DF80400062431
:10E88800DFF868168DF808200393ADF80240684653
:10E898000968884704B010BD80B5052004F0F7FF6B
:10E8A80000F0EEF90C2000F001F802BDDFF83C168C
:10E8B8000968ADF802006846084705F06DB803E03E
:10E8C80011F8013B00F8013B13465A1E002BF7D103
:10E8D80070471144491E03E011F8013900F8013B63
:10E8E80013465A1E002BF7D1704770B504460D46E3
:10E8F800A8B200F00DFB060003D02A462146FFF718
:10E90800DEFF304670BD10B513465A1E3BB110F8F5
:10E91800013B11F8014BA342F6D0002010BD0120A5
:10E9280010BD10B5044610460A460146204605F0BB
:10E938004FF8204610BD00F083BFDFF8B425DFF89C
:10E94800B435126A11541B7805E0DFF8A835DFF8F2
:10E95800A0251B78126AC0181154704710B504001E
:10E9680001D1002010BD04F10C0080B200F0D0FAF3
:10E9780028B1002101600481FF2181720C3010BD93
:10E9880080B508B9052002BD10F8021CFF2901D086
:10E99800042002BD0C3800F0C8FA002002BD38B5CA
:10E9A8000C46010622D5DFF848150A78FF2A08BF69
:10E9B8004D7805D0DFF83C351B78096A9A188D5CCC
:10E9C800FF2D02D1FFF768FF0EE000F09CF9014629
:10E9D800FF2004F8020C234600222846FFF747FFD1
:10E9E80048B12046FFF7CCFF012032BD2146BDE8E3
:10E9F8003840002201E032BD012270B50D00044606
:10EA0800164618D0200648BFFFF746FFDFF8E41483
:10EA180009788C4204D32846FFF7B2FF032070BD63
:10EA2800A5F10C000168002904BF817AFF2904D0F0
:10EA38002846FFF7A5FF052070BD8472012EDFF878
:10EA4800B004294603D1001D00F055F802E0001D6E
:10EA580000F039F800F033F8002070BD2DE9F041DE
:10EA68000446DFF89404DFF888740068804780461D
:10EA780078680026002503E005B9064650F80C0C16
:10EA880050B110F8021CA142F6D1002D08BF05466E
:10EA9800F4D000F014F805E04FF40041204600F0EF
:10EAA800A4F825B132462946381D00F031F8DFF8C0
:10EAB8004C140968404688472846BDE8F0814FF461
:10EAC8000041204642E038B500F00FF8002145F833
:10EAD8000C1C216811B9256006E0114651F80C2C70
:10EAE800002AFAD141F80C5C26E10446DFF8080454
:10EAF80000680D46004738B5FFF7F7FF216845F86D
:10EB08000C1C2560DFF8F4130968BDE83440084799
:10EB180070B5044600F014F8A5F10C0123680A68E2
:10EB28009D420CBF226046F80C2C00220A60FF228E
:10EB38008A72BDE8704001E1DFF8C0130968084730
:10EB4800DFF8B40300680D46164600472DE9F0418A
:10EB58000446DFF8A003DFF8985390F800802006F9
:10EB68000E462CD50420FFF7F9FE070008BF042045
:10EB780039D04FF6FF7038807E80A7F10C062878D0
:10EB8800FF280FBF6D78296A40440D5CFF2D05D121
:10EB98003846FFF7F5FEFFF77FFE0EE0204600F04F
:10EBA800B2F8FF21B1723B46014600222846FFF722
:10EBB8005EFEC0B13846FFF7E3FE012013E044458E
:10EBC80010D200F028F8DFF83813096831F814205B
:10EBD800324321F81420FFF7AFFFE868FFF738FE4B
:10EBE800002000E00320BDE8F08138B50C46C1499B
:10EBF8000978884205460CD200F00DF8C04909682A
:10EC080031F81520A24321F81520FFF795FF0020C1
:10EC180032BD032032BDB8480068004730B5B44C57
:10EC28000020606083B004F015FF05F062F8B14879
:10EC38000578680000F06CF920626A00FF21FFF790
:10EC480070FE0222FF21A01CFFF76BFE05F0A8F85A
:10EC580000F016F81420A54D2968ADF802006846A2
:10EC680088470198206100F00BF81520ADF80200E4
:10EC78006846296888470198801E606100203EBD6B
:10EC88000820ADF80000704730B587B00820ADF80F
:10EC980008001B20ADF80A0001200390944D0FF2E4
:10ECA8007D00924C21680590E8690690A869049057
:10ECB80002A888470499A96108B1FFF7EDFD00F0A3
:10ECC80052F8FFF7DDFF0A20ADF802004FF0FF30E1
:10ECD8000190684621688847F1E780B50021844A99
:10ECE8000A449378FF2B01D1907001E0834203D14D
:10ECF80041F08000C0B202BD491C0229EFD3FFF7E2
:10ED0800CBFDFF2002BD10B580F08004022CA8BF07
:10ED1800FFF7C2FD76482044807810BD38B5044618
:10ED2800FFF779FF05467248C1698C4204BFC06885
:10ED3800FFF78EFD4FEA0500BDE834406F490968CA
:10ED4800084710B50446608850B9A079FFF7C5FF99
:10ED5800FF28E07102D16FF0030010BD002010BD44
:10ED68006FF0010010BD2DE9F04F8BB004F095FF56
:10ED780000245FEA000B03D004F0A1FE4FF0FF3B34
:10ED88005B4DA868010003D0804701E0FFF784FDD0
:10ED98000820ADF808000720544E3168ADF80A0085
:10EDA80002A8884753499DF80E20049F0978E8B9BE
:10EDB800002600E0761C8E42E8D2286A805D9042E8
:10EDC800F8D1F6B2FF2EE1D017F8080CFFF785FF4F
:10EDD80017F8061C012908BF387002D0022908BF9D
:10EDE800B87039463046FFF7DAFDD1E7444F386846
:10EDF800E4B230F8140018B9641CE0B28842F5D3C4
:10EE0800E0B28842DFF8F480DFF8EC901DD2D9F840
:10EE1800000080473968E4B231F814A0002200F0FD
:10EE280047F8384A2C70514652F82420204690471B
:10EE38008246FF202870D9F800008047396831F8E9
:10EE480014204AEA020200F033F804F026FF0746CD
:10EE58005F452AD007B92C4F6869B84238BF0746C2
:10EE6800D9F8000080470446FFF70AFF1C20ADF8D8
:10EE78000200A86931680190684688470821E86956
:10EE8800ADF81410401C1321E861ADF81610099074
:10EE980006971E49A8690891079005A83168884710
:10EEA8000798A861204600F005F80BB0BDE8F08F80
:10EEB80021F81420D8F80010084701700A0A427097
:10EEC8000A0C090E8270C170001D704710B548B158
:10EED800002300E05B1CDCB2944205D2DBB2C45CC8
:10EEE8008C42F7D0002010BD012010BD9C470020A7
:10EEF800784400202C9B0000A0470020A447002055
:10EF0800B4470020089B00008EC2F52825ED0000BC
:10EF1800E0B50821ADF800100190042100F00FF8C9
:10EF280008B100200EBD02980EBD00B583B00821BF
:10EF3800ADF800100190052100F001F807BDADF80B
:10EF48000210684601490968084700009C470020EC
:10EF5800DFF800F0F5950010DFF800F031960010AA
:10EF6800DFF800F05D9600100A4610B5052A18BFB4
:10EF7800042A03D0062A18BF072A08D10C24514BAB
:10EF880062431A4422F8301D9070002010BD022000
:10EF980010BD38B50D4604462888052818BF042832
:10EFA80003D0062818BF072801D1686808B90220CD
:10EFB80032BD0121204603F0B4FC08B9142032BD4B
:10EFC8004FF6FE70844207D0204603F0E6FC2989FC
:10EFD800884201D21B2032BD3B48007800282946D0
:10EFE800204603D0BDE8344001F046BABDE83440BD
:10EFF80001F0F8B980B5354B009313460A46012154
:10F008002CE0E0B5019200230522009202930A4603
:10F018002F4B0A2101F07CF90EBD70B50D4684B066
:10F0280004461646EB88AA886988288800F034FACE
:10F0380058B1002002900196042000902A46254BE2
:10F048001221204601F064F900E0182004B070BDD8
:10F0580080B5214B009313460A46132101F08AF923
:10F0680002BD38B504461D480129017011D11C485C
:10F078000088051DADB20120FFF76AFF94FBF5F08B
:10F0880082B2284601B0BDE8304000230021FFF7D6
:10F0980063BFBDE832400020FFF75ABF03B50F48F1
:10F0A8000078012881B003D102AA01A9FFF758FF0F
:10F0B80007BD0B4A001F10800348017070470848BD
:10F0C8000088704758480020DE460020810501006E
:10F0D80071060100FF05010065060100DB480020FC
:10F0E800F4460020704700005D490860704738B555
:10F0F8000D460446288817280ADBFFF7E0FF298811
:10F10800884205D3002000902B460222554987E00B
:10F11800022032BD80B500F031F80422524900E0E7
:10F12800524904F08AF902BD38B50D4604462879DB
:10F13800022809D1E86810B1072101F02FFC0090DE
:10F148002B4606224A496BE0022032BD80B50A7977
:10F15800102A18BF022A03D100F010F80822DFE7AE
:10F16800022002BD80B500F009F80A224149D8E71B
:10F1780080B500F003F80C223F49D2E70022009244
:10F188000B46704738B50D460446A888022809DBA7
:10F19800286838B1012101F001FC00902B460E22AD
:10F1A80036493DE0022032BD80B50A79102A18BFE1
:10F1B800022A03D1FFF7E2FF1022B1E7022002BDC5
:10F1C80070B50D4682B00446287A1226012809D166
:10F1D800204604F0C6F969880F38884201DA02200F
:10F1E80076BD9226687A0128686808BF46F040060E
:10F1F80010B1032101F0D2FB00902B463246204982
:10F20800204604F01AF976BD38B50D460446A868BC
:10F2180010B1052101F0C2FB00902B4616221949B6
:10F22800204604F00AF932BD80B5FFF7A7FF18227F
:10F23800154976E738B504460020009000231E22C1
:10F248000021204604F0F9F8050006D104480268B8
:10F25800100002D01E2120469047284632BD0000EB
:10F26800D04700209F300100D1300100B7310100A4
:10F2780039310100473201009F320100EF320100AD
:10F28800933201005B330100D53301006E490860F9
:10F29800704780B5002200920B4601226B4900F0AE
:10F2A800BAF802BD80B50A88172A05DB0022009249
:10F2B8000B4603226649F2E7022002BD38B50D4627
:10F2C8000446A878012818BF02280DD128880028EC
:10F2D8001CBF6868002807D0022101F05FFB00907E
:10F2E8002B4605225B4931E0022032BD38B500F0DB
:10F2F8001EF81CBF6868002806D000F036F8009099
:10F308002B460722544921E0022032BD38B500F0CF
:10F318000EF81CBF6868002807D0022101F03EFBE8
:10F3280000902B4609224D4910E0022032BD0D46BF
:10F33800044628880028704738B500F024F808B13A
:10F3480000F013F800902B460B224549204600F0A8
:10F3580062F832BD38B500F016F808B100F005F8CB
:10F3680000902B460D223F49F0E7012101F016BB22
:10F3780038B500F008F808B1FFF7F7FF00902B4602
:10F388000F223949E2E70D4604466868704738B5E8
:10F39800FFF7CDFF1CBF6868002807D0022101F0E5
:10F3A800FDFA00902B4611223049CFE7022032BDEA
:10F3B80080B5002100910023132270E738B50D466F
:10F3C8000446A86810B1052101F0E8FA00902B4620
:10F3D80017222749BAE780B5002100910023192296
:10F3E8005DE738B5FFF7CFFF10B1032101F0D6FA7A
:10F3F80000902B461B2209E038B5FFF7C4FF10B177
:10F40800032101F0CBFA00902B461D221949204612
:10F4180004F013F832BDF8B5044606980090154676
:10F428001E46204604F009F807000AD1064802687B
:10F43800100006D0012D04BF3078451CE9B22046E3
:10F4480090473846F2BD0000CC4700206F300100DD
:10F45800AB300100DD30010095310100233201009D
:10F4680063320100DD320100173301001D33010052
:10F4780085330100F9330100DFF800F0DD8A001060
:10F48800DFF800F0A18B0010DFF800F0D570001055
:10F49800DFF800F09D58001030B540F67B44851F1A
:10F4A800A5423CBF8D1FA54212D2814210D3B2F5AE
:10F4B800FA7F0DDAA3F10A0040F67744A04207D29A
:10F4C800501C49004843B0EBC30F8041C00F30BD0A
:10F4D800002030BD80B505F0FBFA8DF8000006F07D
:10F4E80053FD9D49002008706A469C490880012107
:10F4F80040F603407CE080B50FF2F822412141F24A
:10F508000200FFF7B9FF002002BD7CB5002808BF44
:10F5180000294FF620442DD162BB01A806F094FCC7
:10F528009DF8040000EBC000451DEDB22846FFF72A
:10F53800EFFC060018D020203070042070700020E6
:10F54800B0709DF8040000280CBF0022721D311D08
:10F55800F01C05F047FB32462946204606F0C5FF59
:10F568003046FFF7E2FC15E004218DF80110202059
:10F57800072106E005F036FB04218DF80110202054
:10F5880000218DF800008DF802106A4603212046FC
:10F5980006F0ABFF002076BD1CB504460DF1030153
:10F5A80005F078FB00F01DF9052140F67B4008E0E6
:10F5B80010B582B0044605F07DFB00F040F840F637
:10F5C8007C40FFF759FF002016BD80B500208DF85C
:10F5D80000006A46624800788DF801000421002086
:10F5E8008DF802005F4800788DF8030042F20200AF
:10F5F800FFF742FF002002BD1FB50446089802909D
:10F608000798019006980090204605F0A7FF8DF80E
:10F618000C008DF80D40200A8DF80E0003AA032176
:10F6280042F22000FFF728FF5CE010B582B00446E4
:10F6380005F0D6FF00F003F842F22100C1E78DF88B
:10F6480000008DF80140200A8DF802006A46032167
:10F65800704738B5044642F2160529460020FFF7E0
:10F668000FFF204605F017FC8DF8000020B16A4610
:10F6780001212846FFF700FF002032BD80B5012395
:10F6880005F0FEFD00F01BF842F21E00B0E780B561
:10F69800012105F0B5FE00F012F842F21D00A7E7BF
:10F6A80080B530B1014608222F48FFF708F900203D
:10F6B80000E0122000F003F840F6634098E78DF868
:10F6C80000006A460121704710B584B0089C029476
:10F6D800079C0194069C009405F0ACFF42F21301CC
:10F6E800FFF7CEFE002004B010BD80B51D218DF8B7
:10F6F800001004218DF8011010B9FFF7C5FE00E0D5
:10F7080011208DF802006A4603214FF61D400DE0D6
:10F7180080B51C208DF800006A4604208DF8010091
:10F7280003210C208DF802004FF61C4006F0DDFE88
:10F73800002002BD06F0B6BB80B530B10B49027897
:10F748000A7040784870002000E01220FFF7B7FFE9
:10F7580042F201004CE70000244F0020264F002011
:10F768004C4300204E430020904800208848002049
:10F7780000B585B06A460DF1020101A8FFF788FEC1
:10F788008DF80800222107208DF8090002AA02A896
:10F79800817002218DF80B109DF804108DF80C1063
:10F7A800BDF802108DF80D10090A8DF80E10BDF87D
:10F7B8000010C171090A017241F201000921FFF725
:10F7C8005BFE002005B000BD10B582B004460DF107
:10F7D800030106F03FFB00F004F8042141F2054064
:10F7E800EFE68DF800008DF80140200A8DF8020040
:10F7F8006A467047002000800000C000000000E456
:10F808000000002822000000000000040000F7FFAC
:10F81800FF7F000000303000000000000000000002
:10F8280000000000000000000000000000000000D0
:10F838000000000000000000DFF800F00158001090
:10F8480080B502216846FFF7F7FFBDF8000002BD4A
:10F858007047704770B5DFF8385A28780624604337
:10F86800FFF756FBDFF82C1A086008B9132070BDA3
:10F878000020FF2206E03380401C0023F270B270A3
:10F888003371C0B22B7898420ADA0B6804FB00F691
:10F898001E4400280CBF4FF6FE734FF6FF73EAE7CD
:10F8A8000FF25140FCF7CCFD0FF61510FFF7EEFCF8
:10F8B8000FF6551002F077FF002070BD70B50446B2
:10F8C800208868B160680378426800F040F948B958
:10F8D800606803784268DFF8C00900F03AF908B9AF
:10F8E800022070BDA078C01F0A2801D3182070BD5F
:10F8F800DFF8A8592888010004D02188C0F5803095
:10F90800884201DA012070BD0C20FFF701FB0600D8
:10F9180001D1132070BD002008E06268298880B2F8
:10F9280002EB0012401C5181491C298081B22288B7
:10F938009142F2D30020306008222146301DFEF7A4
:10F94800BEFF686810B96E6004E0084601680029C7
:10F95800FBD10660002070BD38B502460846DFF8C6
:10F968003C194C68002301E02346246894B1A5683B
:10F978006D899542F8D12268002B0CBF4A601A6045
:10F9880018B10822211DFEF79AFF2046FFF7CDFA8D
:10F99800002032BD012032BDDFF80419087070471D
:10F9A80010B5044610461422114203D000F0DAF8CC
:10F9B800012204E04A0608D500F0D4F800220146E6
:10F9C8002046BDE8104002F0EEBFC80701D402206F
:10F9D80010BD002010BD70B505460E46B0061C4689
:10F9E80009D5104600F0BEF801462846BDE870402B
:10F9F800012202F0D8BF8820064210D0104600F03D
:10FA0800B1F8014606F00802284602F0CCFF0100D2
:10FA180009D0617A41B1217A012904D070BDB007BB
:10FA280001D4032070BD002070BD2DE9F047814648
:10FA3800DFF8680844688A4690461E4600E0246855
:10FA4800FCB1002700E07F1CA188B8B28842F6D23A
:10FA5800A068BFB200EB07156889484528BF8245F2
:10FA6800F1D33EB1297868683346424603F028FD51
:10FA78000028E8D0089810B1A16849890180284673
:10FA880000E00020BDE8F087F0B5DFF810285468E2
:10FA980000E02468E4B1A5686E89B042F9DBA78864
:10FAA800BA199042F5DA4FF0000C01E003F1010CAD
:10FAB8001FFA8CF2BA42ECD21FFA8CF305EB031250
:10FAC800B2F80AE08645F1D101B10E801046F0BDCA
:10FAD8000020F0BD2DE9FC4104460027ADF8047074
:10FAE8004FF6FF786089404515461E4608D001AAA2
:10FAF8000092401C2378626880B2FFF796FF0746A1
:10FB08002378626800F023F830B923786268DFF858
:10FB1800880700F01EF808B160890CE02378626855
:10FB2800DFF8800700F015F858B11FB1BDF80400E0
:10FB3800A84203D0284600F0D2F803E07889404470
:10FB480000E0608906B130803846BDE8F681DFF80C
:10FB58005807022103F0B4BC80B500F0F3FA00B1F5
:10FB6800008802BD80B500F0EDFA08B1807802BDCA
:10FB7800102002BD70B5012982B00446154616D082
:10FB8800032918D0052925D0072927D0092929D0E4
:10FB98000B292BD00D292DD00F292FD0112931D089
:10FBA800132933D0172934D0192936D039E02946FA
:10FBB800FFF76FFB33E0FFF782FAADF80000694604
:10FBC8002046FFF76FFB06002CD129882046FCF75A
:10FBD80019FD27E02946FFF771FB20E02946FFF7CA
:10FBE80085FB1CE02946FFF791FB18E02946FFF743
:10FBF800A3FB14E02946FFF7ADFB10E02946FFF709
:10FC0800B7FB0CE02946FFF7C2FB08E0FFF7D0FB83
:10FC180005E02946FFF7D2FB01E0FFF7DCFB0646CB
:10FC280000E00226304676BD2DE9FC410E46054629
:10FC380017461C4601A900F092FA804638BB3800E6
:10FC480014D00020ADF8000069463088FFF71CFF8B
:10FC5800012FBDF8000018BF0027FFF783FF0146FA
:10FC68003A46284602F09FFE804680B9314628462B
:10FC7800FFF7C2FB804650B9019DFF2C07D0AB1C93
:10FC88001E2229460FF25550FCF79EFCEC704046A8
:10FC9800BDE8F6817CB50D460446164601A900F07C
:10FCA8005EFA17281AD0300014D00020ADF80000F2
:10FCB80069462888FFF7E8FE012EBDF8000018BF46
:10FCC8000026FFF74FFF01463246204602F06BFE42
:10FCD800010003D129462046FFF783FB76BD10B506
:10FCE8000446FFF739FF01001CBF611E0C18A0B2C3
:10FCF80010BD00002DE9F0430D4689B08146A87873
:10FD080000261E28174614D1484600F03CFA060083
:10FD18001EBFB078FE28FF2822D0002000900022C5
:10FD2800AB78F0784946FCF724FC304600F040FAFE
:10FD380016E0122804BF6878012813D0484600F05E
:10FD480022FA06000ED0327910000BD0100607D424
:10FD5800A9784846FCF769FC307940F0800030719A
:10FD6800002069E0DFF838452078FF2812D0A8780D
:10FD7800811E17290ED200F08AF958B1A87800F030
:10FD8800B3F938B1287810B96878012804D1A8786F
:10FD9800122801D006204FE0A87800F078F98446B0
:10FDA80002A80090AB88AA6869782878E0470028FC
:10FDB800804640D1A87800F097F9024602A9484643
:10FDC80090478046D8B9AB78042B34D002A800906D
:10FDD800002220784946FCF7CCFB804658BBA9781E
:10FDE80002A8FCF739FC08B100203870A87812285E
:10FDF80004BF697801291ED0EEB130711BE0687824
:10FE0800C8B9A8788DF800008DF804806946A878EC
:10FE1800042818BF0628BDF80800ADF802004846B7
:10FE2800FFF737FA28B16B46012216214846FCF73E
:10FE3800DFFB4FF00008404609B0BDE8F083002022
:10FE480070472DE9FE430D4680462888698881421F
:10FE580001D3010001D101206DE00021ADF80410AB
:10FE680002914FF6FF7900E0401C00210091002329
:10FE78006988002280B2FFF7D8FD070037D0BDF8A7
:10FE88000400002838D16B464A4605214046FCF755
:10FE98000DFC040001D111204DE0029438780228AD
:10FEA80006D101208DF80600BDF80000860827E07D
:10FEB80002208DF806001221BDF8000090FBF1F633
:10FEC8003878102813D1788904F8010B102200F033
:10FED80034F81034BDF80400401CADF80400B1B289
:10FEE800BDF80400884202D278894845BCD1BDF8E3
:10FEF800040080B90A201EE09DF806000128DFD121
:10FF080038780228F3D1788904F8010B022200F02E
:10FF180014F8A41CDEE701A94046FFF7CFF948B161
:10FF280001AB052216214046FCF762FB10B102988E
:10FF380000F00FFD0020BDE8FE837889000A04F870
:10FF4800010B20467968FEF7BABC10B582B04C8820
:10FF58000888844201D3020001D1012016BD00F0B7
:10FF680016F808B90A2016BD002016BD10B582B0D3
:10FF78004C880888844201D3020001D1012016BDB3
:10FF880000F005F808B90A2016BD002016BD0022A9
:10FF980000924A1D0B79214647E510B5044682B008
:10FFA800084669460088FFF76FFD08B9012016BDAD
:10FFB800017ABDF800202046FFF7F2FC16BD70B5A7
:10FFC80082B006460D46002401E0641CA4B2A8884D
:10FFD800844229DA286810F8142000EB44006946A6
:10FFE800407802EB002080B2FFF74EFD50B9286838
:08FFF80010F8141001702868D4
:020000040001F9
:1000000000EB440149784170012076BD017ABDF8CA
:1000100000203046FFF7C8FC0100DAD0296811F84B
:1000200014200A70296801EB440252784A7076BDA8
:10003000002076BD10B50C4682B0208861888142D0
:1000400000D308B9012016BD23799948621DFFF736
:1000500084FD08B9102016BD002000902379618826
:100060002088621DFFF7E5FC08B90A2016BD0020B4
:1000700016BD38B504460D4669462888FFF708FDC9
:1000800008B9012032BD017ABDF800202B46204678
:10009000FFF7A5FC32BD022814D0042814D006288E
:1000A00014D008281AD00A2812D00C2812D00E28F2
:1000B00012D0102812D0122812D0162812D01828C8
:1000C00012D013E07B4870477B4870477B487047ED
:1000D0007B4870477B4870477B4870477B48704738
:1000E0007B4870477B4870477B48704700207047CB
:1000F000022814D0042814D0062814D0082814D0BC
:100100000A2818BF0C2812D00E2812D0102812D09E
:10011000122818BF162810D0182810D012E06F48E7
:1001200070476F4870476F4870476F4870476F4817
:1001300070476F4870476F4870476F4870470FF2BD
:1001400009007047002070470020704755494968F2
:1001500000E0096829B18A6852898242F9D1081DF4
:1001600070470020704710B50C4600F010F860B1E1
:1001700004B120608078FE2801D1172010BDFF282F
:1001800001D1002010BD162010BD022010BD10B5F9
:10019000424A1268002100E0491C3F4C2478CBB24F
:1001A000A34207D2C9B206234B43D45A8442F3D1A7
:1001B000D01810BD002010BD10B50446A01CFCF7DF
:1001C0000FFAFF20E07010BD10B50C46FFF7DFFFFF
:1001D00030B101794A1C944204BF01F080010171E1
:1001E00010BD000010B582B004001EBFA078FF282B
:1001F000FE280BD0002000901E232188E0781722D3
:10020000FCF7BBF9FE20A070FF20E07013BD0000DA
:1002100070B504464FF6FE70844282B037D00800B5
:100220004FF6FF760AD12046FFF7B1FF78BB304684
:10023000FFF7ADFF05002AD0048073BD012906D168
:100240002046FFF7A4FF050021D02E800BE00229F5
:100250001DD10121204602F068FBC0B92046FFF7FE
:1002600096FF050013D0A878FF280ED0FE2807D0EF
:10027000002000901E23E87814222146FCF77DF927
:100280002846FFF799FFFF20A8700020287173BD52
:100290000448008870470000D84800201848002013
:1002A000BCBC010004460020FA460020C4BC01008A
:1002B000B8BC0100A1300100D3300100533101006E
:1002C00049320100B9320100F7320100E731010083
:1002D000693201005D330100DD33010047FE00009B
:1002E0004BFE000053FF000075FF0000A3FF00005D
:1002F000C7FF00003500010073000100DFF800F0C7
:10030000E99400100A7802704A7842708A78C978B5
:1003100002EB0121418070472DE9FC410D46164654
:100320001F460A9A0999044601AB00F021FA80465B
:1003300008BB0199089808703346DFF8B8050178C2
:10034000491CCAB2002A06BF012101220A460170D7
:10035000294601980271009701980279204600F021
:100360000DF8804620B901981E2100F046FA02E0FF
:10037000019800F026FA4046BDE8F6812DE9F041EB
:10038000044684B00E4617469846172000F0C0FA7F
:10039000050026D00A9A100003D04146281D904738
:1003A00000E00020010A2E70E9706F70A87005212E
:1003B000001DADF80800ADF8001001956946DFF8A2
:1003C000380500780028204602D000F059F801E0F6
:1003D00000F00CF80446200004D0284600F0BDFAD6
:1003E00000E01324204604B0BDE8F08110B50B886E
:1003F000DFF808250C2463431A44303A536833B9B4
:100400004B685360098950811181002010BD16206E
:1004100010BD80B5052000F00FF858B9062000F097
:100420000BF838B9042000F007F818B9072000F0DD
:1004300003F800B1012002BD0C2210B5DFF8BC1496
:1004400042431144A1F1300484B06168A9B1DFF8DE
:10045000A82412787AB1ADF800000191694620898C
:10046000ADF80800608900F00BF810B1606800F08A
:1004700074FA00206060012000E0002004B010BD8C
:1004800070B50D4604462889010004D0DFF87014C9
:100490000988814201D21B2070BD6868042100F0E8
:1004A00081FA0646288930702889000A70702888E9
:1004B000B0702888000AF0702889051D4FF6FE707C
:1004C000844213D10C20FEF74DFA01000CD090208D
:1004D00008704C8002200871CD808E60DFF8240403
:1004E0000078FEF760FA18E0132070BD3346AAB218
:1004F00000212046FFF702FF010007D002280ED09E
:10050000072810D012280CD01F280DD1DFF8E803DF
:1005100001780A001CBF491E0170002070BD142024
:1005200070BD022070BD042070BD38B504460020A7
:1005300060600879022821D1CA88042A1EDB8868F5
:1005400001784378C57801EB0321837889B203EB06
:1005500005230D1D95429BB210D1052B18BF042B0E
:1005600003D0062B18BF072B08D1218123806FF001
:10057000030100F017FA6060002032BD012032BD97
:100580000B88037002220B881B0A43700B88012B17
:1005900006D14A88827004224988090AC1700CE099
:1005A000022B0AD14A8882704A88120AC2708A884D
:1005B000027106228988090A417110467047022A91
:1005C0001BDB0A784B7802EB032202800288012AA7
:1005D00005D18A78C97802EB012141800BE0022A1B
:1005E00009D18A78CB7802EB032242800A794979D3
:1005F00002EB0121818000207047012070470A88AA
:1006000002700A88120A42704A8882704A88120A66
:10061000C2708A8802718A88120A4271CA888271FD
:10062000C988090AC17108207047082A18D10A78B8
:100630004B7802EB0322028011F8022F4B7802EB79
:100640000322428011F8022F4B7802EB03228280B2
:1006500011F8022F497802EB0121C1800020704778
:100660000120704705E0022A00D10EE0012070470A
:1006700000BF0A8802700988090A41700220704789
:10068000022A00D101E0012070470A78497802EB84
:10069000012101800020704780B54B8800F8013BA4
:1006A00004224B881B0A00F8013B0B8800F8013B31
:1006B0000B881B0A00F8013B0B8873B94B88022B8F
:1006C00004D14968FEF7FDFB082206E0032B04D1A4
:1006D0000822091DFEF7F7F80C22104602BDF8B5F6
:1006E00004460D4616461020FEF73CF9070016D0CA
:1006F000A02038707D80002078702EB10C22314609
:10070000381DFEF7E0F804E00C220021381DFEF74A
:100710000CF939462046FEF746F90020F2BD0120CB
:10072000F2BD2DE9F04180460D4616461F462020B9
:10073000FEF718F9040019D0A220207066706580B9
:10074000069820716771079929B1182204F10800F1
:10075000FEF7B9F804E0182204F10800FEF7E5F806
:1007600021464046BDE8F041FEF71DB9BDE8F081E5
:1007700070B51E0004460D4621D0012102F0D5F8C7
:10078000D8B161480078002100E0491CC9B281421B
:1007900011DA5E4B1B6803EB01125388002BF4D176
:1007A0000020107001F14000508022B1D4801572F9
:1007B0003260002070BD152070BD142070BD012076
:1007C00070BD10B5044610220021FEF7AEF823E0FC
:1007D000002200E0521C4C4909788A420BDA4B494E
:1007E000096801EB02114B88002BF3D00B7983428F
:1007F000F0D108467047002070474FF47A724A43A0
:1008000000F1090301460FF2190002F00EBF10B506
:100810000446607A02F043FFFF20607210BD0000C2
:1008200010B504001CBF6088002807D0172120469F
:1008300000F005F82046BDE81040C2E710BD1CB529
:100840000446207804280FD10020019000900A4629
:10085000E188207A1323FFF764FFE18802B0BDE846
:100860001040122205202EE013BD072170B504466A
:10087000002539BB18E025480068EDB200EB0516ED
:10088000307800281CBF707AFF280CD0F088A04276
:1008900009D13046FFF7BBFF14213046FFF7CFFFE9
:1008A0003046FFF78EFF6D1C17490978E8B2884281
:1008B000E1D30425FF222146284600F004F86D1CF0
:1008C000082DF7DB70BD10B50C240C4B60431844A9
:1008D000A0F13004608988420AD1606840B1FF2AE3
:1008E0001CBF0178914203D100F037F8002060600E
:1008F00010BD0000DA480020DE46002058480020E5
:10090000F4460020DC460020DD460020E0460020C2
:1009100080B5001D80B2F9F779FA28B1BDE804402E
:100920006FF0030100F03EB802BD000070B500F0AA
:1009300035F8054604F1080080B2FEF7EDFA06002E
:1009400005D02A48B480016831600660083628491D
:10095000096828468847304670BD38B500F01EF853
:10096000224A05461068002101E00146006878B17E
:1009700000F108039C4221BF8388C3180833A342B7
:10098000F3D3036800290CBF13600B60FEF7D1FAA4
:100990002846BDE83440164909680847044615480A
:1009A0000068004738B504460D4600F00FF8010016
:1009B0000AD06842204401F10803984221BF8B8885
:1009C000C9180831814200D2204632BD0749096862
:1009D00041B101F10802904221BF8A888A18083289
:1009E0008242F4D30846704700000000A847002068
:1009F000A4470020A0470020F8B50C460227491E56
:100A0000032915461E4606D9491F04D0891E01290F
:100A100001D9091F1CD1214600F02AFF070017D178
:100A20000799069800F038FF304600F042FF012C8D
:100A300014BF042C0025284600F072F800F032FBA9
:100A400005F0D4FD00F015FD01F0F7FD06F07EF88D
:100A50003846F2BDDFF800F015990010DFF800F01D
:100A60004199001070B5DFF810550446286882B02F
:100A700008B1112076BD00F087F801D1122076BDB3
:100A80000420FEF749FA286078B3022001F09DFDAA
:100A9000286804222146FDF716FF02F033F828B13A
:100AA0000C2000F0DCFE05460D200DE060780228E9
:100AB00005D1122000F0D3FE0546132004E01020DB
:100AC00000F0CDFE0546112000F0C9FE0646DFF815
:100AD000AC04007800F0D5FF0346E0780090324681
:100AE000A0782946FFF7B6FF76BD132076BD80B506
:100AF000DFF88414096809B9122002BD097881421F
:100B000001D0032002BDDFF878040078012103F052
:100B100033F8302000F0C8F9BDE80240002035E28B
:100B200038B5DFF8604405462078012100F0CDF8A3
:100B300000F02AF822D0257004F1080002F0CCF869
:100B40006068C8B9207801001CD005012846FEF76E
:100B5000E3F9606080B12A460021FDF7E6FE00203F
:100B600005E06268C0B20301FF21D154401C227825
:100B7000C1B29142F5D305E0132032BD00202070B0
:100B800002F0AAF8002032BDDFF8FC0300780A2149
:100B90000842704770B5012442F20B02801A09D056
:100BA000401E2FD18868007820B9DFF8CC03006898
:100BB00048BB23E088680578DFF8BC03006808B309
:100BC0002900DFF8BC6310D1407802280CBF032055
:100BD000022000F044FE020003D03078012102F030
:100BE00099FF012000F0D2F9054628000BD030789B
:100BF000012102F0C1FF284600F056F9022001F061
:100C0000E9FC00E00024204670BD80B528B9DFF87B
:100C10006803006820B100207CE7BDE8024000E0E6
:100C200001BD2DE9F8430446E07800281CBF656843
:100C3000002D48D0242000F012FE4FFA80F8002644
:100C4000DFF8349308E03861D9F8000000783946BD
:100C5000FDF7A9FE2935761CE178F0B2884232D240
:100C600095F928004045F5DB284600F09EF800285D
:100C70001CBFD9F800000028ECD0287A143080B2CC
:100C8000FDF770FE0700E5D0D02038700622002066
:100C90007870A91C0D20B8702878F87095F8280095
:100CA000F87268783871781DFDF70DFE287A387370
:100CB0000028C8D007F11400386105F109013A7B1A
:100CC000FDF701FEC0E7BDE8F183F8B5AD4E04467F
:100CD00070680D4680B3002717E000EB07108068AE
:100CE00030B1FEF726F9716801EB0711002088602A
:100CF000706800EB0710C06830B1FEF71AF9716830
:100D000001EB07110020C8607F1CA7427068E4DB7C
:100D100025B1FEF70EF900207060F1BD60B122012F
:100D20000021FDF702FE0027FF2003E071683A0171
:100D30007F1C8854A742F9DBF1BD10B5914841688A
:100D400069B1002200E0521C0478D3B2A34206D25B
:100D5000D2B21301CC5CFF2CF5D1C81810BD002015
:100D600010BD2DE9F041874E044670688846C8B131
:100D7000002701E07F1CFFB23078874212DA7068EA
:100D80003D01415DFF29F5D040194178A142F1D1E3
:100D900006224146801CFDF7BAFD0028EAD07068A3
:100DA000401900E00020BDE8F08170B5724E316856
:100DB000044682B000250020D9B1217801290BD04A
:100DC000227A04F109036946012001F0D4FB00B145
:100DD00005782178042912D031684978032918BF91
:100DE00055EA01020BD020B1012904D115F003000E
:100DF00005D1002076BD0229FBD1E807F9D560783E
:100E0000A11CFFF7AEFF0500207826D0042814BFF0
:100E1000A868E86880B3227A017891420CD104F185
:100E20000901401CFDF773FD012805D1232000F0C6
:100E300016FD002836D0DCE72078042806D0A86804
:100E4000D0B1FEF776F80020A86015E0E86898B108
:100E5000FEF76FF80020E8600EE00428C9D0FFF725
:100E60006CFF0500C5D02078287006226078687075
:100E7000A11CA81CFDF727FD207A401C80B2FEF7BC
:100E80004BF860B12178042914BFA860E860217A8A
:100E900000F8011B04F10901227AFDF714FD207A04
:100EA0000028A6D0012076BD2DE9F843DFF8C880E0
:100EB0000546D8F80000002600281EBFDFF8C490C1
:100EC000D9F80400002855D05DB9002705E03901A4
:100ED000415CFF2918BF761C7F1C99F800108F42D7
:100EE000F5DBF6B2F000083080B2FDF73BFD040000
:100EF00005D10820FDF736FD0446002613256CB306
:100F0000D020207065700120A070E67030001DD0E8
:100F100004F108056560002799F80000874217DA98
:100F2000F0B2A8B1D9F8041038010A5CFF2A0AD03F
:100F300008442A70062241786970761E811CA81C1C
:100F4000FDF7C1FC08357F1CFFB2E5E700206060BB
:100F50002146D8F800000078FDF725FD99F800003B
:100F60000021FFF7B2FED8F80000FDF7E2FF0020F5
:100F7000C8F80000BDE8F183DC470020524500209E
:100F8000E4450020B04500205145002010B504463E
:100F9000232000F064FC01002046BDE8104018BF8B
:100FA0000121C9B2FFF75ABDDFF800F05D990010CA
:100FB000DFF800F09D9900102DE9F04F05466F48CD
:100FC0000078000789B058BF122068D501F0C4FA34
:100FD00008B1102063E001F095FD69490978884265
:100FE00028BF15205BD2674C206808B1112056E05D
:100FF0000A20FDF791FF002820604ED0042001F068
:10100000E4FA20680A222946FDF75DFC2068407852
:1010100028B10E2000F023FC80460F2004E00C20B5
:1010200000F01DFC80460D2000F019FC81461C20BC
:1010300000F015FCADF820001B2000F010FC074666
:10104000192000F00CFC05461A2000F008FC0646AA
:10105000162000F004FC8246152000F000FC8346B8
:101060004948007800F00DFDBDF820202168079266
:101070000697059504960190CDF80CA0081DCDF8B3
:1010800008B00090CB788A7849464046FFF78CFF3D
:10109000040003D001F018F900E01324204609B041
:1010A000BDE8F08F3548007800074CBF3748002076
:1010B00001F03ABA10B50124C01E19D042F20A025A
:1010C000801A0DD0401E08D0401F0DD0801F17D0B1
:1010D0004DF6E672801A0FD018E001F0F5F816E030
:1010E000887800F02FF812E0887800F051F80EE0D0
:1010F000084600F056F80AE0084600F05CF806E002
:101100008878010003D006F047FB00E00024204669
:1011100010BD10B502461B4B12204FF6FE741B6823
:10112000A14205D16BB11878904206D0032010BDC2
:101130004FF6FF72914204D11BB1BDE81040FFF79A
:1011400037BF10BD010000D170470E4900B50968D6
:1011500087B081B10022059204920392029201921B
:1011600000920B1DCA78097800F0B2FF07B05DF855
:1011700004EB01F0A9B807B000BD00005145002004
:10118000204800202845002052450020DC45002052
:10119000010000D1704780B500210091002300229A
:1011A00006E080B5418900910389C2888188C078B2
:1011B00000F0D0FF01BD1FB50446607912281FD191
:1011C000E389A28961892089FEF76AF918B125208F
:1011D00000F045FB00B10120ADF80C0003AA217915
:1011E0006088FDF739FFBDF80C0048B90290019006
:1011F000E0890090A389628921896088FEF768FAF6
:101200001FBD0000DFF800F0A1980010DFF800F02B
:10121000BD980010DFF800F0D9980010DFF800F05A
:101220006D98001070B5DFF8F065054630680C4623
:1012300008B1112070BD00F0E7F801D1122070BD97
:10124000DFF8D805806800281CBF0078002801D18D
:10125000102070BD0C20FDF75FFE306040B3012010
:1012600001F0B3F9306805700021306841700A223E
:101270002146801CFDF727FB00F0C4F9040002D0D2
:1012800000F0A9FA15E0DFF898050078032810D1DE
:101290001D2000F0E4FADFF88C15088048B1DFF873
:1012A000880500784EF66022042102F04BFC00E035
:1012B0001324204670BDF8B50C46DFF87015097888
:1012C0001546052211421E4627D0012CDFF84C1589
:1012D00002D18F680FB301E0CF68F7B1202D02DA99
:1012E0002A0002D00EB90220F2BD08701F22002190
:1012F000781CFDF71AFB2A463146781CFDF7E3FA05
:101300003D70284624B1791CBDE8F440FFF77ABF50
:10131000791CBDE8F440FFF779BF1220F2BD38B563
:10132000DFF8F444216809B9122032BD09788142FE
:1013300001D0032032BDDFF8F0542878022102F0FA
:101340001BFCDFF8D814002048800421287802F024
:1013500013FCDFF8D01400200880032021684870B7
:101360000020BDE83240FFF755BFF8B5044600F055
:101370004BF801D11220F2BD1CB1207801F0F1F838
:1013800008B90220F2BD6078801C202823DA20787A
:1013900000F0A3F908B11820F2BDDFF880546B68A3
:1013A0000021002202E0B61C71181B685BB15E6868
:1013B000767828B9C9B27718BF1C202FF3DB01203B
:1013C000B61CB218F1E7D0B238B16078D2B280184A
:1013D000801C202801DB0B20F2BD0820FDF79CFDBE
:1013E00006000FD0082200F07CF8686830B100E0F9
:1013F000084601680029FBD1066000E06E60746059
:101400000020F2BD1320F2BDDFF820040078052192
:101410000842704710B500F01CF801D1002010BD43
:10142000DFF8F8335968002201E00A46096869B11B
:101430004C6824788442F8D14C680868002A14BFAC
:10144000106058600846FDF774FD00E00024204657
:1014500010BDDFF8D8130978052211427047DFF874
:10146000CC0300780521084218BF00F043B91220D0
:10147000704770B5DFF8A443A06818B1FDF759FDB7
:101480000020A060E06818B1FDF753FD0020E06087
:101490000521DFF89853287808421CD004F1100089
:1014A00001F01DFC287800260521084211D000F02B
:1014B00077F9A06060B100F013F800F071F9E06016
:1014C00010B100F00DF804E0A068FDF732FDA66051
:1014D0001326304670BD002001F001FC002070BDD5
:1014E00020220021FDF721BA2DE9F0478288DFF89C
:1014F0002863DFF82853316842F20607D31B4FF008
:10150000010805D09B1E012B60D99B1E0FD00BE05C
:101510008068007841B1020003D101204870FFF7D4
:1015200079FE01006BD038E04FF0000867E080687A
:1015300007780029F8D04878BD4C012833D100F055
:1015400058F9DFF8E492B0B1012000F088F9824642
:10155000BAF1420F0AD399F800004EF66022022138
:1015600002F0F0FAAAF13C00688010E04FF47A70C3
:1015700000FB0AFA02E000F072F98246BAF1000FAD
:1015800005D099F800005246022102F0C3FA3168F2
:1015900002204870207818B9384600F004F92EE08F
:1015A000002020702BE0207848BB0320FDF7DAF9FB
:1015B00048B1D02101704770042181700146306824
:1015C0000078FDF7F0F900F006F918E08068077878
:1015D000287842F208018A420CBF01260026FF2823
:1015E0000DD00420FDF7BEF9010008D0D02008700E
:1015F0004F7002208870CE702878FDF7D4F94046ED
:10160000BDE8F087F0B5844F386885B070B3847852
:1016100001F078FA28B10A2000F021F905460B20E4
:101620000DE000F0E6F828B1062000F018F90546B4
:10163000072004E0082000F012F90546092000F018
:101640000EF906467648007800F01BFA3968CA7A27
:10165000039203468A7A029228460A1D0192224684
:10166000C97800913146FFF7D9FD00E0012005B0AF
:10167000F0BD38B5014668486B4D02682878674C64
:1016800001291ED161880B0002D0694B1B7823B160
:1016900012B31078BDE8324041E63C29A8BFA1F161
:1016A0003C000CDA022102F067FA60884FF47A718C
:1016B00001FB00F22878022102F02CFA0020608061
:1016C00031BD4AB159490978490705D5022102F0CF
:1016D00053FA002060807CE031BD5049496800E049
:1016E000096829B14A6812788242F9D108467047E0
:1016F00000207047F8B54D480078002405210842C5
:1017000001D11220F2BD454DA86810B900F048F88B
:10171000A860E86810B900F043F8E860A8680028FD
:101720001CBFE968002901D11320F2BDFFF7D8FEE4
:10173000E868FFF7D5FE6E6812E09B1C5018591838
:10174000401C117071684978491C017071680978F2
:101750004170801C71684A784968FDF7B4F83668B2
:10176000AA6896B13CB97068117843785F18BF1CBD
:10177000202FE2DB01247368E9685B780A789B1C00
:1017800088189A18401C0A70DCE71078511CFFF783
:1017900039FDE868411C0078FFF738FD0020F2BDF4
:1017A0002020FDF7B9BB38B51B4D0446286878B139
:1017B0000320FDF7D7F848B1D02101704470032110
:1017C0008170014628680078FDF7EDF804B100E06B
:1017D00031BDBDE8314010B50F4C206840B1FDF778
:1017E000A8FB002020600120BDE8104000F0F2BE00
:1017F00010BD80B50948806858B10278431C69461D
:10180000012000F0B8FE20B10078C00701D501200A
:1018100002BD002002BD0000E0470020C0450020BE
:101820005245002054450020E44500205145002049
:1018300053450020DFF800F049980010DFF800F071
:10184000C9560010282808DA4FF6FF72914204D0DA
:10185000CA4A22F81010002070470220704728283A
:1018600003DAC64931F8100070474FF6FF70704731
:1018700070B504460D46C24E1C2200213046FDF7CD
:1018800054F834777577F8F7D5FA01000EBF0121C7
:1018900000211220317070BD10B5B94CE160A0601C
:1018A00010220021FDF716FB012801D1A0680CE0F1
:1018B00010BD10B5B24C606010220021FDF70AFB8C
:1018C000012801D1606800E010BDBDE81040102182
:1018D00006F0F1B8AA48406870472DE9FC41A84DD0
:1018E0000446002695F81E80042C0F4624DA28783A
:1018F000032818BF102054D101F004F928B900F0D2
:1019000029FE10B900F028FE08B1122049E0012C90
:1019100018BF022C1DD1BFB1062200216846FDF779
:1019200004F800F040F838B90622FF216846FCF7B9
:10193000FCFF00F038F808B1022032E006223946F8
:101940006846FCF7C0FF0BE00621684606F0B3F8D6
:1019500006E0032C04D16868694605F0A5FF064639
:10196000884FAC770421387802F006F900202884EB
:101970009EB9ACB1684600F05BF8064668B9032C26
:101980000ED11D20FFF76BFF288448B138784EF642
:101990006022042102F0D6F802E00EB185F81E8024
:1019A0003046BDE8F681062269463846FCF7AFBFEF
:1019B00070B5044600252000714E05D121B10622E4
:1019C00006F11000FCF77FFF307801280CD10125CB
:1019D000200004D102203070FDF7FBFD04E0002060
:1019E0003070204600F0A8F8284670BD38B50024B5
:1019F000E0B10578624A290006D14178837801EB8D
:101A00000321D182C0781076107802280ED10124EB
:101A1000280006D103201070117ED08AFDF74DFBFF
:101A200001E000201070284600F086F8204632BD04
:101A300010B5534CA17F81B10146062204F1240068
:101A4000FCF741FFA07F04F1240100F008F804F145
:101A50002400BDE81040FFF7EDBE002010BD79B1B5
:101A600002000DD04A79012808BF42F0C00006D01C
:101A700002F03F0203284A7102D142F0400048714F
:101A80007047010018BF01210846704770B53C4DF2
:101A90000446287FFF2815D00A20FCF763FF0600C4
:101AA00010D0D020307074700820B0700622A87F4B
:101AB000F07005F12401301DFCF705FF287F314649
:101AC000FCF771FFE87F01280FD12F48006818B19B
:101AD0008068010018BF8047BDE870402948007841
:101AE0004EF66022042102F02DB870BD24488068B3
:101AF00070472348C068006870472148C1680A6879
:101B0000521C0A60007FFF281CBF4FF48041FDF784
:101B100021B870471A48807F704738B50446184D81
:101B200005F11000FFF78AFE05F110001CB9A97F2E
:101B300009B105F1240032BD70B5114D0446287F6E
:101B4000FF2819D00E20FCF70DFF060014D0D0207E
:101B5000307074700020B070062205F11001F01C86
:101B6000FCF7B1FEE88A70813146287E3073287F09
:101B7000BDE87040FCF717BF70BD00006045002055
:101B800034450020E4450020E8450020DFF800F05F
:101B9000259500102DE9F04104468846122740465D
:101BA0004FF6FE7188421646DFF8885908D1A869B9
:101BB00050B30268100027D041462046904720E0ED
:101BC0004FF6FF71884212D1A86938B1026810003F
:101BD00004D0414620469047070005D031462046B4
:101BE00000F0DAFA07000FD12C706E700CE000F0F4
:101BF0006EFE48B10078A04205D131464046FFF75D
:101C0000C5FF074600E003273846BDE8F08110B560
:101C1000044684B000F072F808B9022029E0208858
:101C2000012100F082FE08B9142022E0208800F093
:101C30008DFE042812D1DFF8FC0881894FF6FF726F
:101C4000914218BF112014D121888181618881803F
:101C5000A188C180E1880181218941810020029011
:101C6000019020890090E388A28861882088FDF790
:101C70002FFD04B010BD30B5044685B0208840214A
:101C800000F053FE002836D02088ADF8040000F0A4
:101C900035F8002500281CBFA07A002807D10021B4
:101CA000684600F0CEF9A07AF0B102251CE0912040
:101CB0008DF800008DF803503E208DF801000121C1
:101CC00006208DF80200A088ADF808006088ADF805
:101CD0000600E088ADF80A002089ADF80C008DF808
:101CE0000350684600F0ADF920880022402100F042
:101CF000BAFD284600E0122005B030BD2389E288F5
:101D0000A1886088FDF7CCBB70B50C46DFF82818B9
:101D10000978022918BF0129154601D1122070BD8A
:101D20000DB9022070BD00F0D2FD060001D11420D3
:101D300070BD1CB1307940F002003071102229468C
:101D400006F11800FCF7BFFD2869B062002070BDE5
:101D5000F8B506000C4601D10220F2BD308800F033
:101D6000B6FD050001D11420F2BDDFF8CC070078E4
:101D7000022818BF012803D0A87C082802D10CB182
:101D80001220F2BDDFF8AC77786908B11120F2BDFE
:101D9000B020FDF7C1F8786108B91320F2BDB02278
:101DA00000F0C2FA786931884180A022311D001DFF
:101DB000FCF789FD796902200870A87C796932886E
:101DC00008280CBF012000200B1DDFF870170978D0
:101DD00005F074F906461CB12146284605F047FB7C
:101DE000300018BF00F055FA3046F2BD38B5044651
:101DF0000D4600F06CFD08B9142032BD8DF800507E
:101E00006946204605F066FA32BD38B50022A0B119
:101E100001230624E4B2051915F8015C303D0A2DB2
:101E20000BD203FB05220A256B43641EE5B2002D8D
:101E3000F0D11046BDE8344001E0022032BD30B59B
:101E400005460C4685B0204600F041FD08B9122039
:101E500019E0DFF8EC06854228BF022013D21022D9
:101E600000216846FCF761FD280A8DF801008DF815
:101E70000050280C8DF802002146280E8DF8030032
:101E8000684605F062F905B030BDF8B50546DFF8E3
:101E9000A8060078022818BF01280C461F4601D169
:101EA0001220F2BD0FB90220F2BD284600F00FFD4E
:101EB000060001D11420F2BDF06A08B1FDF739F82F
:101EC0001C213846FCF715FD0100F16201D11320F9
:101ED000F2BDB07C08280AD1069840B1887E0090F7
:101EE00001F112030A8A284605F0ECFA00E000200E
:101EF000317941F004010CB141F002013171F2BDC0
:101F00002DE9F0410D4600F0E2FC04001FD0A5626F
:101F100000F007FA0546C0B200B92578A66A94F821
:101F200005801020FCF71EFD070010D0D02038706F
:101F3000062200207870A11D0920B87087F8038060
:101F4000381DFCF7C0FCFE603946E8B21EE0BDE873
:101F5000F0812DE9F04104460D4690461F460E20C3
:101F6000FCF700FD06000FD0D020307006220020C4
:101F7000707041460C20B070B580B01DFCF7A3FC1A
:101F800037733146204601E0BDE8F081BDE8F041FD
:101F9000FCF709BDF0B50C0087B050D0A079DFF890
:101FA0009465002830690CBF0825042508B9DFF8BE
:101FB00094050778042D08D1DFF88C05006820B15E
:101FC000416808001CBF00208847207D059004F16F
:101FD0000803608A04903946208A0390E0890290C1
:101FE0000195A0880090E279E07800F071F8E0783F
:101FF00080B9172004900122E08903900295002007
:10200000019004F108000090E379A188384600F0BF
:10201000DDFBE070306908B100F056F9307801005E
:102020000DD0717800F0B8F848B1E378312B04D0C6
:10203000A2883178184600F079F80020307007B097
:10204000F0BD10B5044684B0A08851B100210291C2
:102050000191A189009163892289E188FDF7D0FA75
:102060001FBD04B0BDE810403B21FDF7E2BA70B5DA
:1020700004460026A08800F02AFC18B10678A08843
:1020800000F0D7FBDFF8AC542878010007D0864277
:1020900005D1697800F080F848B100202870300040
:1020A00005D0A379A288A078314600F03FF868698E
:1020B00008B100F0EEF8A08800F048FC042802BF48
:1020C000A088A989884204BF4FF6FF70A88170BD1F
:1020D0002DE9F0410646884617461C461620FCF7B7
:1020E00041FC050020D0D02028706E700520A8701B
:1020F000EF702CB106222146281DFCF7E4FB04E01A
:1021000006220021281DFCF710FC0698688129464C
:10211000079828730898E881099828820A986882A5
:102120000B982875404631E7BDE8F081F8B50446C4
:102130000D4616461F460820FCF714FC48B1D02176
:10214000017044700621817086808771014628469F
:10215000EDE0F1BD2DE9F04105460E4617469846E3
:102160000C20FCF7FFFB040014D0304600F0AFFB5E
:1021700008B9DFF8D0030078D021217065700721FD
:10218000A170E570A680E780A4F8088006996181B7
:102190002146FBE6BDE8F08110B50C4600F0ACFB33
:1021A00028B140882146BDE81040FFF7EFBC12205F
:1021B00010BD2DE9F84F0746894692461C46484611
:1021C00000F085FB5FEA000B1EBFDFF8685369690A
:1021D00000295CD051F8A42F182002B134208A685D
:1021E00002B1143004B11C30496801B1173080B21B
:1021F000FCF7B8FB06004AD0182200F095F800F072
:1022000090F85FEA000808BF9BF80080D02030708B
:1022100077700A20B070A6F8049086F806A006F140
:1022200018076969D1F8A40040B1B7603846D1F801
:10223000A41000F11C071C22FCF745FB6969D1F8CA
:10224000AC0040B1F7603846D1F8AC1000F114078B
:102250001422FCF738FB3CB13761384600F11C070B
:102260001C222146FCF72FFB6869D0F8A81031B179
:1022700077611722D0F8A8103846FCF724FB3146C6
:102280005FFA88F0FCF78FFBBDE8F14F01E0BDE895
:10229000F18F10B5A74C6069A8B1D0F8A40008B1BF
:1022A000FCF747FE6069D0F8A80008B1FCF741FED2
:1022B0006069D0F8AC0008B1FCF73BFE6069FCF740
:1022C00038FE0020606110BD10B59A4C206940B105
:1022D000FCF72FFE002020610420BDE8104000F034
:1022E00079B910BDF8B504460D46284600F0EFFA5E
:1022F000060015D000F015F8070008BF3778062053
:10230000FCF730FB06000BD0062200F00DF8D020C1
:10231000307074700E20B070B5803146F8B206E0AF
:10232000F1BD2620FFF79BBA0021FCF7FEBABDE8FD
:10233000F440FCF738BB2DE9F84305460E46174636
:102340009846304600F0C3FA5FEA00091ED010201C
:10235000FCF708FB040019D01022FFF7E5FFFFF798
:10236000E0FF08B999F80000D021217065700F21B5
:10237000A170A680277284F80980C0B20899A17262
:102380000999E1720A99E160214631E0BDE8F183E3
:102390002DE9F84304468846914600F098FA070074
:1023A00024D01420FCF7DEFA05001FD0FFF7B9FF98
:1023B000060008BF3E78D0202870062200206870F2
:1023C000B91D0B20A870E81CFCF77DFA6C8118F091
:1023D0000101C5F8109018BF01212973F0B218F05F
:1023E000020118BF01216973294601E0BDE8F183AC
:1023F000BDE8F443FCF7D7BA2DE9F14F90460D46FE
:102400009946404600F063FA07000A9EDDF82CA0CA
:10241000DDF830B00D9C3ED09DF8000000283AD188
:10242000387940F010005FEA49714CBF40F002007B
:1024300000F0FD00002E08BFBAF1000F08D1BBF17B
:10244000000F08BF002C03D100F0FB00387122E020
:1024500040F0040038713CB12069B8621022214676
:1024600007F11800FCF72FFA3EB135B9F86A08B148
:10247000FCF75FFD1C2130460AE0BAF1000F0AD0DC
:10248000012D08D1F86A08B1FCF753FD1C21504614
:10249000FCF72FFAF862274D6869002842D086B110
:1024A000D0F8A40028B91C20FCF736FD6969C1F8F2
:1024B000A4006869D0F8A40018B11C223146FCF7CA
:1024C00002FABBF1000F11D06869D0F8A80028B952
:1024D0001720FCF721FD6969C1F8A8006869D0F8E8
:1024E000A80018B117225946FCF7EDF98CB16869BC
:1024F000D0F8AC0028B91420FCF70EFD6969C1F8CA
:10250000AC006869D0F8AC0018B114222146FCF781
:10251000DAF99DF8000053464A46414601B0BDE84D
:10252000F04F46E6BDE8F18F0249886170470749E0
:10253000086070471845002051450020E445002000
:1025400040420F0050450020E8450020D4470020BD
:1025500005F0C6B9264800E02648006800B1012011
:102560007047010001D0172801DBFF2801D10120AD
:102570007047002070472DE9F04D0D46934600242A
:10258000BBF1200F80461F462C7003DB0020BDE806
:10259000F08D0419E0B25845F8D2E4B23E5D641CF7
:1025A000002EF3D0E4B231198B45EFDB17F804A00D
:1025B0005046FFF7D6FF641C0028E7D0701EC245C6
:1025C0002870E6D1E4B23819E1E70B490A781043E4
:1025D0000870704708490A7832EA0000087006D18E
:1025E0000648006818B14068010018BF00477047EE
:1025F000E0470020DC470020D7480020D8470020D3
:1026000038B504460D4600F062F9A0B1807C04287C
:1026100001D0122032BD3748006808B190F89950B7
:102620002946684605F073FA334B6A460221204674
:1026300005F0F7FD32BD142032BD80B52F4800787B
:10264000400707D52E48FFF772FF2E494FF6FF705F
:10265000088001BDBDE802400020FFF768BF7CB5DF
:10266000012403280D4610D042F21301884204D001
:102670004FF6FF7188421ED02AE0A8780C2818BFB8
:10268000112826D100F027F823E0E878A9881D4E0C
:102690001A2804BF33889942F4D06A8900922B89A2
:1026A000EA88FFF757FDA8883188884211D14FF694
:1026B000FF7030800DE068790024122809D1ADF850
:1026C0000040297968886A46FCF798FC012400E0FC
:1026D0000024204676BD38B50A4C20884FF6FF7599
:1026E000A84205D008490A780849FCF79AFC2580D9
:1026F00031BD00002C450020EB8101005145002038
:10270000F045002024450020E44500201C45002021
:10271000F8B5124E04463078FF280D4618D005F162
:10272000080080B2FCF71EF9070011D0207838703D
:102730007D80FF2078702A4607F1080078602146E6
:10274000FCF7C1F830783946FCF72DF92846F2BD80
:102750000020F2BD0149087070470000F6460020D5
:1027600038B5AE4C00220021204602F03FFA207816
:1027700030256843FCF7D0FB6060B8B100210AE067
:1027800005FB01F202444FF6FF735380491C0023FE
:102790001371D362C9B222789142F1DB002000218B
:1027A00004EB8002401C0C289160F9DB31BD002154
:1027B0009A4A02EB8102936813B990600020704737
:1027C000491CC9B20C29F3DB132070472DE9F041F5
:1027D00006460C4617469846204600F078F808B1A1
:1027E000112024E04FF6FF7000F071F805001DD0B5
:1027F00085F8058006220699A81DFCF764F80622D4
:10280000002105F10C00FCF790F86C802F712E7000
:102810000020E86200210898A8740998A8820A9804
:10282000E882204600F0E9F8002000E01520BDE82D
:10283000F08110B500F04BF8040012D0608801213F
:1028400000F0DBF8E06A08B1FCF773FB30220021EE
:102850002046FCF76AF84FF6FF7060800020207178
:1028600010BD022010BD38B50C46154600F02FF8FB
:1028700058B10179002D14BF2143A14301710221F8
:10288000408800F0BAF8002032BD152032BD38B5BE
:102890000C4600F01CF8050017D02879207006229D
:1028A00068796070A91DA01CFCF70DF8062205F1DF
:1028B0000C0104F10800FCF706F8A87CA073A88AB4
:1028C0002082E88A6082002032BD012032BD10B52E
:1028D0000022524B00E0521C1C78D1B2A14209D216
:1028E0005968D2B23024544321444C888442F2D1F6
:1028F000084610BD002010BDF0B5484B5C680022B2
:102900004FF6FF7700E0521C19788A420BDA30212B
:1029100001FB02F561194E88BE42F4D0655D854227
:10292000F1D10846F0BD0020F0BD10B50C464FF6C1
:10293000FE71884206D0FFF7CAFF00281CBF00794D
:10294000204201D0012010BD002010BD80B5FFF74E
:10295000BEFF00B1807C02BD10B5002000212F4ACF
:1029600008E05368C9B230244C4323441B7903B1B7
:10297000401C491C1478CBB2A342F2D3C0B210BDA4
:1029800026480078704710B50C46FFF7A0FF0028D6
:102990001CBFC18AA14202D0C482002010BD012008
:1029A00010BD80B5FFF793FF00B1C08A02BD70B5BE
:1029B00005460C461646FFF78AFF28B94FF6FE700B
:1029C000854218D0142070BD0179C06A28B9CA06A2
:1029D00009D5C90609D40F2070BD01F01202102AD2
:1029E000F7D1002EF5D0052070BD20B1807EA04229
:1029F00001D20C2070BD002070BD70B504460D469C
:102A00000026064800EB86008268100002D02946A6
:102A100020469047761C0C2EF3DB70BD204800202A
:102A2000B0494870704710B5AE4C207005F091FC6D
:102A30002078BDE810400521FCF79ABA7CB5A94D75
:102A400028780C46210419D5FCF70CF8060084F40C
:102A5000004411D000F058F858B93078A22806BFC9
:102A6000A14800786878FF2803D03146FBF79BFF28
:102A700002E03046FBF788FF204676BDE10709D526
:102A8000A86820B1416808001CBF0020884784F076
:102A9000010076BDA10709D5686820B1416808002A
:102AA0001CBF0120884784F0020076BD610727D54E
:102AB0008E4E31880A001DD0481E308080B2E0B9A9
:102AC000FFF748FD48B18A4901200870686820B1C5
:102AD000416808001CBF01208847FEF7FBFE6946DD
:102AE00004F0E2FE6846FEF7A3FF1D20FEF7B7FEE6
:102AF000308002E0042101F03FF884F0040076BD4C
:102B0000002076BDFFF728BF38B502780124912A4E
:102B10004FF6FF7102D0A22A76D07BE04278052AD8
:102B200049D00E2A04D00F2A48D03E2A69D071E03D
:102B300082886C4941F20905531B2DD040F6F97586
:102B40005B1B2FD0DB1E31D05B1E08D09B1E022BDF
:102B500005D9DB1E012B15D9DB1E08D05AE04968C8
:102B6000002958D009680A0055D0884750E06149CB
:102B7000096800294FD04B6819004CD0014642F239
:102B80000E003CE08968002945D00B68190042D04E
:102B90000146104698473BE08068411C0078FEF7EC
:102BA00007FF35E08068FEF721FF31E0806800789C
:102BB000FEF76CFF2FE0FFF75AFA2CE0828842F212
:102BC0000D05531B13D09B1F02D09B1F0FD021E07C
:102BD000494B1B888B420AD048490968D9B10A6819
:102BE000110018D0014642F21300904710E041490D
:102BF000096881B14B6819000DD00146104698470D
:102C000006E000F00AF803E00246408800F04BF8C6
:102C1000044600E00024204632BD70B5054601247C
:102C2000A8780128014611D0022806D0032811D027
:102C3000062815D00A2809D032E02A48806880B3D7
:102C4000416808002DD0284688472AE02946FFF72A
:102C5000A1F926E0A8882A4600F025F8044620E0DD
:102C60000E20FBF77FFE06001BD0A8880122402122
:102C7000FFF7F9FDD02030703146E87870701120F0
:102C8000B070A888B080E888F08028893081688991
:102C90007081A889B08114480078FBF784FE00E0B9
:102CA0000024204670BD70B50C461546FFF74EFE59
:102CB0000126042804D11148006858B1026803E0D5
:102CC0000C48006830B14268100003D02946204605
:102CD00090470646304670BD0249886070470149FA
:102CE00048607047E44500205045002054450020CE
:102CF000534500203045002024450020D4470020C3
:102D0000F8B5144600250E46BC4FBD4B40B1012816
:102D100015D0042818D006281ED0072822D02CE071
:102D2000162928DA1622002107F10C00FBF7FDFD19
:102D30003246214607F10C00FBF7C5FD1EE0022ECE
:102D400019D12088388119E0082E14D1384621463F
:102D5000082200F0AFFD11E0012E0CD1DA6903F179
:102D6000280104E0012E06D1DA6B03F14801207836
:102D700000F030F802E0182500E002252846F2BDF8
:102D800010B50B4600249D4920B1012808D0042825
:102D900009D00DE015220C311846FBF794FD08E030
:102DA0000889188005E01846082200F083FD00E03D
:102DB0000224204610BD01460020C90706D50FF2A7
:102DC00048238F4810220721FAF79EBB70478D4990
:102DD0000860704710B50B7884074CBF43F00203BE
:102DE00003F0FD0304064CBF43F0800303F07F03B0
:102DF00004074CBF43F0080303F0F70384064CBFFD
:102E000043F0200303F0DF030B70AA21084203D034
:102E1000107840F00C0003E018B9107800F0F300CF
:102E2000107010BD2DE9F0410F4615463878022884
:102E30001E464FF000085ED1786801784078069C05
:102E400001EB002080B221001CBFB0F5285F0B20F1
:102E500056D14FF42851401A08D0401E1AD0401EB7
:102E600028D0401E1ED0401E2AD044E0F868FBF750
:102E700028FD079A80B2031B9342B8BF021B92B28F
:102E80001019162803DA3280F86801190EE04FF0A5
:102E90000D0834E0F8680088022131802870000AAB
:102EA00068702CE0062030800622F9682846FBF77F
:102EB0000AFD24E001203080F868007828701EE0C8
:102EC000F868B0B108213180018829700188090AA9
:102ED00069704188A9704188090AE970818829715F
:102EE0008188090A6971C188A971C088000AE871DE
:102EF00005E0308003E0A6F800804FF0010840466E
:102F0000BDE8F0812DE9FC4B0E4680463078002765
:102F1000022891461D466BD17068017840780A9C62
:102F2000DFF8E0B001EB002080B24FF42851401AE6
:102F300006D0401E29D0401E4CD0401E38D057E04D
:102F4000F068FBF7BEFC80B2A04204D32919162911
:102F500003DB0D274DE007274BE0F3682A4649467F
:102F60001819FBF7B0FC2C19F068A4B2C4F11602D2
:102F700000212044FBF7D9FCDBF80000002838D002
:102F80000268100035D0002121E07CBB022DE0D189
:102F900099F8000099F8011000EB0120F168088011
:102FA000DBF8000028B30268100022D001210EE0F7
:102FB000E4B9062DCDD1F06806224946FBF783FC23
:102FC000DBF80000A8B10268100012D003214046CF
:102FD00090470EE054B9012DBBD199F800000100D3
:102FE00013BF0128F1680870802702E00B2700E07A
:102FF00001273846BDE8F68B000000000C46002093
:10300000304600201C480020252E0100052F01001D
:1030100000000000F8B505460C46AF892FB3AA683A
:10302000167830060FD50D2F1FDB0C3FBFB2D0191D
:1030300000903B466888012104F0DAFD002814BFA7
:103040000220012000E000202070B00900F0010003
:10305000607006F03F00A070781EA08080B208B1BA
:10306000A868401CA0600020F2BD0120F2BD0A78D3
:1030700002704A8842704A88120A8270097918E1FF
:1030800004290AD1017811708378417801EB03217A
:103090005180C0781071002070470420704705E00F
:1030A000022B00D1D5E00420704700BF0A880270CF
:1030B0000988090A417002207047022906D1017867
:1030C000407801EB002010800020704704207047FA
:1030D000E6E0042B00D1F4E0042070478A78027007
:1030E0008878098801280CBF042012204843401C1E
:1030F00080B2704710B50B001CD00378491E012B1D
:1031000089B207D14B0801EB93739B08B1EB8304A1
:1031100010D108E0022B0DD1122391FBF3F31224FE
:1031200004FB131131B999B221B110F8011B917050
:1031300013800FE1042010BD10B50C46022200F0F0
:1031400047F8001D611DFBF7BEFB2089801D80B282
:1031500010BD70B51E46062E144619DB049D20785E
:10316000617800EB012028800222A078E17800EB52
:1031700001206880211D02202871681DFBF7A3FB38
:10318000B01F288180B200B1A01DE860002070BD92
:10319000042070BD08888004000C70474B0801EBC8
:1031A00093739B08B1EB830303D1890801D011808D
:1031B0009AE00420704710B50C4600F009F8611D34
:1031C0002279001DFBF77FFB2079001D80B210BD26
:1031D000218801702188090A4170618881706188A5
:1031E000090AC170704710B5029C062B104612D117
:1031F000022121714278017801EB02212180C278FD
:10320000817801EB02216180011D2279601DFBF7AD
:103210005AFB002010BD142B08BF1021E9D0042058
:1032200010BD7CE010B50B000BD003785380491E15
:10323000022B89B205DB91FBF3F403FB141101B9F6
:1032400086E0042010BD31E7022B00D101E004200C
:1032500070471078517800EB012000990880002019
:103260007047088870473CE010B5022B0FDB029CCA
:10327000207261721078517800EB01202080981E36
:10328000608080B200B1901C6060002010BD0420FE
:1032900010BDB2E009B9002070470420704700BF9C
:1032A0000A8802700A88120A42704A888270498825
:1032B000090AC17004207047042B00D101E00420EA
:1032C000704700981178537801EB032101809178C1
:1032D000D27801EB022141800020704708887047B6
:1032E00000BF118001B9002050600020704788881D
:1032F0004004000C704703EBD3704008B3EB400070
:1033000007D15908022904DB00988180026000205F
:1033100070470420704708887047E2E700BF4A887A
:1033200009880270514389B2481C80B2704710B5B9
:103330000B000BD003785380491E042B89B205DBA8
:1033400091FBF3F403FB141101B901E0042010BD5B
:103350001480401C5060002010BD14E010B5042BF8
:103360000EDB00F062F8D478917801EB0421418003
:10337000191F818089B201B1111D8160002010BD2B
:10338000042010BD00BF0A8802700A88120A427029
:103390004A8882704A88120AC2708888001D80B2EA
:1033A000704710B5042913DB03784478091F03EB39
:1033B00004231380C4788378918003EB042389B2BB
:1033C000002914BF001D002090605380002010BD14
:1033D000042010BD0978017001207047012B04D131
:1033E000009910780870002070470420704709B9D0
:1033F000002070470420704700BF0A8802700A88C6
:10340000120A42704888801C80B2704710B5022BA7
:1034100009DB00F00AF8991E418089B201B1911CC4
:103420004160002010BD042010BD0298117854782E
:1034300001EB04210180704709B900207047042086
:1034400070472DE9F04784B080460C9D0C469146AC
:103450009A4655B91720FDF75BFA0126050005D1FC
:103460001324204604B0BDE8F08700262846012733
:1034700000F8019B14B15146A047471C5FEA096060
:103480000DD510214046FFF750FAD8B9BFB2EA195E
:103490003946284604F05FFB044668B90C3704201F
:1034A000ADF800000195ADF8087069464046FBF79D
:1034B00074FD00280446D4D0002ED2D02846FDF753
:1034C0004CFACEE71924F7E730B5022918BF1029C6
:1034D00085B00446154603D1022B18BF102B01D02E
:1034E000002017E00A469A4203D12946FBF70FFA5B
:1034F00010E01029694606D1284600F00DF8102288
:103500006946204604E000F007F810226946284684
:10351000FBF7FDF905B030BD38B504000D4618BF06
:10352000002D0BD010220FF264012846FBF7CBF9D7
:103530002078287360786873012032BD002032BD86
:1035400038B504464FF6FE7084420D460BD0172D59
:1035500009DBFBF7B8FD2946884204D32046BDE8C5
:103560003440FFF710BA012032BD80B54FF6FE712E
:10357000884205D0FFF715FA010005D1172002BDDA
:10358000BDE80140FBF79FBD02BD0000FB349B5F1F
:10359000800000800010000000000000784B1988B7
:1035A000FF2905D1188078220021181DFBF7BDB92D
:1035B00070472DE9F04104460D46280448BF85F4C4
:1035C000004030D428002DD06E48006880478046E7
:1035D0002F46002025FA00F1C9071AD568490A8844
:1035E000121BC2EB0212821801EBC2010F1D012156
:1035F00001FA00F6396808001CBF78688847B1B244
:10360000204600F0CEFA08B93860786086EA0507EF
:1036100002E0401C0F28DDDB5B4909684046884713
:10362000B8B200E00020BDE8F08110B582B00024FF
:10363000FFE7009400F05CF816BD2DE9F047044662
:103640005048514F0068884680470F2C824620DA48
:103650004B4D05EBC4004068D8B10F2094FBF0F946
:10366000C9EB09110120611A00FA01F628884844C3
:10367000B1B2C0B200F095FA58B128884844424629
:10368000B1B2C0B200F046FA39685046884700200F
:1036900003E03968504688470220BDE8F087F8B556
:1036A00004463848384E006880470F2C05461ADA21
:1036B000334800EBC4077968A9B10F2194FBF1F2FC
:1036C000C2EB021300880121E31A9940801889B2E5
:1036D000C0B200F051FA00207860B8602846316826
:1036E00088470020F2BD3168284688470220F2BD95
:1036F0002DE9F44F80462348234C006889461E4636
:10370000804783465FEA080004D12168584688470D
:10371000022031E00025DFF868A00AEBC5077868D1
:1037200018BB9DF82800009A01280CBF174B184BB6
:103730000F2095FBF0F0C0EB001E4FF0010CA5EB45
:103740000E010CFA01F1BAF800C0604489B2C0B2AF
:10375000984750B9C7F80480C7F8089006B135708B
:10376000216858468847002006E06D1C0F2DD4DBE9
:103770002168584688470820BDE8F28F0000000005
:103780009C440020A0470020A4470020453B0100A6
:10379000153B010038B54FF6FF74A0420DD1002053
:1037A000164A137898420EDA21F8204001EB800582
:1037B0000023401CAB70C0B2F3E700F00BF810B16F
:1037C00004800021817031BD80B500F003F800B1A4
:1037D000807802BD10B5002200E0521C074C24780E
:1037E000D3B2A34207D2D2B231F822308342F4D10D
:1037F00001EB820010BD002010BD00002048002019
:1038000070B514461D4600F01CF8064608480068CE
:10381000804703E016F8011B04F8011B29464D1EE2
:1038200089B20029F6D1BDE870400249096808470D
:10383000A0470020A44700200B460146184600F090
:1038400010B81D2290FBF2F21D2303FB120001F5BC
:10385000E83101EB0030704780B5084909684969D3
:1038600005E080B5054B1B689B69984700E08847D9
:10387000034A0021116002BD00000000A8010010F1
:103880008404604202000A4A08BF0FF2210050601F
:10389000517070477047064A010004BF51780129F2
:1038A00002D011785268104770470000704700003E
:1038B0007044002062B38B0708D0521E11F8013B00
:1038C00000F8013B00F024808B07F6D1830740F01D
:1038D000208000BF103A07D330B4B1E83810103A56
:1038E000A0E83810F9D230BC530724BFB1E8081063
:1038F000A0E8081044BF51F8043B40F8043BD2074D
:1039000024BF31F8022B20F8022B44BF0B78037040
:103910007047083A07D3B1E80810083A40F8043B6A
:1039200040F804CBF7D25307E4E70000030000207F
:1039300013F0030F09D0521E22BF13F8010B11F828
:1039400001CBB0EB0C00F3D07047121F22BF53F82D
:10395000040B51F804CB6045F7D0121D0AD200BA0F
:103960009CFA8CFCB0EB0C0038BF6FF0000088BFF5
:1039700001207047521E22BF13F8010B11F801CB32
:10398000B0EB0C00F6D0521C08BF10467047000088
:10399000006801074CBF042000F0030070470000DE
:1039A00000F10103810704D010F8011B89B18107E0
:1039B000FAD10268B2F10131914311F0803F04BFA6
:1039C00050F8042FF6E710F8011B11B110F8011B95
:1039D000FBE7C01A7047000062F30F2262F31F4238
:1039E000401810F0030308D0C91A1FD3DB0748BFE3
:1039F00000F8012D28BF20F8022D130030B4144622
:103A00001546103928BF20E93C00FAD8490728BFDD
:103A100020E90C0048BF40F8042D890028BF20F899
:103A2000022D48BF00F8012D30BC7047C91818BFDF
:103A300000F8012DCB0728BF00F8012D70470000CA
:103A400000B583B00820ADF8000012209C49096839
:103A5000ADF802006846884701980EBD10B5994C34
:103A60000020A060FFF7ECFF606010BD70B5044659
:103A70000D46164600F018F808B1466070BD1020DB
:103A8000FBF74AFA78B18472058146600021016033
:103A9000C1608C490A6812B9086070BD0A46116895
:103AA0000029FBD1106070BD864A12682AB11389C3
:103AB0008B4204BF937A8342F7D11046704708B116
:103AC0000021018170472DE9F041FFF7B9FF7D4EDC
:103AD0007D4977680C68C51BB4F57A7F14D0A4FBC8
:103AE00005014FF47A72002304F0E4FF4FF47A7872
:103AF000A8FB0023054608FB013310461946224661
:103B0000002304F0D7FFC01970602846BDE8F041DB
:103B100005F048B8F8B504466A4800680D461646F0
:103B200008B9FFF7D0FF69480068804700F01FF828
:103B300000F048F80446384688470CB10020F2BD32
:103B40000820F2BDF8B50446604800680D461646E8
:103B5000804700F00CF804005D4918BFE660096872
:103B6000384688470CB10020F2BD0820F2BD074658
:103B700032462946204679E770B500F026F8064619
:103B800029462046FFF790FF040018BFFFF797FF74
:103B900000F018F8304688470CB1002070BD0620B0
:103BA00070BDF8B500F011F8074629462046FFF72A
:103BB0007BFF002600B1466800F004F838468847CD
:103BC0003046F2BD42490968704704463F480068E4
:103BD0000D4600472DE9F147DFF8F080394DD8F860
:103BE0000000DFF8ECA081B080470246A868019988
:103BF0000818A8601046DAF8001088472E68002ED2
:103C00004DD00027D8F8000080478146BDF8060057
:103C10000024002804BF9DF80500002807D1307952
:103C20009DF80420904202D3801A307106E070683B
:103C3000019981423ABF401A70607460B08858B9E7
:103C4000F08858B9F06868B1318908000AD0B07AB4
:103C5000FAF780FFF0687060B08808B9F08808B1A2
:103C6000308930B93068002F0CBF28603860344686
:103C700000E037463668DAF800104846884764B1F5
:103C8000A088002804BFE088002803D12189A07AF9
:103C9000FAF760FF2046FBF74CF9002EB2D1BDE8E1
:103CA000F3870848016841B10A484A6809688242B6
:103CB00098BF10460029F8D17047002070470000D7
:103CC0009C470020C047002088440020A0470020D7
:103CD000A44700208EC2F52800B583B00821ADF8B6
:103CE00000108DF804001721ADF8021068461D4938
:103CF000096888479DF805000EBD1B48002181809A
:103D00000121017070472DE9F0410D4617490978EE
:103D100001248842064602D2134F387808B90120A0
:103D20001DE01348006880478046B88804FA06F60C
:103D30004DB920EA0601B98060B159B90020FFF7FA
:103D4000CBFF044606E010B90120FFF7C5FFB88895
:103D50003043B88040460749096888472046BDE897
:103D6000F08100009C470020B84700202C9B0000F9
:103D7000A0470020A447002030B585B01446082293
:103D80000291ADF80020002238490968ADF804001E
:103D9000ADF802201D46684688479DF80C1021703A
:103DA0000499296005B030BD1CB51220FBF7B4F8AA
:103DB0002F49086012220021FAF7B7FD002000F019
:103DC0001DFC012004F07EFA0220FFF7E7FB032030
:103DD00004F018FF0420FEF726FE052005F068F821
:103DE0000620F8F754FB0720F9F748FB0820F6F700
:103DF000A5F801AB6A4600211020FFF7BDFF9DF832
:103E000000100820FAF79DFD00249DF800102046C0
:103E1000FAF79FFD641C082CF7DB13BD10B582B0C8
:103E200005F0BAF8134B144A14495020FFF7A4FFC9
:103E300060B10520FFF72FFD0820ADF800000C2031
:103E40000A490968ADF80200684688470C480068CE
:103E500080470446FAF7E0FCFAF7E4FE09490968EE
:103E600020468847FAF714FF002016BD9C47002023
:103E7000B447002084440020D64800204BED0000C9
:103E8000A0470020A4470020DFF800F03DAC001060
:103E9000DFF800F089D10010DFF800F0C9B400109D
:103EA000DFF800F019570010DFF800F0618400100F
:103EB000DFF800F08D670010DFF800F041B500106A
:103EC000DFF800F055B50010DFF800F0BD800010FD
:103ED000DFF800F01DB50010DFF800F02D8A0010AB
:103EE000DFF800F071940010DFF800F0E5730010C7
:103EF000DFF800F035A30010DFF800F0E1AC0010AF
:103F0000DFF800F0FD750010DFF800F0EDAB0010F9
:103F1000DFF800F065860010DFF800F0298400105B
:103F2000DFF800F0B9860010DFF800F095D6001039
:103F3000DFF800F00DB50010DFF800F0B5770010E5
:103F4000DFF800F0F182001080B54FF49E720FF29E
:103F50003001DFF88C0CFFF7BDFCDFF8880C002186
:103F600001700122DFF8801C0A7302220A70DFF858
:103F7000201DC0F80D10DFF8901EC0F82D1001BDF7
:103F8000990400211905002179040021F0B5174C8E
:103F900040216118C878022805D009480021016035
:103FA00008498847F0BD256E074E356060072843F5
:103FB0002066276824600E48804727603560F0BD82
:103FC0002C110440A56500002840044010B5074CA2
:103FD000A17D002905D10121A175480204493E397E
:103FE00088472068002800D0804710BD5402002177
:103FF0008B39000010B50549054A72B6C87801280A
:1040000002DC01204870121D62B6104794020021A4
:104010006D470000F8B51A4E0546316B1948CC09BA
:10402000E401002D11D01849097802290FD0007B36
:10403000044372B60120154F4002B847114820389A
:104040000088C109C90704D016E0C07AF0E7407BB8
:10405000EEE70F493463CC61400AC0070CD0012061
:104060008003F16A002D01D0014300E0814308463E
:10407000F1620749403948630020B84762B6F8BD8D
:10408000800200218800002196020021DF3C000010
:10409000404004400749002800D00420064A72B678
:1040A0000978C90701D0105800E0802062B640B2FC
:1040B000704700006B020021586004402DE9F04178
:1040C0000FF24C00DFF8641E2722036844688568FD
:1040D000C6680769D0F814C0D0F818E0D0F81C8082
:1040E0000B604C608D60CE600F61C1F814C0C1F8E8
:1040F00018E0C1F81C8020302031521EE5D1426802
:104100008368006808604A608B60BDE8F081000049
:10411000546100007F140200060005000F00080033
:104120004800520080FF3F00000000000000000037
:10413000000000000000000030400040014003404B
:1041400007400F404F40CF40CF41CF43CF47CF4FE5
:10415000CF3FCF2FCF1FCF0F000000000000000087
:1041600000000F00080000003F00000040003F007A
:104170000000040068000E00DC00060043001A0086
:104180000500000000000200000000000000000028
:104190000400C00000000400C00000000700000090
:1041A000000000000000000000000000000000000F
:1041B00050C00091007070C00091007082312100E9
:1041C000319110B10070018101B100A182313291B1
:1041D00010B101911110418141226340F10600703C
:1041E00051C0019130181039833108D01831416F16
:1041F0003100319110B1831414166F6800702510CE
:1042000050C00091F4C340C12014036F3110410429
:104210005082F0228440512622C082312100319107
:1042200010B163393110410482C0823121003191D3
:1042300010B163393110A2C082312100319110B127
:1042400050101531051405920070536452C031109E
:1042500031066131C102566412C131102139710633
:104260005131E1025664007051C0019101CCE2C0AD
:104270005664536411C1C2C0566454B0007154A056
:1042800064B0F0800022B54011C122C1566451C013
:104290000191E2C0823160820200329110B100C30C
:1042A000C86853644012B09032B000C3CE6840C2B8
:1042B000D0688012B09032B00070536401C122C146
:1042C000566401C1C2C0566453829D64C012B0904E
:1042D00032B00070536472C281C0566422C111C1F1
:1042E000566402C011C1566462C031C3566462C3D1
:1042F00011C1566402C311C15664538253399D647F
:10430000E2C35B641122F84042C281C8566452C2C3
:1043100011C1566472C2E1CE566402C281C85664AD
:1043200002C201C85664B0C00C690070536442C236
:1043300001C8566452C211C0566472C2E1C05664CC
:1043400002C001C1566462C001C3566422C101C1EA
:10435000566462C301C1566402C301C156645382EC
:104360009D64007002C1623101C0A080001E324114
:10437000101A34612010101A136F236E11161216C2
:1043800034690070E092D08200223B45C0B20070D8
:10439000000000000000000000000000000000001D
:1043A000000000000000000000000000000000000D
:1043B0000000000000000000067305720B720E7210
:1043C00050B00071818060B050A09280F0EFF19207
:1043D00002933A65412278458080F1C1100430167D
:1043E00001110114016C8B618C618D618E618F6193
:1043F0009061916193619561976199617062736257
:104400009180F2C0210421318280422A1214321696
:1044100001112114016CA661C761AC617362A661D0
:10442000C761AC6173629B619B619B619B619B6196
:104430009B61AC649B61D5649B61E2649B610E658A
:104440009B612A659B618280E0DFF2923A65B0B0A1
:10445000A261B1B00673057230B05861D0CF3A6531
:1044600084C203C0C0C368649078509160781031F2
:10447000617810140092507840316178100040311A
:10448000717810001092B078609281782192307823
:10449000403141781000309210C0F0919B6154A0DF
:1044A000F0805022CF45408000226646C76100C898
:1044B0006091598150B0918041222E46C0CF3A651B
:1044C0001282823182394239281077641282F112C5
:1044D00012042F101F312F1440C120140D6F6D399D
:1044E000DE10F4C34E0482C082312E006D39A2C0AA
:1044F00082312D001A828A392082803180390BC0A6
:104500000B18AC7830824039021011C0013010C055
:104510000118021882312100C126919103B013B015
:1045200063B053B003823914418001226646B481DE
:10453000C491D5819518B51C1C4EC51C544A659173
:10454000F08010220C422C623D9110B13E9110B1CE
:1045500065910F925981F914AB18BC10F08050226C
:10456000C74110222C460C62B0CF3A6563B030824E
:104570000010F2C02004021011C0013010C0011858
:10458000021882312100C1269191919113B003B09C
:1045900063B053B064B054B00071418001226646EC
:1045A00063B064B0F0805022C741B181C191D18124
:1045B0009118619131B0446212828231823942395C
:1045C0002810776459810582591420820BC00B187A
:1045D000AC7880C0007163B0626A0C620182628153
:1045E0008231823DA0EFF19202933A6503A09B6174
:1045F000A28077649B6150B000719B612DE9F04F00
:10460000DFF8F44ADFF8F45A2070072100206862CE
:1046100083B0DFF8EC0A01700D21418040F22221C5
:104620008180DFF8E00ADFF8D41BA9628A7E02707D
:10463000FF2ACB7E437008BFFF2B0E7F86704F7F13
:10464000C77091F81EC080F804C0C97F417116D1AF
:10465000FF2E08BFFF2F12D1BCF1FF0F08BFFF29AB
:104660000DD1DFF8C41B0A7802704A7842708A784C
:104670008270CA78C2700A79027149794171DFF893
:10468000D41B0278DFF8D08BDFF8D07BDFF8D06B5B
:104690000A70002342784A704FF0180A82788A70B4
:1046A000C278CA7002790A714079DFF8B82B487174
:1046B000FF20DFF8B41B087048708870C87008715C
:1046C000487101212970111D0B708B725A32A02381
:1046D0008B81087103238B7348710723CB73887117
:1046E00000230B74C87128234B82087201230B75B9
:1046F000487200238B75537001234B751370002291
:10470000DFF8681B2B720A710023CA810B754FF406
:104710002072012300F00FF90A824A824B75DFF8FC
:10472000501B00F008F98B7300200871C873888251
:104730000A8205204A8288750020DFF8381BDFF8DE
:10474000383B0880D8F82C104878A8710878387061
:10475000C01C8A782A710AFB00F08A681279521EFE
:104760001A7080B2CA786A71CA686A618969DFF8AA
:104770000C2BE9614FF496711180FAF7CDFBB06014
:1047800008B900F09CB83878010000F09B804FF425
:104790009071484380B2FAF7BFFBDFF8E49AC9F89A
:1047A000040008B9B06888E038788001FAF7B4FBF3
:1047B000A86120B900F0BCF8D9F804007DE0387891
:1047C000FAF7AAFB286228B900F0B2F800F0ACF8BA
:1047D000A86972E038780AFB00F0FAF79DFBDFF871
:1047E000A4AACAF8000038B900F0A2F800F09CF8BA
:1047F00000F097F8286A60E03878DFF8FCBB4001E9
:10480000FAF78AFBCBF8000050B900F091F800F0FD
:104810008BF800F086F800F07DF8DAF800004CE044
:1048200038780001FAF778FBDFF8D01B086060B930
:1048300000F07EF800F078F800F073F800F06AF805
:1048400000F06BF8DBF8000037E038780001FAF789
:1048500063FBDFF8AC1B086080B900F069F800F07A
:1048600063F800F05EF800F055F800F056F8DBF859
:104870000000FAF75EFBDFF8840B1DE0387830218A
:104880004843FAF749FBDFF87C1B0860D0B900F019
:104890004FF800F049F800F044F800F03BF800F061
:1048A0003CF8DBF80000FAF744FBDFF8500B006837
:1048B000FAF73FFBDFF8480B0068FAF73AFB4FF4D2
:1048C000804122E000F0C6FB07460820ADF800005A
:1048D0001E20ADF802004FF40050DFF8F81B096805
:1048E00001906846884704F091FBD8F80C0069797C
:1048F00000880843DFF83C1D0880384600F080FA45
:10490000884700F078FA4FF400512078FAF722F93E
:10491000BDE8F78F286AFAF70CBBDAF80000FAF75F
:1049200008BBA869FAF705BBD9F80400FAF701BB80
:10493000B068FAF7FEBA087248728872C8720873D3
:104940004873704770B50C46E00788B00DD5FFF787
:104950009BFA38B100218160DFF88C0B0068010000
:1049600018BF804784F00100A8E0DFF89057DFF817
:104970001029A86923074FF4907121D55268DFF8F8
:10498000F0385B7D594311440022069200EB8310FE
:10499000CA8E120905928A8E04924A8E5208039298
:1049A00000220292019200F134020092002290F85B
:1049B00030308979002001F092FC84F008007DE01D
:1049C000E30610D500200690059004900390029015
:1049D00001900090002300220021022001F07FFCC2
:1049E00084F010006AE0A30707D500F069F83C20C6
:1049F00001F075FC84F0020060E0630721D56B785C
:104A000052685943114400EB8312881D11F82C3F62
:104A100006934B891B090593838B0493C988490826
:104A2000039100210291019102F13401009192F869
:104A3000303001780122002001F051FC84F00400A4
:104A40003CE0200607D500F03BF83B2001F047FC96
:104A500084F0800032E0A00508D5DFF8B00C0168D2
:104A600041F00041016084F4007027E0600504D546
:104A7000FAF7F2FE84F4806020E0600405D581201E
:104A800001F066FD84F4804018E0A00415D54FF0D5
:104A9000FF30686205F03FFA6E69366805F13C0345
:104AA00005F1500205F12C0105F16800B0472861BD
:104AB00000F012F884F4005000E0002008B070BD4F
:104AC00000200690059004900390029001900090C1
:104AD0000023012200217047F8B5DFF82046DFF8F7
:104AE000A05763692069DFF87467183300221B68D8
:104AF0004FF0FF319847DFF86007DFF83C1BC06AD2
:104B0000806840790870002705F029FADFF8000C6A
:104B1000FFF7BEF9FFF7C0F9FFF7C2F9DFF8F40BB2
:104B200000210170017141718171C1710172417285
:104B30000022DFF8300700F10E010A70A0224A803F
:104B400007224A7103220A7100220A738A7200F84E
:104B5000592F0122CA720021427081700020DFF8B3
:104B60000C178873DFF80817C8730BE068684FF4F8
:104B70009071794308444179012908BF04F090FD00
:104B80007F1CFFB230788742F0DBFFF78DF9A07908
:104B9000DFF8841B087005F0E1FC04F09EFBDFF8F1
:104BA0007C1B00200870DFF8781B08700120DFF8FC
:104BB000741B08700020DFF8701B08700120DFF8FC
:104BC0006C1B08700020DFF8681B0870DFF8641B9E
:104BD0000870DFF8641B0880DFF8641C0870F2BD01
:104BE00004040021A30300216C0300212DE9F041FE
:104BF0001446DFF8685608B12A780270DFF880861C
:104C000011B198F801000870002C3DD00026002753
:104C10001CE0C9B2DBB2605402F130000179E1540A
:104C2000591C427900F036F8827900F033F8C279E5
:104C300000F030F8027A00F02DF8427A00F02AF8FD
:104C40000078C9B24E1C60547F1CFFB2287887429E
:104C50001ADA3846FFF72CF90028F5D1D8F8040005
:104C60004FF490717943F6B20844DFF890148969E3
:104C7000A75501EB871200680078711C4B1C802837
:104C80000CBF00200120C4E70020BDE8F081000037
:104C900011040021C9B26254491C704738B500F0B4
:104CA00040F8010009D1DFF854048069A901405897
:104CB0000A21B0FBF1F02080002032BD38B500F0B1
:104CC00030F801002CD1DFF8B805DFF83024406857
:104CD000926900F0C1F8811D0B7802EB8315220068
:104CE00007D0CB8D898D5B1C4900E20059438A4275
:104CF00001D2122032BD0A216143296090F892004E
:104D000068B100F0A7F904460020687128684108DE
:104D1000A879FEF792FC00F073F82046884700203F
:104D200032BD05460C46FFF7C3B82DE9F8435FEAEC
:104D30000109144618BF002C06461D4600D00DB9C7
:104D4000122056E0FFF7B4F8010052D101F0C0F88C
:104D5000461830680078802818BF0C2049D106F129
:104D6000E307B87DC00758BF112042D5B87C0128A1
:104D700008BF3A203DD000F06DF980460120B8749C
:104D8000002019F800103218401C082882F8AC10D6
:104D9000F7DB06F1B40021780170617841700020E2
:104DA0004242295C3244401C102882F8E210F7DBB2
:104DB00006F1A400FFF780F806F19800FFF780F8ED
:104DC00000F019F8002086F866003870787096F8C0
:104DD0009200012802D178730A2102E00020787342
:104DE00003213046FFF770F800F00AF84046884784
:104DF0000020BDE8F2830C21DFF88C0CFFF768B8C7
:104E0000DFF8881C096870475104002138B50C0090
:104E1000054601D1122032BDFFF74AF8010017D133
:104E200000F017F801680978402901D00C2032BD44
:104E300000214B42625C0344491C102983F8E220A4
:104E4000F7DB012180F8E410052104F0BCFC002010
:104E500032BDDFF82C0440684FF490716943084478
:104E6000704710B50446FFF723F8010016D100F093
:104E70003CF801680978402901D00C2010BD00F1F0
:104E8000F0010A78012A03D106220A77022102E002
:104E900006224A700D2104F096FC002010BD10B5CA
:104EA0000446FFF705F801001ED100F01EF800F1DE
:104EB000F8010A78022A06D1817900F1F90200206E
:104EC00001F0CEF80FE002681278802A08BF0821AE
:104ED00007D0402A07D14978090701D4112010BD15
:104EE0000E21FEF7F1FF002010BDDFF894034068AB
:104EF0004FF4907161430844704710B5040001D12C
:104F0000122010BDDE48407808B10C2010BD04F01E
:104F1000E4F9DFF87C0B2278417811404170627827
:104F2000817811408170002010BD000000C0002178
:104F300038B50C00054605D0C749C96A89680979A2
:104F4000884201D3122032BD05F040F8DFF8E806B0
:104F5000057001202070002032BDBF4AD26A9268DD
:104F60001279904201D312207047C3490870002083
:104F7000704710B5140018D011B1012908D014E001
:104F800005F04CF810F1800F20700CD1302010BDCE
:104F9000B148C06A80680168007900EB40000844AD
:104FA00010F8030C2070002010BD122010BD2DE958
:104FB000F8430C0005469046994605D05FEA090083
:104FC00018BFB9F1010F01D0122041E04B4F3879E1
